:020000040800F2
:1000000000060020E1010008B10E0008310E0008D2
:10001000890E0008310E00085D0E0008E30100089B
:10002000E3010008E3010008E30100088121000862
:10003000E3010008E3010008E3010008E301000810
:10004000E3010008E3010008E3010008E301000800
:10005000E3010008E3010008493200087532000896
:10006000A1320008CD320008F9320008E30100088F
:10007000E3010008E3010008E3010008E3010008D0
:10008000E3010008E3010008E3010008E3010008C0
:10009000E3010008E3010008E3010008253300083C
:1000A000E3010008E3010008E3010008E3010008A0
:1000B000BD300008E3010008E3010008E301000887
:1000C000E3010008E3010008E3010008E301000880
:1000D000E3010008E3010008E3010008E301000870
:1000E0008D330008E3010008E3010008E301000884
:1000F000E3010008E3010008E3010008E301000850
:10010000E3010008E3010008E3010008E30100083F
:10011000E3010008E3010008E3010008E30100082F
:10012000E3010008E3010008E3010008E30100081F
:10013000E3010008E3010008E3010008E30100080F
:10014000E3010008E3010008E3010008B928000802
:10015000E3010008E3010008E3010008E3010008EF
:10016000E3010008E3010008E3010008E3010008DF
:10017000E3010008E3010008E3010008E3010008CF
:10018000E3010008E3010008E3010008E3010008BF
:10019000E3010008E3010008E3010008E3010008AF
:1001A000E3010008E3010008E3010008E30100089F
:1001B000E3010008E3010008E3010008E30100088F
:1001C000E3010008E3010008E3010008E30100087F
:1001D000E3010008E3010008E3010008E30100086F
:1001E00002E000F000F8FEE772B63A4880F30888B3
:1001F000394880F3098839484EF60851CEF200019B
:10020000086040F20000CCF200004EF63471CEF2ED
:1002100000010860BFF34F8FBFF36F8F40F2000003
:10022000C0F2F0004EF68851CEF200010860BFF334
:100230004F8FBFF36F8F4FF00000E1EE100A4EF6C4
:100240003C71CEF200010860062080F31488BFF3F1
:100250006F8F02F015F801F0F1FF02F093FE4FF0FE
:1002600055301F491B4A91423CBF41F8040BFAE745
:100270001C49194A91423CBF41F8040BFAE71A495C
:100280001A4A1B4B9A423EBF51F8040B42F8040B2A
:10029000F8E700201749184A91423CBF41F8040B87
:1002A000FAE701F0CFFF02F0C1FE144C144DAC424E
:1002B00003DA54F8041B8847F9E700F041F8114CC1
:1002C000114DAC4203DA54F8041B8847F9E701F0FA
:1002D000B7BF000000060020002200200000000838
:1002E0000000002000060020B8370008002200208F
:1002F0004022002040220020A82D0020E00100081C
:10030000E0010008E0010008E00100082DE9F04FDD
:100310002DED108AC1F80CD0C3689D46BDEC108A43
:10032000BDE8F08F002383F311882846A047002002
:1003300001F034FBFEE701F0AFFA00DFFEE700005A
:1003400038B501F0EDFE054601F010FF0446D8B9BE
:100350000F4B9D421AD001339D4218BF044641F213
:10036000883504BF01240025002001F0E3FE0CB114
:1003700000F076F800F032FD00F0A4FB284600F013
:10038000C3F800F06DF8F9E70025EDE70546EBE767
:10039000010007B008B500F067FBA0F12003584248
:1003A000584108BD07B541F21203022101A8ADF87A
:1003B000043000F077FB03B05DF804FB38B5202370
:1003C00083F311881748C3680BB101F06DFB164A1F
:1003D000144800234FF47A7101F02AFB002383F3C1
:1003E0001188124C236813B12368013B23606368B2
:1003F00013B16368013B63600D4D2B7833B96368BB
:100400007BB9022000F05AFC322363602B78032B67
:1004100007D163682BB9022000F050FC4FF47A73C7
:10042000636038BD40220020BD0300085C2300202B
:1004300054220020084B187003280CD8DFE800F085
:1004400008050208022000F027BC022000F012BCC0
:10045000024B00225A607047542200205C23002087
:10046000244B254A10B51C461968013140D004338D
:100470009342F9D16268214B9A4239D9204B9B684B
:1004800003F1006303F580339A4231D2002000F07B
:1004900033FB0220FFF7CEFF1A4B1A6C00221A64BE
:1004A000196E1A66196E596C5A64596E5A665A6EEC
:1004B0005A6942F080025A615A6922F080025A61F8
:1004C0005A691A6942F000521A611A6922F0005200
:1004D0001A611B6972B64FF0E0232021C3F8084D62
:1004E000D4E9003281F311889D4683F308881047D0
:1004F00010BD00BF0000010820000108FFFF000838
:1005000000220020003802402DE9F04F93B0AA4BA2
:1005100000902022FF210AA89D6800F009FCA74A4C
:100520001378A3B9A6480121C3601170202383F377
:100530001188C3680BB101F0B7FAA24AA0480023A2
:100540004FF47A7101F074FA002383F31188009B51
:1005500013B19D4B009A1A609C4A009C1378032BA0
:100560001EBF00231370984A4FF0000A18BF536053
:10057000D3465646D146012000F08EFB24B1924B63
:100580001B68002B00F01182002000F06DFA039030
:10059000039B002BF2DB012000F06CFB039B213B53
:1005A000162BE8D801A252F823F000BF0906000874
:1005B00031060008C5060008770500087705000821
:1005C000770500084F0700081F09000839080008D0
:1005D0009B080008C3080008E90800087705000820
:1005E000FB080008770500086D090008A906000847
:1005F00077050008B109000815060008A9060008DB
:10060000770500089B0800080220FFF7C3FE0028BA
:1006100040F0F581009B0221BAF1000F08BF1C4693
:1006200005A841F21233ADF8143000F03BFAA2E70E
:100630004FF47A7000F018FA071EEBDB0220FFF788
:10064000A9FE0028E6D0013F052F00F2DA81DFE89D
:1006500007F0030A0D10133605230593042105A89E
:1006600000F020FA17E054480421F9E75848042123
:10067000F6E758480421F3E74FF01C08404600F025
:100680003DFA08F104080590042105A800F00AFAD3
:10069000B8F12C0FF2D1012000FA07F747EA0B0B53
:1006A0005FFA8BFB4FF0000900F08EFB26B10BF0D8
:1006B0000B030B2B08BF0024FFF774FE5BE74648D3
:1006C0000421CDE7002EA5D00BF00B030B2BA1D1FD
:1006D0000220FFF75FFE074600289BD0012000F0B4
:1006E0000BFA0220FFF7A6FE00265FFA86F84046C6
:1006F00000F012FA044690B10021404600F01CFAC6
:1007000001360028F1D1BA46044641F21213022103
:1007100005A8ADF814303E4600F0C4F92BE70120DF
:10072000FFF788FE2546244B9B68AB4207D9284635
:1007300000F0E4F9013040F067810435F3E7234B22
:1007400000251D70204BBA465D603E46ACE7002E8A
:100750003FF460AF0BF00B030B2B7FF45BAF022079
:10076000FFF768FE322000F07FF9B0F10008FFF6D5
:1007700051AF18F003077FF44DAF0F4A926808EBB2
:10078000050393423FF646AFB8F5807F3FF742AF8F
:10079000124B0193B84523DD4FF47A7000F064F9F1
:1007A0000390039A002AFFF635AF019B039A03F8E2
:1007B000012B0137EDE700BF002200205823002065
:1007C00040220020BD0300085C23002054220020AA
:1007D00004220020082200200C22002058220020A1
:1007E000C820FFF7D7FD074600283FF413AF1F2DA1
:1007F00011D8C5F1200242450AAB25F0030028BFFD
:10080000424683490192184400F06CFA019A8048EC
:10081000FF2100F08DFA4FEAA8037D490193C8F348
:100820008702284600F08CFA064600283FF46DAF98
:10083000019B05EB830537E70220FFF7ABFD00289E
:100840003FF4E8AE00F0A4F900283FF4E3AE00273F
:10085000B846704B9B68BB4218D91F2F11D80A9B12
:1008600001330ED027F0030312AA134453F8203C9F
:1008700005934046042205A900F01CFB043780467E
:10088000E7E7384600F03AF90590F2E7CDF8148032
:10089000042105A800F006F906E70023642104A856
:1008A000049300F0F5F800287FF4B4AE0220FFF7BF
:1008B00071FD00283FF4AEAE049800F051F90590A8
:1008C000E6E70023642104A8049300F0E1F800287F
:1008D0007FF4A0AE0220FFF75DFD00283FF49AAE42
:1008E000049800F04DF9EAE70220FFF753FD0028D5
:1008F0003FF490AE00F05CF9E1E70220FFF74AFD1B
:1009000000283FF487AE05A9142000F057F9042110
:100910000746049004A800F0C5F83946B9E732202C
:1009200000F0A2F8071EFFF675AEBB077FF472AEAB
:10093000384A926807EB090393423FF66BAE0220F8
:10094000FFF728FD00283FF465AE27F003074F446A
:10095000B9453FF4A9AE484600F0D0F8042105900F
:1009600005A800F09FF809F10409F1E74FF47A7047
:10097000FFF710FD00283FF44DAE00F009F9002804
:1009800044D00A9B01330BD008220AA9002000F0B2
:10099000D7F900283AD02022FF210AA800F0C8F990
:1009A000FFF700FD1C4800F0FFFF13B0BDE8F08F1B
:1009B000002E3FF42FAE0BF00B030B2B7FF42AAE6F
:1009C0000023642105A8059300F062F8074600287B
:1009D0007FF420AE0220FFF7DDFC804600283FF4C4
:1009E00019AEFFF7DFFC41F2883000F0DDFF05981B
:1009F00000F01CFA464600F0E7F93C46BBE5064627
:100A000052E64FF0000905E6BA467EE637467CE638
:100A10005822002000220020A086010070B50F4B54
:100A20001B780133DBB2012B0C4611D80C4D296821
:100A30004FF47A730E6AA2FB03320146224628461F
:100A4000B047844204D1074B00221A70012070BDC8
:100A50004FF4FA7000F0A8FF0020F8E71022002001
:100A6000502500209023002007B5002302460121D5
:100A70000DF107008DF80730FFF7D0FF20B19DF88A
:100A8000070003B05DF804FB4FF0FF30F9E700000A
:100A90000A4608B50421FFF7C1FF80F00100C0B28B
:100AA000404208BD30B4054C2368DD69044B0A465A
:100AB000AC460146204630BC604700BF50250020B0
:100AC000A086010070B501F01DFA094E094D308075
:100AD000002428683388834208D901F00DFA2B6876
:100AE00004440133B4F5803F2B60F2D370BD00BFE6
:100AF000922300206423002001F0C6BA00F10060B8
:100B000000F580300068704700F10060920000F549
:100B1000803001F045BA0000054B1A68054B1B8870
:100B20009B1A834202D9104401F0E6B900207047B5
:100B3000642300209223002038B5084D044629B1D3
:100B400028682044BDE8384001F0F6B92868204400
:100B500001F0DAF90028F3D038BD00BF642300208B
:100B600010F003030AD1B0F5047F05D200F1005064
:100B7000A0F51040D0F80038184670470023FBE776
:100B800000F10050A0F51040D0F8100A70470000A6
:100B9000064991F8243033B10023086A81F82430E3
:100BA0000822FFF7B1BF0120704700BF6823002073
:100BB000014B1868704700BF002004E070B52A4B55
:100BC0001B68C3F30B0204461B0C62B140F21340D6
:100BD000824230D040F2194082422ED040F2214071
:100BE00082422CD10322214D0C2000FB0252556879
:100BF00042F20102934224D0B3F5805F23D041F248
:100C00000102934221D041F2030293421FD041F2EC
:100C10000702934214BF3F233123013C0C44013DA2
:100C20000A46A24215D215F9016F501C9EB100F878
:100C3000016C0246F5E70122D5E70222D3E70C4D0D
:100C4000D6E73323E9E74123E7E75A23E5E75923CA
:100C5000E3E7104605E02C258442157001D9901C6D
:100C60005370401A70BD00BF002004E0B834000883
:100C70008C340008022804D1054B4FF000729A61B1
:100C800070470128FCD1034B4FF08042F7E700BFCB
:100C90000004024000000240022804D1054B4FF43A
:100CA00000729A6170470128FCD1034B4FF48042D7
:100CB000F7E700BF0004024000000240022805D10F
:100CC000064A536983F40073536170470128FCD1CD
:100CD000034A536983F48043F6E700BF00040240EF
:100CE0000000024010B50023934203D0CC5CC454F2
:100CF0000133F9E710BD000010B5013810F9013FCC
:100D00003BB191F900409C4203D11AB10131013A43
:100D1000F4E71AB191F90020981A10BD1046FCE7CB
:100D200003460246D01A12F9011B0029FAD1704776
:100D300002440346934202D003F8011BFAE77047CE
:100D40002DE9F8431F4D144695F8242007468846A0
:100D500052BBDFF870909CB395F824302BB9202259
:100D6000FF2148462F62FFF7E3FF95F82400C0F10A
:100D70000802A24228BF2246D6B24146920005EBA5
:100D80008000FFF7AFFF95F82430A41B1E44F6B295
:100D9000082E17449044E4B285F82460DBD1FFF7B5
:100DA000F7FE0028D7D108E02B6A03EB82038342C9
:100DB000CFD0FFF7EDFE0028CBD10020BDE8F883AF
:100DC0000120FBE768230020024B1A78024B1A70BF
:100DD000704700BF902300201022002010B50F4C58
:100DE0000F4800F0F7F821460D4800F01FF924687D
:100DF0000C48626DD2F8043843F00203C2F804389C
:100E000000F0D2FD0849204600F016FA626DD2F8D3
:100E1000043823F00203C2F8043810BDAC350008D2
:100E20005025002040420F00B435000870470000F4
:100E300000B59BB0EFF3098168226846FFF752FFC7
:100E4000EFF30583044B9A6BDA6A9A6A9A6A9A6A94
:100E50009A6A9A6A9B6AFEE700ED00E000B59BB0D3
:100E6000EFF3098168226846FFF73CFFEFF3058343
:100E7000044B9A6B9A6A9A6A9A6A9A6A9A6A9B6A05
:100E8000FEE700BF00ED00E000B59BB0EFF3098185
:100E900068226846FFF726FFEFF30583034B5A6B82
:100EA0009A6A9A6A9A6A9A6A9B6AFEE700ED00E07B
:100EB000FEE7000030B5094D0A4491420DD011F80B
:100EC000013B5840082340F30004013B2C4013F041
:100ED000FF0384EA5000F6D1EFE730BD2083B8ED80
:100EE000026843681143016003B11847704700006E
:100EF00013B5446BD4F894341A681178042915D1C9
:100F0000217C022912D11979128901238B401342C5
:100F10000CD101A904F14C0001F03AFFD4F894443B
:100F2000019B21790246206800F0CEF902B010BD85
:100F3000143001F0BDBE00004FF0FF33143001F05B
:100F4000B7BE00004C3001F08FBF00004FF0FF3300
:100F50004C3001F089BF0000143001F08BBE00005E
:100F60004FF0FF31143001F085BE00004C3001F02D
:100F70005BBF00004FF0FF324C3001F055BF000066
:100F80000020704710B5D0F894341A6811780429FD
:100F9000044617D1017C022914D1597952890123C1
:100FA0008B4013420ED1143001F01EFE024648B1B0
:100FB000D4F894444FF4807361792068BDE8104000
:100FC00000F070B910BD0000406BFFF7DBBF000000
:100FD000704700007FB5124B036000234360C0E9F7
:100FE0000233012502260F4B05740446029001933B
:100FF00000F18402294600964FF48073143001F00A
:10100000CFFD094B0294CDE9006304F523724FF440
:101010008073294604F14C0001F096FE04B070BDC7
:10102000E8340008C90F0008F10E00080B68202200
:1010300082F311880A7903EB820290614A790932BE
:1010400043F822008A7912B103EB820398610223EC
:101050000374C0F89414002383F3118870470000D0
:1010600038B5037F044613B190F85430ABB9201D56
:1010700001250221FFF734FF04F1140025776FF0FA
:10108000010100F0B9FC84F8545004F14C006FF0F9
:101090000101BDE8384000F0AFBC38BD10B50121FA
:1010A00004460430FFF71CFF0023237784F85430F4
:1010B00010BD000038B504460025143001F088FD4D
:1010C00004F14C00257701F057FE201D84F85450A0
:1010D0000121FFF705FF2046BDE83840FFF752BF6A
:1010E00090F8443003F06003202B07D190F845209E
:1010F000212A4FF0000303D81F2A06D8002070478A
:10110000222AFBD1C0E90E3303E0034A826307229F
:10111000C2630364012070471122002037B5D0F864
:1011200094341A681178042904461AD1017C0229E2
:1011300017D11979128901238B40134211D100F183
:101140004C05284601F0D8FE58B101A9284601F007
:101150001FFED4F89444019B21790246206800F0D8
:10116000B3F803B030BD0000F0B500EB810385B0EB
:101170009E6904460D46FEB1202383F3118804EBDB
:101180008507301D0821FFF7ABFEFB685B691B6814
:1011900006F14C001BB1019001F008FE019803A973
:1011A00001F0F6FD024648B1039B2946204600F0B7
:1011B0008BF8002383F3118805B0F0BDFB685A69F2
:1011C0001268002AF5D01B8A013B1340F1D104F1CB
:1011D0004402EAE7093138B550F82140DCB1202358
:1011E00083F31188D4F894241368527903EB8203B3
:1011F000DB689B695D6845B104216018FFF770FEEC
:10120000294604F1140001F0F9FC2046FFF7BAFE6C
:10121000002383F3118838BD7047000001F0A6B8A1
:10122000012303700023C0E90133C36183620362B9
:10123000C36243620363704738B50446202383F3D7
:1012400011880025C0E90355C0E90555416001F04A
:101250009DF80223237085F3118838BD70B500EB2B
:10126000810305465069DA600E46144618B1102213
:101270000021FFF75DFDA06918B110220021FFF7E2
:1012800057FD31462846BDE8704001F049B90000DD
:10129000826802F0011282600022C0E904228261A9
:1012A00001F0CAB9F0B400EB81044789E468012574
:1012B000A4698D403D43458123600023A2606360A3
:1012C000F0BC01F0E5B90000F0B400EB810407893F
:1012D000E468012564698D403D4305812360002356
:1012E000A2606360F0BC01F05FBA000070B5022339
:1012F000002504460370C0E90255C0E90455C564E1
:10130000856180F8345001F0A7F863681B6823B149
:1013100029462046BDE87040184770BD037880F824
:1013200050300523037043681B6810B504460BB1A9
:10133000042198470023A36010BD000090F85020BE
:10134000436802701B680BB1052118477047000005
:1013500070B590F83430044613B1002380F834306F
:1013600004F14402204601F089F963689B68B3B92F
:1013700094F8443013F0600535D00021204601F088
:10138000DBFB0021204601F0CDFB63681B6813B135
:10139000062120469847062384F8343070BD204645
:1013A00098470028E4D0B4F84A30E26B9A4288BFEC
:1013B000E36394F94430E56B002B4FF0200380F297
:1013C0000381002D00F0F280092284F8342083F399
:1013D00011880021D4E90E232046FFF775FF002372
:1013E00083F31188DAE794F8452003F07F0343EA9A
:1013F000022340F20232934200F0C58021D8B3F5B7
:10140000807F48D00DD8012B3FD0022B00F0938075
:10141000002BB2D104F14C02A2630222E2632364E6
:10142000C1E7B3F5817F00F09B80B3F5407FA4D185
:1014300094F84630012BA0D1B4F84C3043F00203AD
:1014400032E0B3F5006F4DD017D8B3F5A06F31D0AF
:10145000A3F5C063012B90D8636894F846205E68BA
:1014600094F84710B4F848302046B047002884D09C
:101470004368A3630368E3631AE0B3F5106F36D0E3
:1014800040F6024293427FF478AF5C4BA3630223A1
:10149000E3630023C3E794F84630012B7FF46DAF7C
:1014A000B4F84C3023F00203C4E90E55A4F84C30D4
:1014B000256478E7B4F84430B3F5A06F0ED194F802
:1014C000463084F84E30204601F01EF863681B68F1
:1014D00013B1012120469847032323700023C4E958
:1014E0000E339CE704F14F03A3630123C3E7237882
:1014F000042B10D1202383F311882046FFF7C8FE68
:1015000085F311880321636884F84F5021701B68AC
:101510000BB12046984794F84630002BDED084F873
:101520004F300423237063681B68002BD6D0022140
:1015300020469847D2E794F848301D0603F00F0183
:1015400020460AD501F08CF8012804D002287FF447
:1015500014AF2B4B9AE72B4B98E701F073F8F3E7A6
:1015600094F84630002B7FF408AF94F8483013F01D
:101570000F01B3D01A06204602D501F0F1FAADE70B
:1015800001F0E4FAAAE794F84630002B7FF4F5AEB8
:1015900094F8483013F00F01A0D01B06204602D566
:1015A00001F0CAFA9AE701F0BDFA97E7142284F82D
:1015B000342083F311882B462A4629462046FFF71C
:1015C00071FE85F31188E9E65DB1152284F83420B7
:1015D00083F311880021D4E90E232046FFF762FE31
:1015E000FDE60B2284F8342083F311882B462A462B
:1015F00029462046FFF768FEE3E700BF18350008DC
:10160000103500081435000838B590F83430044619
:10161000002B3ED0063BDAB20F2A34D80F2B32D83B
:10162000DFE803F0373131082232313131313131E5
:1016300031313737C56BB0F84A309D4214D2C36898
:101640001B8AB5FBF3F203FB12556DB9202383F31C
:1016500011882B462A462946FFF736FE85F3118866
:101660000A2384F834300EE0142384F83430202325
:1016700083F3118800231A4619462046FFF712FE0D
:10168000002383F3118838BD036C03B1984700230E
:10169000E7E70021204601F04FFA0021204601F043
:1016A00041FA63681B6813B1062120469847062358
:1016B000D7E7000010B590F83430142B044629D039
:1016C00017D8062B05D001D81BB110BD093B022B42
:1016D000FBD80021204601F02FFA0021204601F01E
:1016E00021FA63681B6813B1062120469847062338
:1016F00019E0152BE9D10B2380F83430202383F334
:10170000118800231A461946FFF7DEFD002383F3F4
:101710001188DAE7C3689B695B68002BD5D1036C3D
:1017200003B19847002384F83430CEE7024B0022FF
:10173000C3E900339A6070479423002000230374A8
:101740008268054B1B6899689142FBD25A68036016
:1017500042601060586070479423002008B5202331
:1017600083F31188037C032B05D0042B0DD02BB9F8
:1017700083F3118808BD436900221A604FF0FF33DC
:101780004361FFF7DBFF0023F2E7D0E9003213608B
:101790005A60F3E7002303748268054B1B6899685D
:1017A0009142FBD85A6803604260106058607047ED
:1017B00094230020054B19690874186802681A60A0
:1017C0005360186101230374FEF7A0BD9423002029
:1017D00030B54B1C0B4D87B0044610D02B690A4A1C
:1017E00001A800F025F92046FFF7E4FF049B13B1A0
:1017F00001A800F059F92B69586907B030BDFFF70F
:10180000D9FFF8E7942300205D17000838B50C4D88
:1018100041612B6981689A689142044603D8BDE80A
:101820003840FFF78BBF1846FFF7B4FF01232C6148
:10183000014623742046BDE83840FEF767BD00BF6F
:1018400094230020044B1A681B6990689B68984297
:1018500094BF0020012070479423002010B5084C4D
:10186000236820691A6822605460012223611A7477
:10187000FFF790FF01462069BDE81040FEF746BD26
:101880009423002008B5FFF7DDFF18B1BDE808403C
:10189000FFF7E4BF08BD0000FFF7E0BFFEE7000070
:1018A00010B50C4CFFF742FF00F0B4F80A49802253
:1018B000204600F03BF8012344F8180C037400F0B4
:1018C0006FFC002383F3118862B60448BDE8104022
:1018D00000F04CB8BC2300201C3500082C35000853
:1018E00000F01CB9EFF3118020B9EFF3058320223B
:1018F00082F311887047000010B530B9EFF305840A
:10190000C4F3080414B180F3118810BDFFF7BAFFC7
:1019100084F31188F9E70000034A516853685B1AA1
:101920009842FBD8704700BF001000E0826002229E
:10193000028270478368A3F17C0243F80C2C026991
:1019400043F83C2C426943F8382C074A43F81C2CD6
:10195000C26843F8102C022203F8082C002203F876
:10196000072CA3F1180070472503000810B52023A9
:1019700083F31188FFF7DEFF00210446FFF746FFDF
:10198000002383F31188204610BD0000024B1B6921
:1019900058610F20FFF70EBF94230020202383F30C
:1019A0001188FFF7F3BF000008B50146202383F339
:1019B00011880820FFF70CFF002383F3118808BD6E
:1019C00049B1064B42681B6918605A601360436056
:1019D0000420FFF7FDBE4FF0FF3070479423002036
:1019E0000368984206D01A68026050605961184630
:1019F000FFF7A4BE7047000038B504460D462068C6
:101A0000844200D138BD036823605C604561FFF704
:101A100095FEF4E7054B03F11402C3E905224FF0EC
:101A2000FF310022C3E90712704700BF9423002052
:101A300070B51C4EC0E9032305460C4601F08EFA32
:101A4000334653F8142F9A420DD13062C5E9012470
:101A50002A600A2C2CBF00190A30C6E90555BDE8DA
:101A6000704001F069BA316A431AE31838BF1C4666
:101A70009368A34202D9081901F06CFA73699A6855
:101A800094420CD85A68AC602B606A6015609A6802
:101A90005D60121B9A604FF0FF33F36170BD1B68ED
:101AA000A41AECE79423002038B51B4C63699842D4
:101AB0000DD0D0E9003213605A6000228168C26004
:101AC0009A680A449A604FF0FF33E36138BD2246BA
:101AD000036842F8143F002193425A60C16003D169
:101AE000BDE8384001F030BA9A688168256A0A4436
:101AF0009A6001F033FA63699A68411B8A42E5D91A
:101B0000AB181D1A092D206A98BF01F10A02BDE821
:101B10003840104401F01EBA942300202DE9F04112
:101B2000184C002704F11406656901F017FA236ABE
:101B3000AA68C11A8A4215D813442362D5E9003233
:101B400013605A606369D5F80C80EF60B34201D12D
:101B500001F0FAF987F311882869C047202383F33D
:101B60001188E1E76169B14209D013441B1ABDE84D
:101B7000F0410A2B2CBFC0180A3001F0EBB9BDE8C8
:101B8000F08100BF9423002000207047FEE7000092
:101B9000704700004FF0FF307047000002290CD062
:101BA000032904D00129074818BF00207047032AE1
:101BB00005D8054800EBC200704704487047002074
:101BC000704700BF1036000820220020C4350008EE
:101BD00070B59AB00546084601A9144600F0C2F84F
:101BE00001A8FFF79DF8431C5B00C5E90034002203
:101BF000237003236370C6B201AB02341046D1B226
:101C00008E4204F1020401D81AB070BD13F8011B12
:101C100004F8021C04F8010C0132F0E708B5202397
:101C200083F311880348FFF779FA002383F31188BF
:101C300008BD00BF5025002090F8443003F01F027B
:101C4000012A07D190F845200B2A03D10023C0E9CF
:101C50000E3315E003F06003202B08D1B0F84830B4
:101C60002BB990F84520212A03D81F2A04D8FFF762
:101C700037BA222AEBD0FAE7034A82630722C2630B
:101C800003640120704700BF1822002007B5052912
:101C900017D8DFE801F0191603191920202383F360
:101CA0001188104A01900121FFF7D8FA01980E4AD5
:101CB0000221FFF7D3FA0D48FFF7FCF9002383F365
:101CC000118803B05DF804FB202383F311880748D3
:101CD000FFF7C6F9F2E7202383F311880348FFF7E3
:101CE000DDF9EBE764350008883500085025002051
:101CF00038B50C4D0C4C0D492A4604F10800FFF78D
:101D000067FF05F1CA0204F110000949FFF760FFFF
:101D100005F5CA7204F118000649BDE83840FFF71E
:101D200057BF00BF182A0020202200204435000899
:101D30004E3500085935000870B5044608460D4672
:101D4000FEF7EEFFC6B22046013403780BB9184601
:101D500070BD32462946FEF7CFFF0028F3D101209F
:101D6000F6E700002DE9F04705460C46FEF7D8FFE0
:101D70002A49C6B22846FFF7DFFF08B10936F6B296
:101D800027492846FFF7D8FF08B11036F6B2632E70
:101D90000BD8DFF88880DFF88890224FDFF890A01A
:101DA0002E7846B92670BDE8F08729462046BDE862
:101DB000F04701F063BB252E2CD10722414628466F
:101DC000FEF79AFF60B9184B224603F1100153F851
:101DD000040B42F8040B8B42F9D107351034DFE7CE
:101DE000082249462846FEF787FF98B90F4BA21CE8
:101DF000197809090232C95D02F8041C13F8011BA5
:101E000001F00F015345C95D02F8031CF0D11834ED
:101E10000835C5E704F8016B0135C1E73036000825
:101E2000593500084936000838360008107AFF1F77
:101E30001C7AFF1FBFF34F8F024AD368DB03FCD429
:101E4000704700BF003C024008B5094B1B7873B9CE
:101E5000FFF7F0FF074B1A69002ABFBF064A5A6016
:101E600002F188325A601A6822F480621A6008BD52
:101E7000762C0020003C02402301674508B50B4B3F
:101E80001B7893B9FFF7D6FF094B1A6942F000425D
:101E90001A611A6842F480521A601A6822F4805259
:101EA0001A601A6842F480621A6008BD762C00201D
:101EB000003C02400B28F0B516D80C4C0C49237896
:101EC0007BB90C4D0E460C234FF0006255F8047B95
:101ED00046F8042B013B13F0FF033A44F6D10123EB
:101EE000237051F82000F0BD0020FCE7A82C002052
:101EF000782C00205C360008014B53F82000704716
:101F00005C3600080C2070470B2810B5044601D938
:101F1000002010BDFFF7CEFF064B53F824301844C5
:101F2000C21A0BB90120F4E712680132F0D1043B68
:101F3000F6E700BF5C3600080B2838B5044628D801
:101F4000FFF7D0FCFFF776FFFFF77EFF124AF3237F
:101F5000D360E300DBB243F4007343F00203136188
:101F6000136943F48033136105462046FFF762FF8F
:101F7000FFF7A0FF094B53F8241000F0E9F82846BA
:101F8000FFF77CFFFFF7B8FC2046BDE83840FFF7BD
:101F9000BBBF002038BD00BF003C02405C360008DB
:101FA00012F001032DE9F04105460E4614464BD1CF
:101FB0008218B2F1016F61D8314B1B6813F0010335
:101FC0005CD0304FFFF78EFCFFF73EFFF323FB6042
:101FD000FFF730FF314640F20128032C18D824F0D7
:101FE0000104284E0C446D1A40F20118A1423369D5
:101FF00005EB01072AD123F001033361FFF73EFF10
:10200000FFF77AFC0120BDE8F081043C0435E4E7E9
:10201000AB07E4D13B6923F440733B613B6943EA7E
:1020200008033B6151F8046B2E60BFF34F8FFFF73D
:1020300001FF2B689E42E8D03B6923F001033B611E
:10204000FFF71CFFFFF758FC0020DCE723F4407388
:102050003361336943EA080333610B883B80BFF384
:102060004F8FFFF7E7FE3F8831F8023BBFB2BB421C
:10207000BCD0336923F001033361E1E71846C2E7BE
:1020800000380240003C0240084908B50B7828B1EE
:102090001BB9FFF7D9FE01230B7008BD002BFCD044
:1020A000BDE808400870FFF7E9BE00BF762C0020AD
:1020B00010B50244064BD2B2904200D110BD441C70
:1020C00000B253F8200041F8040BE0B2F4E700BF7F
:1020D000502800400F4B30B51C6F240407D41C6FF0
:1020E00044F400741C671C6F44F400441C670A4CE1
:1020F000236843F4807323600244084BD2B29042B9
:1021000000D130BD441C00B251F8045B43F82050AC
:10211000E0B2F4E700380240007000405028004070
:1021200007B5012201A90020FFF7C2FF019803B003
:102130005DF804FB13B50446FFF7F2FFA04205D09B
:10214000012201A900200194FFF7C4FF02B010BDD5
:1021500070470000034B1A681AB9034AD2F8742872
:102160001A607047AC2C00200030024008B5FFF721
:10217000F1FF024B1868C0F3407008BDAC2C002082
:10218000EFF3098305494A6B22F001024A63683381
:1021900083F30988002383F31188704700EF00E080
:1021A000202080F3118862B60C4B0D4AD96821F4C7
:1021B000E0610904090C0A43DA60D3F8FC200949FC
:1021C00042F08072C3F8FC200A6842F001020A6003
:1021D0001022DA7783F82200704700BF00ED00E09C
:1021E0000003FA05001000E010B5202383F31188E6
:1021F0000E4B5B6813F4006314D0F1EE103AEFF36A
:102200000984683C4FF08073E361094BDB6B236604
:1022100084F30988FFF716FB10B1064BA36110BDCC
:10222000054BFBE783F31188F9E700BF00ED00E001
:1022300000EF00E0370300083A0300087047000091
:10224000FEE700000A4B0B480B4A90420BD30B4BA6
:10225000DA1C121AC11E22F003028B4238BF002280
:102260000021FEF765BD53F8041B40F8041BECE7A2
:10227000F8370008A82D0020A82D0020A82D002048
:102280007047000070B5D0E915439E6800224FF0FA
:10229000FF3504EB42135101D3F800090028BEBFFB
:1022A000D3F8000940F08040C3F80009D3F8000BD0
:1022B0000028BEBFD3F8000B40F08040C3F8000BED
:1022C000013263189642C3F80859C3F8085BE0D29C
:1022D0004FF00113C4F81C3870BD00001D4B03EB18
:1022E00080022DE9F043D2F80CC05D6DDCF81420BB
:1022F000461CD2F800E005EB063605EB40185168A5
:1023000071450AD3D5F83438012202FA00F023EAE5
:102310000000C5F83408BDE8F083BCF81040AEEB0F
:102320000103A34228BF2346D8F81849A4B2B3EB4F
:10233000840FF0D89468A4F1040959F8047F376039
:10234000A4EB09071F44042FF7D81C440B449460E6
:102350005360D4E7B02C0020890141F020010161D5
:1023600003699B06FCD41220FFF7D6BA10B5054CC2
:102370002046FEF755FF4FF0A0436365024BA3656F
:1023800010BD00BFB02C0020B036000870B5037837
:10239000012B054650D12A4B446D98421BD1294B45
:1023A0005A6B42F080025A635A6D42F080025A65BD
:1023B0005A6D5A6942F080025A615A6922F08002CD
:1023C0005A610E2143205B6900F0D4FB1E4BE36091
:1023D0001E4BC4F800380023C4F8003EC02323601D
:1023E0006E6D4FF40413A3633369002BFCDA0123F1
:1023F00033610C20FFF790FA3369DB07FCD412201D
:10240000FFF78AFA3369002BFCDA0026A66028461B
:10241000FFF738FF6B68C4F81068DB68C4F814680D
:10242000C4F81C684BB90A4BA3614FF0FF336361DA
:10243000A36843F00103A36070BD064BF4E700BF3F
:10244000B02C00200038024040140040030020025D
:10245000003C30C0083C30C0F8B5446D0546002152
:102460002046FFF779FFA96D00234FF001128F6816
:10247000C4F834384FF00066C4F81C284FF0FF3021
:1024800004EB431201339F42C2F80069C2F8006BAB
:10249000C2F80809C2F8080BF2D20B686A6DEB6546
:1024A000636210231361166916F01006FBD1122027
:1024B000FFF732FAD4F8003823F4FE63C4F800388A
:1024C000A36943F4402343F01003A3610923C4F834
:1024D0001038C4F814380A4BEB604FF0C043C4F80E
:1024E000103B084BC4F8003BC4F81069C4F800392D
:1024F000EB6D03F1100243F48013EA65A362F8BDAB
:102500008C36000840800010426D90F84E10D2F8D2
:10251000003823F4FE6343EA0113C2F80038704721
:102520002DE9F84300EB8103456DDA68166806F083
:102530000306731E022B05EB41130C4680460FFA6F
:1025400081F94FEA41104FF00001C3F8101B4FF022
:10255000010104F1100398BFB60401FA03F3916975
:102560008EBF334E06F1805606F5004600293AD05C
:10257000578A04F15801490137436F50D5F81C18A8
:102580000B43C5F81C382B180021C3F810195369E8
:102590000127611EA7409BB3138A928B9B08012AD7
:1025A00088BF5343D8F85C20981842EA034301F1EE
:1025B000400205EB8202C8F85C00214653602846C1
:1025C000FFF7CAFE08EB8900C3681B8A43EA8453FD
:1025D000483464011E432E51D5F81C381F43C5F8FA
:1025E0001C78BDE8F88305EB4917D7F8001B21F4E8
:1025F0000041C7F8001BD5F81C1821EA0303C0E707
:1026000004F13F0305EB83030A4A5A60284621463A
:10261000FFF7A2FE05EB4910D0F8003923F4004380
:10262000C0F80039D5F81C3823EA0707D7E700BF00
:102630000080001000040002826D1268C265FFF77E
:1026400021BE00005831436D49015B5813F400402E
:1026500004D013F4001F0CBF0220012070470000BB
:102660004831436D49015B5813F4004004D013F422
:10267000001F0CBF022001207047000000EB810109
:10268000CB68196A0B6813604B6853607047000091
:1026900000EB810330B5DD68AA691368D36019B90E
:1026A000402B84BF402313606B8A1468426D1C4426
:1026B000013CB4FBF3F46343033323F0030302EB65
:1026C000411043EAC44343F0C043C0F8103B2B68B9
:1026D00003F00303012B09B20ED1D2F8083802EB44
:1026E000411013F4807FD0F8003B14BF43F08053B7
:1026F00043F00053C0F8003B02EB4112D2F8003B1C
:1027000043F00443C2F8003B30BD00002DE9F04126
:10271000244D6E6D06EB40130446D3F8087BC3F8D6
:10272000087B38070AD5D6F81438190706D505EB03
:1027300084032146DB6828465B689847FA071FD563
:10274000D6F81438DB071BD505EB8403D968CCB960
:102750008B69488A5A68B2FBF0F600FB16228AB9E8
:102760001868DA6890420DD2121AC3E900242023B7
:1027700083F311880B482146FFF78AFF84F3118801
:10278000BDE8F081012303FA04F26B8923EA020316
:102790006B81CB68002BF3D021460248BDE8F041A5
:1027A000184700BFB02C002000EB810370B5DD6836
:1027B000436D6C692668E6604A0156BB1A444FF4C3
:1027C0000020C2F810092A6802F00302012A0AB2A6
:1027D0000ED1D3F8080803EB421410F4807FD4F82C
:1027E000000914BF40F0805040F00050C4F80009C8
:1027F00003EB4212D2F8000940F00440C2F800098D
:10280000D3F83408012202FA01F10143C3F8341865
:1028100070BD19B9402E84BF4020206020682E8AE8
:102820008419013CB4FBF6F440EAC44040F0005087
:102830001A44C6E7F8B504461E48456D05EB441337
:10284000D3F80869C3F80869F10717D5D5F8103827
:10285000DA0713D500EB8403D9684B691F68DA687F
:10286000974218D2D21B00271A605F60202383F39F
:1028700011882146FFF798FF87F31188330617D593
:10288000D5F834280123A340134211D02046BDE8D7
:10289000F840FFF723BD012303FA04F2038923EA7A
:1028A000020303818B68002BE8D021469847E5E7B7
:1028B000F8BD00BFB02C00202DE9F74F984C666D95
:1028C0007569B3691D4015F48058756107D02046BD
:1028D000FEF70CFD03B0BDE8F04FFFF785BC002DFF
:1028E00012DAD6F8003E8E489F071EBFD6F8003E8B
:1028F00023F00303C6F8003ED6F8043823F00103A2
:10290000C6F80438FEF71AFD280505D58448FFF7F8
:10291000B9FC8348FEF702FDA9040CD5D6F80838A7
:1029200013F0060FF36823F470530CBF43F41053F5
:1029300043F4A053F3602A0704D56368DB680BB146
:1029400077489847EB0274D4AF0227D5D4F8549057
:10295000DFF8CCB100274FF0010A09EB4712D2F89B
:10296000003B03F44023B3F5802F11D1D2F8003B94
:10297000002B0DDA62890AFA07F322EA0303638166
:1029800004EB8703DB68DB6813B139465846984788
:10299000A36D01379B68FFB29F42DED9E80617D5C9
:1029A000676D3A6AC2F30A1002F00F0302F4F012E4
:1029B000B2F5802F00F08880B2F5402F08D104EBEB
:1029C00083030022DB681B6A07F5805790426DD1B4
:1029D0002903D6F8184813D5E20302D50020FFF7E3
:1029E00095FEA30302D50120FFF790FE670302D5F1
:1029F0000220FFF78BFE260302D50320FFF786FE99
:102A00006D037FF567AFE00702D50020FFF712FFE7
:102A1000A10702D50120FFF70DFF620702D50220B2
:102A2000FFF708FF23077FF555AF0320FFF702FFED
:102A300050E7636DDFF8E8B0019300274FF0010A1B
:102A4000A36D9B685FFA87F999453FF67DAF019BBF
:102A500003EB4913D3F8002902F44022B2F5802F8A
:102A600022D1D3F80029002A1EDAD3F8002942F037
:102A70009042C3F80029D3F80029002AFBDB606DDF
:102A80004946FFF769FC22890AFA09F322EA03039F
:102A9000238104EB8903DB689B6813B149465846E0
:102AA00098474846FFF71AFC0137C9E7910708BF66
:102AB000D7F80080072A98BF03F8018B02F10102C2
:102AC00098BF4FEA182881E7023304EB830207F529
:102AD00080575268D2F818C0DCF80820DCE9001CE6
:102AE000A1EB0C0C002188420AD104EB830463683B
:102AF0009B699A6802449A605A6802445A6067E780
:102B000011F0030F08BFD7F800808C4588BF02F88A
:102B1000018B01F1010188BF4FEA1828E3E700BFEC
:102B2000B02C0020436D03EB4111D1F8003B43F47E
:102B30000013C1F8003B7047436D03EB4111D1F81E
:102B4000003943F40013C1F800397047436D03EBBB
:102B50004111D1F8003B23F40013C1F8003B70474A
:102B6000436D03EB4111D1F8003923F40013C1F890
:102B70000039704700F1604303F561430901C9B2B0
:102B800083F80013012200F01F039A4043099B00C1
:102B900003F1604303F56143C3F880211A60704775
:102BA00030B5039C0172043304FB0325C0E90653CE
:102BB000049B03630021059BC160C0E90000C0E9DC
:102BC0000422C0E90842C0E90A11436330BD000095
:102BD000416A0022C0E90411C0E90A22C2606FF014
:102BE0000101FEF709BF0000D0E90432934201D190
:102BF000C2680AB9181D7047002070470369196040
:102C0000C2680132C260C26913448269036193429F
:102C100024BF436A03610021FEF7E2BE38B50446D3
:102C20000D46E3683BB16269131D1268A362134449
:102C3000E362002007E0237A33B929462046FEF7F5
:102C4000BFFE0028EDDA38BD6FF00100FBE70000A1
:102C5000C368C269013BC36043691344826943612D
:102C6000934224BF436A436100238362036B03B131
:102C70001847704770B52023044683F31188866A8D
:102C80003EB9FFF7CBFF054618B186F311882846F9
:102C900070BDA36AE26A13F8015BA362934202D398
:102CA0002046FFF7D5FF002383F31188EFE70000EC
:102CB0002DE9F84F04460E46174698464FF0200976
:102CC00089F311880025AA46D4F828B0BBF1000F7B
:102CD00009D141462046FFF7A1FF20B18BF31188AF
:102CE0002846BDE8F88FD4E90A12A7EB050B521A63
:102CF000934528BF9346BBF1400F1BD9334601F1E2
:102D0000400251F8040B43F8040B9142F9D1A36A35
:102D100040334036A3624035D4E90A239A4202D3B5
:102D20002046FFF795FF8AF31188BD42D8D289F378
:102D30001188C9E730465A46FDF7D4FFA36A5B44C1
:102D40005E44A3625D44E7E710B5029C0172043360
:102D500004FB0321C0E906130023C0E90A33039BE7
:102D60000363049BC460C0E90000C0E90422C0E919
:102D70000842436310BD0000026AC260426AC0E9B3
:102D800004220022C0E90A226FF00101FEF734BEDE
:102D9000D0E904239A4201D1C26822B9184650F8FA
:102DA000043B0B607047002070470000C368C26995
:102DB0000133C3604369134482694361934224BF72
:102DC000436A43610021FEF70BBE000038B504469C
:102DD0000D46E3683BB123691A1DA262E269134400
:102DE000E362002007E0237A33B929462046FEF744
:102DF000E7FD0028EDDA38BD6FF00100FBE70000C9
:102E000003691960C268013AC260C26913448269E9
:102E10000361934224BF436A036100238362036B0F
:102E200003B118477047000070B520230D460446D3
:102E3000114683F31188866A2EB9FFF7C7FF10B1D8
:102E400086F3118870BDA36A1D70A36AE26A01331C
:102E50009342A36204D3E16920460439FFF7D0FF0F
:102E6000002080F31188EDE72DE9F84F04460D4668
:102E7000904699464FF0200A8AF311880026B346FF
:102E8000A76A4FB949462046FFF7A0FF20B187F354
:102E900011883046BDE8F88FD4E90A073A1AA8EB42
:102EA0000607974228BF1746402F1BD905F140035C
:102EB00055F8042B40F8042B9D42F9D1A36A403306
:102EC000A3624036D4E90A239A4204D3E16920463A
:102ED0000439FFF795FF8BF311884645D9D28AF361
:102EE0001188CDE729463A46FDF7FCFEA36A3B442C
:102EF0003D44A3623E44E5E7D0E904239A4217D15A
:102F0000C3689BB1836A8BB1043B9B1A0ED01360DC
:102F1000C368013BC360C3691A44836902619A4272
:102F200024BF436A0361002383620123184670476C
:102F30000023FBE700F088B84FF08043002258637D
:102F40001A610222DA6070474FF080430022DA6093
:102F5000704700004FF08043586370474FF0804344
:102F6000586A70474B6843608B688360CB68C36066
:102F70000B6943614B6903628B6943620B680360B1
:102F80007047000008B5264B26481A6940F2FF1129
:102F90000A431A611A6922F4FF7222F001021A61CF
:102FA0001A691A6B0A431A631A6D0A431A651E4A94
:102FB0001B6D1146FFF7D6FF02F11C0100F5806082
:102FC000FFF7D0FF02F1380100F58060FFF7CAFF7C
:102FD00002F1540100F58060FFF7C4FF02F17001B7
:102FE00000F58060FFF7BEFF02F18C0100F5806004
:102FF000FFF7B8FF02F1A80100F58060FFF7B2FF0C
:1030000002F1C40100F58060FFF7ACFF02F1E001BE
:1030100000F58060FFF7A6FFBDE8084000F09AB811
:103020000038024000000240BC36000808B500F03D
:1030300007FAFEF735FCFFF78DF8BDE80840FEF70C
:1030400057BE000070470000104B1A6C42F001029E
:103050001A641A6E42F001021A660D4A1B6E9368DA
:1030600043F0010393604FF0804353229A624FF084
:10307000FF32DA6200229A615A63DA605A600122F2
:103080005A6108211A601C20FFF774BD0038024005
:10309000002004E04FF0804208B51169D3680B406E
:1030A000D9B2C9439B07116107D5202383F3118847
:1030B000FEF716FC002383F3118808BD08B5FFF75F
:1030C000E9FFBDE80840FFF78FB800001F4B1A6901
:1030D0006FEAC2526FEAD2521A611A69C2F3080249
:1030E0001A614FF0FF301A695A69586100215A6914
:1030F00059615A691A6A62F080521A621A6A02F0B9
:1031000080521A621A6A5A6A58625A6A59625A6A2C
:103110001A6C42F080521A641A6E42F080521A669B
:103120001A6E0B4A106840F480701060186F00F43B
:103130004070B0F5007F1EBF4FF4803018671967EC
:10314000536823F40073536000F05AB9003802400A
:1031500000700040334B4FF080521A64324A4FF4F3
:10316000404111601A6842F001021A601A68910722
:10317000FCD59A6822F003029A602A4B9A6812F0F2
:103180000C02FBD1196801F0F90119609A601A6804
:1031900042F480321A601A689203FCD55A6F42F0EA
:1031A00001025A671F4B5A6F9007FCD51F4A5A609D
:1031B0001A6842F080721A601B4A53685904FCD5A1
:1031C000184B1A689201FCD5194A9A60194B1A6873
:1031D000194B9A42194B21D1194A1168194A914247
:1031E0001CD140F205121A60144A136803F00F0351
:1031F000052BFAD10B4B9A6842F002029A609A684A
:1032000002F00C02082AFAD15A6C42F480425A6445
:103210005A6E42F480425A665B6E704740F2057205
:10322000E1E700BF0038024000700040085440074A
:1032300000948838002004E011640020003C024023
:1032400000ED00E041C20F41084A08B5516913681A
:103250000B4003F00103536123B1054A13680BB11E
:1032600050689847BDE80840FEF7BEBF003C0140EB
:10327000282D0020084A08B5516913680B4003F057
:103280000203536123B1054A93680BB1D068984794
:10329000BDE80840FEF7A8BF003C0140282D0020F3
:1032A000084A08B5516913680B4003F004035361E1
:1032B00023B1054A13690BB150699847BDE808402E
:1032C000FEF792BF003C0140282D0020084A08B5B7
:1032D000516913680B4003F00803536123B1054A99
:1032E00093690BB1D0699847BDE80840FEF77CBFF1
:1032F000003C0140282D0020084A08B55169136898
:103300000B4003F01003536123B1054A136A0BB15C
:10331000506A9847BDE80840FEF766BF003C014090
:10332000282D0020174B10B55A691C68144004F46E
:1033300078725A61A30604D5134A936A0BB1D06A16
:103340009847600604D5104A136B0BB1506B984731
:10335000210604D50C4A936B0BB1D06B9847E2055C
:1033600004D5094A136C0BB1506C9847A30504D5DA
:10337000054A936C0BB1D06C9847BDE81040FEF73E
:1033800033BF00BF003C0140282D00201A4B10B570
:103390005A691C68144004F47C425A61620504D5E1
:1033A000164A136D0BB1506D9847230504D5134A87
:1033B000936D0BB1D06D9847E00404D50F4A136E9E
:1033C0000BB1506E9847A10404D50C4A936E0BB113
:1033D000D06E9847620404D5084A136F0BB1506F42
:1033E0009847230404D5054A936F0BB1D06F9847D3
:1033F000BDE81040FEF7F8BE003C0140282D00203B
:10340000062108B50846FFF7B5FB06210720FFF7A0
:10341000B1FB06210820FFF7ADFB06210920FFF7CD
:10342000A9FB06210A20FFF7A5FB06211720FFF7BD
:10343000A1FBBDE8084006212820FFF79BBB000048
:1034400008B5FFF743FE00F00BF8FDF7E7FEFDF7C8
:10345000BFFDFFF7F7FDBDE80840FFF76BBD0000BB
:103460000023054A19460133102BC2E9001102F16D
:103470000802F8D1704700BF282D0020034611F83C
:10348000012B03F8012B002AF9D1704753544D3317
:1034900032463F3F3F00000053544D3332463430F4
:1034A000780053544D3332463432780053544D3300
:1034B0003246343436585800000000008C3400087E
:1034C0003F00000013040000983400083F00000093
:1034D00019040000A23400083F000000210400008D
:1034E000AC3400083F000000000000004D0F000851
:1034F000390F0008750F0008610F00086D0F0008F4
:10350000590F0008450F0008310F0008810F00080F
:103510000000000001000000000000006D61696E05
:103520000000000069646C6500000000243500089C
:10353000D823002050250020010000009D1800081D
:10354000000000004172647550696C6F7400254280
:103550004F415244252D424C002553455249414C80
:1035600025000000020000000000000069110008B2
:10357000D511000840004000E8290020F82900206B
:103580000200000000000000030000000000000036
:10359000191200080000000010000000082A002096
:1035A000000000000100000000000000B02C00201E
:1035B000010102008D1C00089D1B0008391C000839
:1035C0001D1C000843000000CC3500080902430020
:1035D000020100C0320904000001020201000524BA
:1035E0000010010524010001042402020524060044
:1035F00001070582030800FF09040100020A000018
:10360000000705010240000007058102400000009C
:1036100012000000183600081201100102000040DC
:1036200009124157000201020301000004030904CA
:1036300025424F41524425004D6174656B4634303C
:10364000352D626473686F7400303132333435362F
:1036500037383941424344454600000000400000ED
:103660000040000000400000004000000000010099
:103670000000020000000200000002000000020042
:103680000000020000000200000002000000000034
:103690005113000809160008B51600084000400044
:1036A000102D0020102D002001000000202D0020F2
:1036B00080000000400100000300000000008012B4
:1036C00000000000AAAAAAAA00000000FFBF000094
:1036D0000000000000A00A0000001400000000002C
:1036E000AAAAAAAA00001000FFFD00000000000026
:1036F000000000001500000000000000AAAAAAAA0D
:1037000015000000FFFF00000000000000000000A6
:103710000000000000000000AAAAAAAA0000000001
:10372000FFFF00000000000000000000000000009B
:1037300000000000AAAAAAAA00000000FFFF0000E3
:103740000000000000000000000000000000000079
:10375000AAAAAAAA00000000FFFF000000000000C3
:10376000000000000000000000000000AAAAAAAAB1
:1037700000000000FFFF000000000000000000004B
:1037800000000000000000000A000000000000002F
:103790000300000000000000000000000000000026
:1037A0000000000000000000000000000000000019
:1037B00000000000000000007D000000000000008C
:1037C00000000F0000000000FF009600000000084D
:1037D0000096000000000800040000002C360008DD
:1037E00000000000000000000000000000000000D9
:1037F0000000000000000000FFFFFFFFFFFFFFFFD1
:10380000FFFFFFFFFFFFFFFFFFFFFFFFFFFFFFFFC8
:10381000FFFFFFFFFFFFFFFFFFFFFFFFFFFFFFFFB8
:10382000FFFFFFFFFFFFFFFFFFFFFFFFFFFFFFFFA8
:10383000FFFFFFFFFFFFFFFFFFFFFFFFFFFFFFFF98
:020000040801F1
:1000000000060020C512010869700A08C56F0A08B9
:1000100031700A08C56F0A08FD6F0A08C712010887
:10002000C7120108C7120108C71201087DDC0C08BD
:10003000C7120108C7120108C7120108C712010838
:10004000C7120108C7120108C7120108C712010828
:10005000C7120108C712010815E80C083DE80C0892
:1000600065E80C088DE80C08B5E80C088D8C0C08C8
:10007000B58C0C08E18C0C080D8D0C08398D0C0822
:10008000618D0C088D8D0C08118C0C08C7120108AD
:10009000C7120108C7120108C7120108DDE80C08E1
:1000A00015EA0C0829EA0C083DEA0C0841EA0C089C
:1000B00045EA0C08C712010859EA0C0819930C0804
:1000C000C1940C08C7120108C7120108C712010821
:1000D000C7120108B1E90C08C5E90C08D9E90C08F8
:1000E00041E90C08C7120108C712010869EA0C08A7
:1000F0006DEA0C0881EA0C0885EA0C08B98D0C0839
:10010000C7120108C7120108C7120108C712010867
:10011000EDE90C0801EA0C08C7120108C712010832
:10012000E58D0C080D8E0C08398E0C08658E0C08B8
:10013000918E0C08C7120108C7120108C7120108E6
:10014000C7120108C7120108C7120108A9E30C0869
:10015000B98E0C08E58E0C08118F0C08C712010827
:10016000C7120108C7120108C7120108C712010807
:10017000C7120108C7120108C7120108C7120108F7
:10018000C7120108C7120108C7120108C7120108E7
:10019000C7120108C7120108C7120108C7120108D7
:1001A000C7120108C7120108C7120108C7120108C7
:1001B000C7120108C7120108C7120108C7120108B7
:1001C000C7120108C7120108C7120108C7120108A7
:1001D000C7120108C7120108C7120108C712010897
:1001E000913501085D670108F5A101089105020834
:1001F000D14E0208B1D60208955504082D14060800
:10020000351A060845770608E5DC0608A9E406085D
:10021000E1E70608514D0708896E0708A144080860
:100220005DB90808B5C6080841610A08E5660A080C
:1002300041640B08F1BE0B080DE60B08DDFB0B0853
:10024000692B0C0895310C0800000000000000002C
:1002500081F0004102E000BF83F0004330B54FEA77
:1002600041044FEA430594EA050F08BF90EA020FE4
:100270001FBF54EA000C55EA020C7FEA645C7FEA77
:10028000655C00F0E2804FEA5454D4EB5555B8BF9A
:100290006D420CDD2C4480EA020281EA030382EA0B
:1002A000000083EA010180EA020281EA0303362D9D
:1002B00088BF30BD11F0004F4FEA01314FF4801C70
:1002C0004CEA113102D0404261EB410113F0004F82
:1002D0004FEA03334CEA133302D0524263EB430339
:1002E00094EA050F00F0A780A4F10104D5F1200ED7
:1002F0000DDB02FA0EFC22FA05F2801841F1000132
:1003000003FA0EF2801843FA05F359410EE0A5F105
:1003100020050EF1200E012A03FA0EFC28BF4CF036
:10032000020C43FA05F3C01851EBE37101F00045EC
:1003300007D54FF0000EDCF1000C7EEB00006EEBF9
:100340000101B1F5801F1BD3B1F5001F0CD3490883
:100350005FEA30004FEA3C0C04F101044FEA4452DA
:1003600012F5800F80F09A80BCF1004F08BF5FEA61
:10037000500C50F1000041EB045141EA050130BD41
:100380005FEA4C0C404141EB0101013C28BFB1F553
:10039000801FE9D291F0000F04BF01460020B1FA9E
:1003A00081F308BF2033A3F10B03B3F120020CDA71
:1003B0000C3208DD02F1140CC2F10C0201FA0CF04F
:1003C00021FA02F10CE002F11402D8BFC2F1200CB4
:1003D00001FA02F120FA0CFCDCBF41EA0C0190406A
:1003E000E41AA2BF01EB0451294330BD6FEA0404B3
:1003F0001F3C1CDA0C340EDC04F11404C4F120029E
:1004000020FA04F001FA02F340EA030021FA04F3AF
:1004100045EA030130BDC4F10C04C4F1200220FA06
:1004200002F001FA04F340EA0300294630BD21FA44
:1004300004F0294630BD94F0000F83F4801306BF0A
:1004400081F480110134013D4EE77FEA645C18BFFE
:100450007FEA655C29D094EA050F08BF90EA020F95
:1004600005D054EA000C04BF1946104630BD91EA8D
:10047000030F1EBF0021002030BD5FEA545C05D190
:100480004000494128BF41F0004130BD14F58004CF
:100490003CBF01F5801130BD01F0004545F0FE4143
:1004A00041F470014FF0000030BD7FEA645C1ABF78
:1004B000194610467FEA655C1CBF0B46024650EAAF
:1004C000013406BF52EA033591EA030F41F40021DB
:1004D00030BD00BF90F0000F04BF0021704730B561
:1004E0004FF4806404F132044FF000054FF0000136
:1004F00050E700BF90F0000F04BF0021704730B5F7
:100500004FF4806404F1320410F0004548BF4042CB
:100510004FF000013EE700BF42004FEAE2014FEA20
:1005200031014FEA02701FBF12F07F4393F07F4FFB
:1005300081F06051704732F07F4208BF704793F0FE
:100540007F4F04BF41F40021704730B54FF4607411
:1005500001F0004521F000411CE700BF50EA010214
:1005600008BF704730B54FF000050AE050EA0102BD
:1005700008BF704730B511F0004502D5404261EB2D
:1005800041014FF4806404F132045FEA915C3FF46E
:10059000D8AE4FF003025FEADC0C18BF03325FEA0B
:1005A000DC0C18BF033202EBDC02C2F1200300FABC
:1005B00003FC20FA02F001FA03FE40EA0E0021FAE1
:1005C00002F11444BDE600BF70B54FF0FF0C4CF4CF
:1005D000E06C1CEA11541DBF1CEA135594EA0C0F81
:1005E00095EA0C0F00F0DEF82C4481EA030621EABC
:1005F0004C5123EA4C5350EA013518BF52EA0335F7
:1006000041F4801143F4801338D0A0FB02CE4FF0A8
:100610000005E1FB02E506F00042E0FB03E54FF0D8
:100620000006E1FB03569CF0000F18BF4EF0010ED0
:10063000A4F1FF04B6F5007F64F5407404D25FEACC
:100640004E0E6D4146EB060642EAC62141EA55517F
:100650004FEAC52040EA5E504FEACE2EB4F1FD0CC1
:1006600088BFBCF5E06F1ED8BEF1004F08BF5FEA3F
:10067000500E50F1000041EB045170BD06F00046F1
:1006800046EA010140EA020081EA0301B4EB5C049E
:10069000C2BFD4EB0C0541EA045170BD41F4801196
:1006A0004FF0000E013C00F3AB8014F1360FDEBFBB
:1006B000002001F0004170BDC4F10004203C35DA97
:1006C0000C341BDC04F11404C4F1200500FA05F31A
:1006D00020FA04F001FA05F240EA020001F00042BB
:1006E00021F0004110EBD37021FA04F642EB060131
:1006F0005EEA430E08BF20EAD37070BDC4F10C045B
:10070000C4F1200500FA04F320FA05F001FA04F21E
:1007100040EA020001F0004110EBD37041F100010A
:100720005EEA430E08BF20EAD37070BDC4F1200515
:1007300000FA05F24EEA020E20FA04F301FA05F27D
:1007400043EA020321FA04F001F0004121FA04F225
:1007500020EA020000EBD3705EEA430E08BF20EAF5
:10076000D37070BD94F0000F0FD101F0004640002F
:1007700041EB010111F4801F08BF013CF7D041EAB1
:10078000060195F0000F18BF704703F000465200B5
:1007900043EB030313F4801F08BF013DF7D043EA86
:1007A0000603704794EA0C0F0CEA135518BF95EA3C
:1007B0000C0F0CD050EA410618BF52EA4306D1D1C3
:1007C00081EA030101F000414FF0000070BD50EAE2
:1007D000410606BF1046194652EA430619D094EA6C
:1007E0000C0F02D150EA013613D195EA0C0F05D156
:1007F00052EA03361CBF104619460AD181EA0301AA
:1008000001F0004141F0FE4141F470014FF0000061
:1008100070BD41F0FE4141F4780170BD70B54FF0FC
:10082000FF0C4CF4E06C1CEA11541DBF1CEA13557C
:1008300094EA0C0F95EA0C0F00F0A7F8A4EB05045E
:1008400081EA030E52EA03354FEA013100F0888055
:100850004FEA03334FF0805545EA131343EA12631E
:100860004FEA022245EA111545EA10654FEA0026D3
:100870000EF000419D4208BF964244F1FD0404F58C
:10088000407402D25B084FEA3202B61A65EB0305E8
:100890005B084FEA32024FF480104FF4002CB6EBA5
:1008A000020E75EB030E22BFB61A754640EA0C0025
:1008B0005B084FEA3202B6EB020E75EB030E22BF65
:1008C000B61A754640EA5C005B084FEA3202B6EBA6
:1008D000020E75EB030E22BFB61A754640EA9C0065
:1008E0005B084FEA3202B6EB020E75EB030E22BF35
:1008F000B61A754640EADC0055EA060E18D04FEAF3
:10090000051545EA16754FEA06164FEAC30343EA92
:1009100052734FEAC2025FEA1C1CC0D111F4801F5F
:100920000BD141EA00014FF000004FF0004CB6E758
:1009300011F4801F04BF01430020B4F1FD0C88BFF7
:10094000BCF5E06F3FF6AFAEB5EB030C04BFB6EB02
:10095000020C5FEA500C50F1000041EB045170BDF5
:100960000EF0004E4EEA113114EB5C04C2BFD4EB22
:100970000C0541EA045170BD41F480114FF0000EA6
:10098000013C90E645EA060E8DE60CEA135594EA22
:100990000C0F08BF95EA0C0F3FF43BAF94EA0C0F25
:1009A0000AD150EA01347FF434AF95EA0C0F7FF49A
:1009B00025AF104619462CE795EA0C0F06D152EAEE
:1009C00003353FF4FDAE1046194622E750EA4106D2
:1009D00018BF52EA43067FF4C5AE50EA41047FF4E3
:1009E0000DAF52EA43057FF4EBAE12E74FF0FF3C48
:1009F00006E000BF4FF0010C02E000BF4FF0010C19
:100A00004DF804CD4FEA410C7FEA6C5C4FEA430C91
:100A100018BF7FEA6C5C1BD001B050EA410C0CBFE0
:100A200052EA430C91EA030F02BF90EA020F002042
:100A3000704710F1000F91EA030F58BF994208BFA9
:100A400090422CBFD8176FEAE37040F00100704766
:100A50004FEA410C7FEA6C5C02D150EA013C07D1BD
:100A60004FEA430C7FEA6C5CD6D152EA033CD3D008
:100A70005DF8040B704700BF8446104662468C4602
:100A80001946634600E000BF01B5FFF7B7FF002835
:100A900048BF10F1000F01BD4DF808EDFFF7F4FF5E
:100AA0000CBF012000205DF808FB00BF4DF808EDE9
:100AB000FFF7EAFF34BF012000205DF808FB00BF0C
:100AC0004DF808EDFFF7E0FF94BF012000205DF82E
:100AD00008FB00BF4DF808EDFFF7CEFF94BF0120E3
:100AE00000205DF808FB00BF4DF808EDFFF7C4FFDC
:100AF00034BF012000205DF808FB00BF4FEA410C25
:100B00007FEA6C5C02D150EA013C0AD14FEA430C07
:100B10007FEA6C5C02D152EA033C02D14FF0000044
:100B200070474FF0010070474FEA410212F5001282
:100B300015D211D56FF47873B3EB625212D94FEA24
:100B4000C12343F0004343EA505311F0004F23FA0E
:100B500002F018BF404270474FF00000704750EA63
:100B6000013005D111F0004008BF6FF00040704720
:100B70004FF00000704700BF4A0011D212F500127A
:100B800011D20DD56FF47873B3EB62520ED44FEAE5
:100B9000C12343F0004343EA505323FA02F0704765
:100BA0004FF00000704750EA013002D14FF0FF30A3
:100BB00070474FF0000070474FEA4102B2F1E04346
:100BC00024BFB3F5001CDCF1FE5C0DD901F0004C34
:100BD0004FEAC0024CEA5070B2F1004F40EB830084
:100BE00008BF20F00100704711F0804F21D113F1B0
:100BF0003872BCBF01F00040704741F480114FEAE9
:100C00005252C2F11802C2F1200C10FA0CF320FA71
:100C100002F018BF40F001004FEAC1234FEAD3238E
:100C200003FA0CFC40EA0C0023FA02F34FEA4303F8
:100C3000CCE77FEA625307D150EA01331EBF4FF081
:100C4000FE4040F44000704701F0004040F0FE409C
:100C500040F40000704700BF80F0004002E000BF99
:100C600081F0004142001FBF5FEA410392EA030F97
:100C70007FEA226C7FEA236C6AD04FEA1262D2EBE1
:100C80001363C1BFD218414048404140B8BF5B42E6
:100C9000192B88BF704710F0004F40F4000020F07F
:100CA0007F4018BF404211F0004F41F4000121F095
:100CB0007F4118BF494292EA030F3FD0A2F10102DF
:100CC00041FA03FC10EB0C00C3F1200301FA03F11D
:100CD00000F0004302D5494260EB4000B0F5000F40
:100CE00013D3B0F1807F06D340084FEA310102F1FF
:100CF0000102FE2A51D2B1F1004F40EBC25008BFB1
:100D000020F0010040EA03007047490040EB00007A
:100D1000013A28BFB0F5000FEDD2B0FA80FCACF17B
:100D2000080CB2EB0C0200FA0CF0AABF00EBC250A8
:100D300052421843BCBFD0401843704792F0000F96
:100D400081F4000106BF80F400000132013BB5E7E9
:100D50004FEA41037FEA226C18BF7FEA236C21D05F
:100D600092EA030F04D092F0000F08BF08467047C4
:100D700090EA010F1CBF0020704712F07F4F04D192
:100D8000400028BF40F00040704712F100723CBFA5
:100D900000F50000704700F0004343F0FE4040F4CF
:100DA000000070477FEA226216BF08467FEA23638D
:100DB0000146420206BF5FEA412390EA010F40F478
:100DC000800070474FF0000304E000BF10F00043C4
:100DD00048BF40425FEA000C08BF704743F09643AB
:100DE00001464FF000001CE050EA010208BF7047C6
:100DF0004FF000030AE000BF50EA010208BF70474D
:100E000011F0004302D5404261EB41015FEA010C61
:100E100002BF84460146002043F0B64308BFA3F159
:100E20008053A3F50003BCFA8CF2083AA3EBC2533B
:100E300010DB01FA02FC634400FA02FCC2F120025A
:100E4000BCF1004F20FA02F243EB020008BF20F091
:100E50000100704702F1200201FA02FCC2F12002F7
:100E600050EA4C0021FA02F243EB020008BF20EAEC
:100E7000DC7070477BB972B90029BEBF00204FF00B
:100E8000004106E008BF00281CBF6FF000414FF092
:100E9000FF3000F015BAADF1080C6DE904CE002961
:100EA00009DB002B1ADB00F0A3F8DDF804E0DDE934
:100EB000022304B07047404261EB4101002B1BDB71
:100EC00000F096F8DDF804E0DDE9022304B04042CA
:100ED00061EB4101524263EB43037047524263EBC3
:100EE000430300F085F8DDF804E0DDE9022304B0F7
:100EF000404261EB41017047524263EB430300F013
:100F000077F8DDF804E0DDE9022304B0524263EB38
:100F10004303704753B94AB9002908BF00281CBFD2
:100F20004FF0FF314FF0FF3000F0CAB9ADF1080CBF
:100F30006DE904CE00F05CF8DDF804E0DDE90223A1
:100F400004B0704730B1012390FAA0F0B0FA80F0FD
:100F50001844704708460029FBD02123F4E700BF5E
:100F6000430803F05533C01A830803F0333300F00D
:100F70003330184400EB101000F00F3000EB00206D
:100F800000EB0040000E704707EE900AF5EEC07AC5
:100F9000F1EE10FA01D400F00BB8F1EE677A08B563
:100FA00017EE900A00F004F8404261EB410108BDE1
:100FB000D0B5FFF7B1FA0C4B002206460F46FFF7FB
:100FC00003FBFFF7D9FD0446FFF784FA074B002225
:100FD000FFF7FAFA02460B4630463946FFF73CF96E
:100FE000FFF7CAFD2146D0BD0000F03D0000F041F2
:100FF0002DE9F047089D04468E46002B4DD18A42CC
:10100000944669D9B2FA82F252B101FA02F3C2F1FE
:10101000200120FA01F10CFA02FC41EA030E94408F
:101020004FEA1C48210CBEFBF8F61FFA8CF708FBB0
:1010300016E341EA034306FB07F199420AD91CEB88
:10104000030306F1FF3080F01F81994240F21C81BA
:10105000023E63445B1AA4B2B3FBF8F008FB103302
:1010600044EA034400FB07F7A7420AD91CEB040437
:1010700000F1FF3380F00A81A74240F20781644407
:10108000023840EA0640E41B00261DB1D44000238C
:10109000C5E900433146BDE8F0878B4209D9002DF0
:1010A00000F0EF800026C5E9000130463146BDE87A
:1010B000F087B3FA83F6002E4AD18B4202D38242E4
:1010C00000F2F980841A61EB030301209E46002D93
:1010D000E0D0C5E9004EDDE702B9FFDEB2FA82F2E8
:1010E000002A40F09280A1EB0C014FEA1C471FFA46
:1010F0008CFE0126200CB1FBF7F307FB131140EA2D
:1011000001410EFB03F0884208D91CEB010103F1F9
:10111000FF3802D2884200F2CB804346091AA4B2BB
:10112000B1FBF7F007FB101144EA01440EFB00FE8F
:10113000A64508D91CEB040400F1FF3102D2A645F4
:1011400000F2BB800846A4EB0E0440EA03409CE793
:10115000C6F12007B34022FA07FC4CEA030C20FA40
:1011600007F401FA06F31C43F9404FEA1C4900FA60
:1011700006F3B1FBF9F8200C1FFA8CFE09FB1811DD
:1011800040EA014108FB0EF0884202FA06F20BD950
:101190001CEB010108F1FF3A80F08880884240F2A0
:1011A0008580A8F102086144091AA4B2B1FBF9F0E4
:1011B00009FB101144EA014100FB0EFE8E4508D9DF
:1011C0001CEB010100F1FF346CD28E456AD9023864
:1011D000614440EA0840A0FB0294A1EB0E01A14249
:1011E000C846A64656D353D05DB1B3EB080261EBB7
:1011F0000E0101FA07F722FA06F3F1401F43C5E991
:10120000007100263146BDE8F087C2F12003D840C6
:101210000CFA02FC21FA03F3914001434FEA1C4708
:101220001FFA8CFEB3FBF7F007FB10360B0C43EAFA
:10123000064300FB0EF69E4204FA02F408D91CEBAA
:10124000030300F1FF382FD29E422DD902386344A8
:101250009B1B89B2B3FBF7F607FB163341EA034148
:1012600006FB0EF38B4208D91CEB010106F1FF3897
:1012700016D28B4214D9023E6144C91A46EA00468E
:1012800038E72E46284605E70646E3E61846F8E620
:101290004B45A9D2B9EB020864EB0C0E0138A3E769
:1012A0004646EAE7204694E74046D1E7D0467BE74A
:1012B000023B614432E7304609E76444023842E7C2
:1012C000704700BF02E000F000F8FEE772B6374852
:1012D00080F30888364880F3098836483649086024
:1012E00040F20000CCF200004EF63471CEF2000164
:1012F0000860BFF34F8FBFF36F8F40F20000C0F262
:10130000F0004EF68851CEF200010860BFF34F8F17
:10131000BFF36F8F4FF00000E1EE100A4EF63C7104
:10132000CEF200010860062080F31488BFF36F8FAF
:10133000BCF002FDBBF030FD4FF055301F491B4A99
:1013400091423CBF41F8040BFAE71D49184A91420B
:101350003CBF41F8040BFAE71A491B4A1B4B9A425F
:101360003EBF51F8040B42F8040BF8E7002018497F
:10137000184A91423CBF41F8040BFAE7BCF0E0FC8C
:10138000BBF05EFD144C154DAC4203DA54F8041B5F
:101390008847F9E702F0ECF8114C124DAC4203DA41
:1013A00054F8041B8847F9E7BCF0C8BC00060020CD
:1013B000002200200000010808ED00E000000020ED
:1013C00000060020407C0F0800220020942C002002
:1013D000982C0020C85B0120E001010848020108A8
:1013E00048020108480201082DE9F04F2DED108A4E
:1013F000C1F80CD0C3689D46BDEC108ABDE8F08FE3
:10140000002383F311882846A0470020BBF036FA5A
:10141000FEE7BBF093F800DFFEE7000001F0FF01FC
:10142000102A2BDB10F0070F08D010F8013B013A0F
:101430008B422DD010F0070F42B3F6D1F0B441EA41
:10144000012141EA014122F007047FF00007002357
:10145000F0E80256083C85EA010586EA010685FAAD
:1014600047F5A3FA87F586FA47F6A5FA87F68EB907
:10147000EED1F0BC01F0FF0102F0070232B110F82A
:10148000013B013A83EA010313B1F8D10020704710
:1014900001387047002D06BF35460338073815F070
:1014A000010F07D1013015F4807F02BF013015F420
:1014B000C03F0130F0BC0138704700BF10F8012B6D
:1014C00011F8013B012A28BF9A42F7D0D01A704781
:1014D000034613F8012B002AFBD1181A0138704774
:1014E00038B50022002304460D46FFF7DFFA28B97D
:1014F00020462946BDE8384000F00AB8204605F1EC
:10150000004100F005F8404261EB410138BD00BFE9
:10151000D0B50C4B002206460F46FFF755F8FFF7F3
:101520002BFB0446FEF7D6FF074B0022FFF74CF8D3
:1015300002460B4630463946FEF78EFEFFF71CFB8F
:101540002146D0BD0000F03D0000F04103680022BC
:101550001B6818477FB503914021054683F062FF61
:10156000039A18B90124204604B070BD134E0392AB
:1015700096F98633002BF5D063F020FE437A039A68
:1015800053B963F01BFE847A039A2CB90C4B4021AB
:10159000284683F04FFFE6E7D6F87C3DB6F988137E
:1015A000B3F906309942DDDD064B00934021064B2E
:1015B000284683F03FFF0024D5E700BFA04C002061
:1015C0008C620D08AB620D0899620D08F0B50D46EE
:1015D0009DB02021044683F025FF002800F09D8067
:1015E0004F4E96F98633ABB1D6F87C2DB6F98833D9
:1015F000B2F90A1003F10A02914203DD40F28D3282
:10160000934207DC474B2A462021204683F012FFF5
:10161000002080E096F97533022B05D1424B2A4613
:101620002021204683F006FFB6F84833A3F57A73ED
:101630009BB241F6583293420DD83C4F96EDED7A6D
:10164000D7F8BC3DD3ED097AB4EEE77AF1EE10FAA3
:1016500003DD374BD7E7374BD5E796EDEE7AD3ED81
:101660000B7AB4EEE77AF1EE10FAF2DCB6F98233D7
:10167000002B01DC304BC6E796F814240D2A06D85F
:101680000123934013F4215F01D02C4BBBE72C487E
:1016900010F054FA012806D1D7F8C80D8AF060FF7F
:1016A00098B101281AD00021602204A80391C0F04B
:1016B0009FFA2449D7F8C40D642303AA8AF038FBA3
:1016C00000BB03AB0093204B02E0204B0093204B68
:1016D0002A462021204683F0ADFE99E796F8903DFA
:1016E00073B11C48192150F019FB48B11948D6F8BC
:1016F0006063192150F038FB8642D4DD164BE5E7D4
:10170000164BE3E71649D7F8BC0D642303AA87F00C
:10171000CFF90028D5D01DB0F0BD0120FBE700BFF8
:10172000A04C0020B4620D08C7620D08A06C002018
:10173000FF620D08EF620D0819630D082E630D0896
:10174000B48B0020A8630D08AC630D0873630D080B
:101750004E630D08E039002092630D0883630D0885
:10176000BE630D0807B504488CF07CFA00F0010058
:1017700003B05DF804FB00BF407A00202DE9F04380
:10178000DFF844910446D9F88C010368A5B01B69C1
:101790000D469847804615F01BFD00210746602244
:1017A0000CA80B91C0F024FA64230BAA41463846DA
:1017B00015F002F8064648B93A4A0BAB29462046CE
:1017C00084F034F8304625B0BDE8F083A9F56160B7
:1017D00071F0C8F8B8F1000F03D194F91E30012B55
:1017E0000AD1314812F0BAFC80B9304A2946204665
:1017F00084F01CF80026E5E710F0060FE2D0A9F50A
:10180000405012F0ABFC08B9294AEFE703A938466B
:1018100014F004FE28B19DF80D305B0601D5254A71
:10182000E4E7DFF8A880D8EDE97AF5EEC07AF1EECA
:1018300010FA4FF00003C5DD089309930A930DF1E8
:10184000200907AB019305AA06AB04A9CDF80090C7
:10185000384615F0C5F9484630F058FED8EDE97A1B
:10186000B4EEE70AF1EE10FA01DB134ABEE79DED94
:10187000057AF4EEC77AF1EE10FA01D80F4AB5E70F
:101880009DED047AF4EEC77AF1EE10FA01D80C4A15
:10189000ACE79DED067AF4EEC77AF1EE10FA91D836
:1018A000084AA3E7C4630D08A02C0020CD630D08EF
:1018B000E4630D080A640D0818640D082D640D0812
:1018C00043640D0859640D08A05C0020A04C002062
:1018D00008B5064B93F8A5319B0704D5044A83F05D
:1018E000A5FF002008BD0120FCE700BFA05C002090
:1018F00070640D0870B50C4C0546D4F88C01036873
:101900005B690E46984710B10124204670BDA4F5CE
:10191000405012F035FC04460028F5D1034A314608
:10192000284683F083FFF0E7A05C002080640D0868
:101930002DE9F046464ED6F8B03193F8CB509BB027
:1019400081468A4665B9434B1B68986A03685B6B9E
:101950009847044640B9404A5146484683F066FFDE
:1019600028461BB0BDE8F08663F028FC202164F017
:101970009BFC58B163F022FC1F2164F095FC88B3F6
:10198000364A5146484683F051FF002496F882318A
:1019900003F01403142B05D1314A5146484683F015
:1019A00045FF00245146484684F038FE0021884215
:1019B0004FF0600202A808BF0C460191C0F018F970
:1019C000D6F8B001036801AA1B6864219847054650
:1019D00080B9244A01AB5146484683F027FF2C4684
:1019E0002546BDE763F0EAFBA52164F05DFC002815
:1019F000C6D1CBE7002CF3D0D9F808303BB9D9F8E1
:101A0000003051465B6B484698470446E8E751462C
:101A10004846FFF7DBFD514607464846FFF758FFAB
:101A20003840C4B251464846FFF794FD5146044041
:101A30004846FFF75FFF51460440484683F01EFFCB
:101A400051460440484684F001FE0440C8E700BF08
:101A5000A05C0020408E002094640D08AB640D084B
:101A6000C5640D08DD640D0808B5FFF761FF054A80
:101A700092F8801160F3041182F88011024A90718B
:101A800008BD00BFA05C00201D900020F7B50546F2
:101A90000F4683F06BFC044678B10221284683F0A0
:101AA000C1FC064648B115488CF0DCF8C205C0F30D
:101AB0000723C0F3002403D53446204603B0F0BD0D
:101AC0009B07F9D50D488CF0DBF80D4B03F66C53F2
:101AD000D3ED007AF8EEE77A30EE670ADFED097AA7
:101AE000B0EEC00AB4EEE70AF1EE10FAE4DD064B00
:101AF0003A460221284683F09DFCDEE7407A00202A
:101B0000A06C00200000C842E8640D08F8B5044647
:101B10000F4683F053FF10210546204683F082FCD8
:101B200058B12046FFF71EFE064630B9044B3A4630
:101B30001021204683F07EFC35462846F8BD00BFC4
:101B4000FC640D0870B505460E4683F00FFC044694
:101B500078B18021284683F065FC50B1074B93F89B
:101B60004D3743B1064B32468021284683F062FC54
:101B70000024204670BD0446FBE700BFA05C0020A7
:101B800010650D0838B50D4D0446D5F8C80D8AF01E
:101B9000E7FC012810D0D5F8C80D8AF0E1FC022836
:101BA00004D02046BDE8384083F0E2BB04480FF083
:101BB000C5FF0128F5D138BD0020FCE7A06C00204E
:101BC000B48B0020F0B5134C04F5005385B0D3F866
:101BD000742D0092D3F8782D0192D3F87C2D0292C7
:101BE000D3F8803D03936A4606460F4684F0C8FC4E
:101BF00039460546304683F051FC04F540542840F0
:101C000094F8803160F3C303C3F3C00084F88031DB
:101C100005B0F0BDA02C00202DE9F843064627486A
:101C2000DFF8A890DFF8A8800F4670F09BFE04460E
:101C3000D9F88C0103681B699847054630B914F040
:101C4000060F03D1D9F8C031022B09D139463046ED
:101C500083F010FD054618B9002488F807400AE013
:101C600039463046FFF78AFD04460028F4D02DB9E6
:101C7000012388F807302046BDE8F8830821304664
:101C800083F0D0FB0028F3D00D4823F0D1FC0028CE
:101C9000EED00C4B93F81424B02101FB023203F573
:101CA0000053B2F81E22B3F976339A42E0DD064BB8
:101CB0003A460821304683F0BDFBCDE7904E002028
:101CC000C02D0020A02C002024650D08A05C002061
:101CD0001D9000202DE9F3410E46054615F078FAD7
:101CE000804614F05DFB044640B9514A0121284664
:101CF00083F09CFD204602B0BDE8F0814D4FD7F83F
:101D00008C01036831469B699847044658B9D7F857
:101D10008C0103681B6C9847474A034601212846FB
:101D200083F084FDE6E7AB68002BE3D01021284662
:101D300083F078FB20B3D8ED937A98ED920A20EEE9
:101D4000270ABDF0F7FCDFED3D7AA7F5805320EEC2
:101D5000270AB3F94833DFED3A7A20EE270A07EE77
:101D6000903AF8EEE77AB4EEE70AF1EE10FA07DD02
:101D7000344B01221021284683F05CFB0024B9E794
:101D80004021284683F04EFB38B3012E1ED0232E6F
:101D90001CD0042E1AD02C4CD4F87C3DB3F908305A
:101DA00000EE103AA4F50050B8EEC00A00F0BEFBF9
:101DB000B5EEC00AF1EE10FA1DDD244B00930122AE
:101DC000234B4021284683F035FBD7E7D7F88C0119
:101DD0000368DB6B98470028DDD01E4B1B68D86A70
:101DE0000368DB6998470128014619D11A4A284639
:101DF00083F01CFDC2E7D7F88C0103685B69984744
:101E000030B1D4F87C3DB3F90830002BE5DDD4E7E0
:101E1000D7F88C0103681B6898470B28DDD1F0E7E1
:101E20003146284602B0BDE8F04184F08FB800BFCB
:101E300034650D08A05C002045650D08E02E654264
:101E40000000C84259650D08A04C0020AB620D0887
:101E500061650D08408E00206D650D0870B5054662
:101E60000E46FFF78BFC084B0446D87131462846D6
:101E7000FFF740FD31460028284608BF002484F0C3
:101E80005BFA204070BD00BF1D9000202DE9F0419D
:101E90004E4F3B78002B40F096804D4CD4F8B0511B
:101EA00095F8CB5001263E701DB13B702846BDE829
:101EB000F08184F079FC054630B9464A38701378D1
:101EC00043F001031370F1E757F018FC314656F068
:101ED00001FCA4F5405006F0C1FD3F4B1E710B26DE
:101EE0004BF04AF8013E4BF015F816F0FF06F7D11B
:101EF0003A4800F089FF15F06BF9D0F80022C4F8D9
:101F0000D82190F87C32DA074DD414F0CBFC57F08E
:101F1000F5FB3C2157F08AF90023C4F898310021E1
:101F20002E482F4E00F0F6FF2C4812F017F901460C
:101F30002C488FF009FE2C4B1B68D86A03680121DE
:101F40001B689847D4F8B00103689B6A9847012141
:101F5000D4F8B0018CF040FE57F0D0FB8046D4F8A6
:101F60008C0103681B68984796F808230146404691
:101F700056F08CFDA6F5005006F062FD53F0E4FA31
:101F800052F020FE00233B7095F0A0F8B4F88231A7
:101F900006F5005623F4087343F02003C6F8D40D69
:101FA000A4F8823182E79B07B9D431460B4804F08C
:101FB000CDFD0E488BF064FEDFED0D7A20EE270A92
:101FC00084ED660AABE7002570E700BF982C00207F
:101FD000A05C00203C9000201D900020A02C002040
:101FE000A04C00201C580020408E0020407A002089
:101FF0000AD7233C2DE9F043374DD5F8B03193F89B
:10200000CB3087B0002B64D062B1012901D02329E5
:1020100008D195F98031002B04DB0024204607B05D
:10202000BDE8F08384F076FC04460028F5D015F076
:10203000CFF807461CF016F98046384613F0BAFE72
:10204000D8B198F92430022B17D100264FF000099F
:10205000F1B203AA38460191CDF80C90CDF810905A
:10206000CDF8149014F044FA019918B103AA40462F
:102070001BF0A8FD0136032EEAD11848012106F015
:102080005BFF1648012106F08BFE0021D5F8B00158
:102090008CF0A2FD124832F075FF57F02FFB0021A3
:1020A00056F018FB0F4B1B68D86A036800211B68A9
:1020B000984795F88231D5F88C110B486FF345138A
:1020C00085F882310B1A594259413C3092F022FF77
:1020D000A4E70124A2E700BFA05C0020A02C002000
:1020E000A0850020408E00203C87002010B5064CC3
:1020F000D4F88C0103685B6A984718B1D4F8B03102
:1021000093F8CB0010BD00BFA05C002030B52DEDD2
:10211000028B89B00C46B0EE408AFFF7E7FF054618
:10212000002838D0B4EE488AF1EE10FA7CBFDFED1B
:102130001C8ADFED1C7A226863689FED1A0A68BF6B
:10214000DFED198A029278BF68EE288A02A878BF6C
:1021500068EEA78AD4ED027A0393F1EE677ACDEDAB
:10216000047A2FF0D5FDB4EE488A00220123F1EE67
:1021700010FACDE900238DED050ACDED060A9FED9D
:102180000A0A0A488DED071AF0EE680A68BF13467E
:1021900005A90DF0B1FD284609B0BDEC028B30BD9C
:1021A000E02E65420000C84200000000588A00206E
:1021B00007B50191FFF79AFF30B10199044803B0C8
:1021C0005DF804EB00F0FABA03B05DF804FB00BF61
:1021D000A02C0020014870F051BD00BF904E00209F
:1021E00008B500F5405090F88031C3F340128A42A0
:1021F0000BD061F3451380F8803131B157F07EFA8E
:10220000BDE808400F2157F011B808BD70B500F5C2
:1022100040560546D6F8C0318B420C4612D00129F3
:1022200011D0022916D059B957F068FA1B2156F07F
:10223000FDFF0D4A05F53D50062118305AF0E2FB2E
:10224000C6F8C04170BD57F059FA1A2156F0EEFF9A
:10225000064AEFE7012100F05DFE57F04FFA1D211D
:1022600056F0E4FF024AE5E7D8650D08ED650D0874
:10227000E8650D0810B500F540520C4692F8A531FE
:1022800003F00101A14209D064F3000382F8A531F3
:10229000DB0704D405F0B0FF024B9C7210BD06F0C2
:1022A00093F9F9E71D90002000F5405090F8A53112
:1022B00061F3410380F8A531014B1973704700BFEA
:1022C0001D90002010B5044662F078FF202163F0D5
:1022D000EBFF04F54053003893F8822118BF01202A
:1022E00060F3820283F8822110BD000010B504461D
:1022F00053F02AF904F54052436FD2F8B02104F5A7
:102300008044D360D4F8BC2D9366D4F8C42DC2F8B1
:10231000FC32D4F8BC0D03685B6D9847D4F8BC0D53
:102320000368BDE810409B6D1847000070B52DEDA7
:10233000028B00F540550446D5F8B03193F8CB3008
:10234000002B74D095F98031002B70DB00F5A04391
:1023500093F82438002B6AD1D5F88C0103685B69A7
:102360009847002863D1334BD3F88C0103681B686E
:1023700098470B285BD004F580469FED2F7AD6F85E
:10238000C43DD3EDDB7AF0EEE77AF4EEC77AF1EEF6
:1023900010FA4CD5D5F8B001443059F069FE034627
:1023A000DFED260A93ED000A9F20B7EE001A2CF00D
:1023B00059FAB5EEC00AF1EE10FA38DD04F59B408B
:1023C00020308BF069FCDFED1E7AB0EEC00AB4EE6F
:1023D000E70AF1EE10FA2AD504F58054D6F8BC0DC0
:1023E000D4F8083507EE903A0368D3F89830B8EE81
:1023F000E78A984738EE400ADFED127AB0EEC00A5D
:10240000B4EEE70AF1EE10FA11D5D4F80C3540F22B
:10241000E63203F2F313934209D8BDEC028BD5F8F0
:10242000B0019FED090ABDE870408DF057BEBDECCC
:10243000028B70BDA05C0020000000340000000092
:10244000000070420000FA430AD7233C08B500F5AB
:102450004050D0F8B00103681B699847F6EE007A47
:1024600020EE270AB5EEC00AF1EE10FA48BF9FED44
:10247000010A08BD0000000038B52DED028B00F503
:1024800080450446D5F8BC3DDFED110A93ED370ACF
:1024900004F540547120B7EE001A2CF0E3F9D4F89B
:1024A000B001D5F8C45D03681B69B0EE408A984757
:1024B00038EE400ABDEC028BDFED067A05F50575B6
:1024C000284620EE270ABDE838407BF0BFBF00BF9A
:1024D0000000000000007A4400F5AB53D3ED005A31
:1024E000D2ED007AD3ED036A91ED006A26EEE77A29
:1024F00067EEA57AA6EE257AE6EE267A81ED007AD9
:10250000C2ED007A7047000000F50050B0F92C3C95
:1025100033B9B0F982030028B8BF404280B2704797
:1025200083EAE370A0EBE370F8E7000070B52DEDEF
:10253000028B00F5405382B093F8A51111F001060B
:10254000044605D09FED2E0A02B0BDEC028B70BD93
:102550008DED010A62F032FE037F002BF2D0DFED39
:10256000298ADFED270A9DED010AB0EE681A4E2098
:102570002CF078F904F500554FF4C8723146B5F9DE
:102580008A03B0EE408A2CF0ABF9A5F88A03204606
:1025900011F08CFBB5F98A3307EE900AB8EEE77AB2
:1025A00007EE903AF8EEE77A77EE676AB4EEE68ADD
:1025B000F1EE10FA0DD52046FFF7A6FF07EE900AC0
:1025C00038EE668AB8EEE70A20EE088A88EE260A18
:1025D000BAE777EE877AB4EEE78AF1EE10FAB1DD6A
:1025E000B5F9823300EE103A38EE678AB8EEC00AC9
:1025F00078EEE77A20EE088A88EE270AA4E700BF83
:102600000000000000007A4400207047002070475E
:102610007047000000F50E501830704700487047B2
:10262000E8950D0800F54050D0F88C0103681B6850
:1026300018470000034808603321117008221A600F
:10264000704700BFA4690D0800F54050D0F88C0118
:102650000368DB6C1847000000F54050D0F88C018F
:1026600003689B6C1847000000F5405300F5B1402B
:10267000D3F88C3144301B1A58425841704700003F
:1026800010B500F540500C46D0F88C010368DB6DA6
:10269000984707EE900A9FED057AF8EE677A0120D9
:1026A00067EE877AC4ED007A10BD00BF0AD7233CDD
:1026B00010B500F540500C46D0F88C0103689B6DB6
:1026C000984707EE900A9FED057AF8EEE77A012029
:1026D00067EE877AC4ED007A10BD00BF0AD7233CAD
:1026E00010B500F540500C46D0F88C0103681B6E05
:1026F0009847DFED047A20EE270A012084ED000AD6
:1027000010BD00BF0AD7233C69F088BB12F056BC4D
:102710006DF002B864F0FEBF52F060BE29F0DCBF7D
:1027200056F05AB918F0E4BB65F074BB62F0A0B97A
:1027300060F0AABA10F052BF11F0AEBB06F038BE7E
:1027400012F0CEBB05F0ACBD05F0F8BA05F01EBA2C
:102750006BF018B910F090B8FFF7E8BD11F082B82F
:1027600011F0F2BA03F0A0B911F006B810F07EBF74
:1027700062F072BC4BF0FEBD24F008BA06F0DAB984
:1027800002F05ABD65F056BB11F0FCBA06F0C8BDA8
:1027900004F0C8B906F01EBF05F08ABA06F07ABA8E
:1027A00010F0A8BEFFF7A2BD2AF0B4BA05F08ABFA8
:1027B0000AF0F6BA0AF0E0B90AF074B91FB500F5EC
:1027C00040530446D3F88C01039103685B6A984731
:1027D00060B1DFED070A0399002304F5BB400093C5
:1027E000B0EE600A1A4638300DF0DCF804B010BDC7
:1027F0000000000010B52DED028B00F5405304469B
:10280000D3F88C0103685B6AB0EE408A984720B920
:102810000024BDEC028B204610BD9FED080A04F594
:10282000BB4028EE000A38300CF086FB0446002836
:10283000EED003480121FFF7D3FCEAE70000C842CD
:10284000A02C00200A4A92F98021002A0B4605DAC2
:1028500000228A604A600A600120704700F58040CB
:10286000D0F8BC2D783207CA83E80700F4E700BF30
:10287000A05C002070B5204B036000F500531F4A98
:10288000C3F8582F00F540530446D3F8140108B19B
:102890001AF020FF1A4B236004F5805393F8D42FCD
:1028A00042B9D3F8D05F2DB1284628F01DFD284647
:1028B0001AF00CFF04F59050183081F0FDFF04F57C
:1028C000895065F05BF904F6F44504F69446B54288
:1028D00004D0183D284628F05DF9F8E7094BC4F804
:1028E000C83804F6C41059F09FF804F5136059F085
:1028F0009BF8204670BD00BFB06D0D08D87B0E0858
:10290000BC590E081C230E0838B54C4B044640F841
:10291000043B69F0A3FB04F1100017F063FF04F11E
:10292000680052F0E9FA04F5907022F091FD04F588
:102930008C6016F0D9FC04F284501AF0CDFE04F637
:10294000C80029F06DFD04F5476069F065F904F5EC
:1029500054604FF009F904F57F6055F00BFE04F563
:10296000885004306FF0E0FA04F5895065F0EEF815
:1029700004F58A501C3019F09FFC04F59050183073
:1029800081F086FF04F59150143052F077FE04F583
:10299000945008306AF040FD04F580530025284A21
:1029A00083F8AC5204F5955004F595530C331C3064
:1029B00013604AF023F904F598502946103012F0BC
:1029C000E9FE04F5CB507BF07FFF04F5F3500430B3
:1029D0007EF07EFF04F5FB501C3081F0B3F804F567
:1029E000FF5081F0E9FC04F50050383012F0D4FCBF
:1029F00004F5065018307CF039FD04F507503030EE
:102A00006FF054FE04F50A50303082F0DDFA04F520
:102A1000005304F50C5083F808530A4D203082F01F
:102A2000F5FB2B6813B1084894F022FB20460749B8
:102A30004DF060FF2C60204638BD00BFBC590E0829
:102A4000009A002008910020FC650D08C4580E086B
:102A500010B511F09FF862F0B1FB0368BDE81040BB
:102A60005B681847FFF7F4BF10B5044606F0B0F9ED
:102A7000204611F09DFB204603F09EFE2046BDE857
:102A8000104004F005B80000FFF7EEBF70B500F588
:102A900047551C350446284617F07EFD1BF0E2FB27
:102AA00090F9213093B390F840337BB304F5405351
:102AB00004F28456D3F8B001443059F0D9FA0346F1
:102AC000DFED130A93ED000A9F20B7EE001A2BF0FA
:102AD000C9FE94F9B835012B284608BF86ED0E0AC9
:102AE000002117F0EDFADFED0B7A04F2DC7494EDBF
:102AF000287A20EE270ADFED087AA7EE270A30466B
:102B000084ED280ABDE870401BF0BCBA70BD00BF60
:102B100000000000CDCCCC3D6666663FFFF7B6BF37
:102B200010B50121044611F07FFB60B1114BD3F8C1
:102B30008C0103689B6A984728B9204602F08AFAFC
:102B4000204602F097FA4FF40011204611F06CFB7A
:102B500018B12BF059F929F03FFB4FF480212046A2
:102B600011F062FB28B12BF04FF9BDE8104029F0BD
:102B700041BA10BDA05C0020FFF7D2BF70B500F5D0
:102B800080450446D5F8BC0D9FED5A0A86B06C30DE
:102B90002FF0BEF804F5985003A910308DED030A0C
:102BA000CDED040A8DED051A12F0A0FC022120469D
:102BB00011F03AFB70B10121204611F035FB48B904
:102BC0004D4BD3F88C0103689B6A984710B9204697
:102BD00002F040FA0121204611F026FB48B9464B8D
:102BE000D3F88C0103689B6A984710B9204602F01D
:102BF00041FA0121204611F017FB10B9204602F0DE
:102C000091FA4FF40031204611F00EFB30B104F57B
:102C10004053D3F8B00103685B6C984740212046CD
:102C200011F002FB60B104F57F60019055F068F887
:102C300004F58053019893F920310BB155F0A2F9B6
:102C40004FF48061204611F0EFFA18B104F57F606F
:102C500055F0F0F82021204611F0E6FA58B104F5BD
:102C60004056D6F88C0103681B69984718B3D5F80D
:102C7000C40D87F099FF8021204611F0D5FA38B3B2
:102C80002BF0C2F829F0DAF91021204611F0CCFA25
:102C900018B1D5F8BC0D84F0CDFC4FF400412046AE
:102CA00011F0C2FA18B304F59C405C3006B0BDE8E0
:102CB000704065F0F1B920460DF02EFD0028D6D108
:102CC000D6F88C0103685B6998470028CFD0D2E71B
:102CD0004FF48021204611F0A7FA0028D0D14FF4FC
:102CE0000021204611F0A0FA0028C9D1CCE706B097
:102CF00070BD00BFE02E6542A05C0020FFF73EBF24
:102D000010B50121044611F08FFA10B1204602F0EF
:102D100009FA8021204611F087FA58B14FF480213A
:102D2000204611F081FA28B92BF06EF8BDE810406A
:102D300029F060B910BD0000FFF7E2BF10B50446EE
:102D400005F094FD204605F0DFFB204605F0D4FD9C
:102D5000204612F057F92046BDE8104003F008BDA8
:102D6000FFF7ECBF70B54FF6FF71044611F05CFA47
:102D700004F5405528B1D5F880210721204602F0FE
:102D800001FAD5F8B03193F8CB308BB92046FFF774
:102D900099FAD5F8B00104F50053026893F81414B9
:102DA000166A93F89E23B047D5F8B0018DF062F90A
:102DB00064F064F863F060FD204612F015F995F8B0
:102DC00080310F4A04F58044DB43D4F8BC5DC3F383
:102DD000C01353712B681E6F52F0B6FB52F01EF8F1
:102DE0002846B047D4F8C44D52F0AEFB04F5057444
:102DF00052F014F82046BDE870407BF08DB900BF5A
:102E00001D900020FFF7AEBF70B500F5AB5300F585
:102E100040551B68C5F8C43100F5805606F26C5366
:102E200004461B68C5F8C831D6F8100500F58C407B
:102E300050302BF0EBFCD5F8C431C5F8D031D5F8C3
:102E4000C831C5F8CC01C5F8D4314FF6FF71204622
:102E500011F0EAF938B1D6F8102520460921BDE86D
:102E6000704002F067B970BD30B500F54053D3F83B
:102E7000C041002C4CD093F88121D10748D56FF385
:102E8000000283F8812100F50052012CD2F8741D54
:102E9000D2F8785DB1F908400BBFD3ED725AD3ED8B
:102EA000755AD3ED717AD3ED747A07EE104AB5F9FD
:102EB000084006EE904A0CBFF8EEE66AF8EEE66AC5
:102EC000B8EEC77A25EEE66A00F5AB53A7EE276A9F
:102ED00067EEA67AD3ED006AE7EE257A93ED037AE2
:102EE00027EE877AA6EE267ABDEEC77A17EE104A4D
:102EF0000C8193ED007AD2F8782D67EE877A93ED06
:102F0000037AE6EE477AFDEEE77A17EE903A138100
:102F100030BD000038B505462DED028B00F540545C
:102F200071B1284610F0BEFCD4F8CC311B1A03F264
:102F3000F31340F2E63293420CD8BDEC028B38BD5D
:102F4000D4F8C031022BF8D110F090FCB0F57A7FA4
:102F5000E7D2F2E7C4F8CC0100F58C40503064238E
:102F600090FBF3F308EE103ADFED097AB8EEC88A69
:102F700028EE278AB0EE480ABCF0F2F984ED740A14
:102F8000B0EE480ABCF072FB84ED750AD5E700BFCD
:102F900035FA8E3C00F598500121103014F07CB8C1
:102FA000FFF7F8BF10B5044610F086FE102120464A
:102FB00011F03AF970B1204601F09AFF4FF4001178
:102FC000204611F031F928B92AF01EFFBDE8104063
:102FD00029F002B910BD0000FFF7E4BFF8B50446C0
:102FE000254606F021FA224B45F83C3B214BA465CF
:102FF000C4E91734204BC4E91934204BE36604F1CB
:10300000800019F0A5FF04F19C0019F0A1FF04F164
:10301000B80019F09DFF4FF6FF76194BC4F8CC307D
:10302000A4F8D06004F1D40019F092FF4FF0FF37FC
:10303000144B1549C4F8307128461D604DF05AFCF8
:10304000A4F87870A4F8946004F5A27019F080FFD9
:1030500004F5B07019F07CFF04F5BE7019F078FF2C
:10306000002384F89031C4F8B4312046F8BD00BF85
:10307000B8C20D08B1270108B5270108B927010812
:103080000000FFFFE88F002000300E0810B5044656
:1030900006F0CAF90A4B23600123A38704F140001C
:1030A00019F056FF04F1500019F052FF04F16000CE
:1030B00019F04EFF04F1700019F04AFF204610BDD0
:1030C0009CCC0D082DE9F043044689B0FFF71CFCA9
:1030D000A74B236004F50F5004F5005502F088F962
:1030E00004F50E530C3304F53657C5F8883D062316
:1030F00085F88C3D4FF07C5805A907F11800CDF8F4
:10310000148059F0A7F807F1300092F0A7FE04F5FB
:103110009B460023203604F5375785F8C83D192310
:1031200004A985F8D43DC5F8D06D07F12000CDF88D
:10313000108059F08FF807F1380092F08FFE4FF0B1
:103140000108182304F5385004F53A5785F81C3E59
:10315000183785F8108EC5F8186E303064F008F90D
:10316000384682F00FF906AE824BC5F8983E3146DC
:10317000381D8DF818804EF0D3F904F53B5010300F
:103180004BF0B6F804F53C50103082F0E5F87A4B7D
:103190007A4FC5F8103F04F53C5031462830069769
:1031A00059F058F804F53C5031463430069704F590
:1031B0003D5959F04FF8314604F53D50069709F155
:1031C000180959F047F86E4BC5F8583F09F114003B
:1031D00092F044FE04F53E5704F53F58103708F1CD
:1031E0003408384614375DF017FEB845F9D104F5B8
:1031F00040580723C8F818310023A8F81C314FF4B1
:10320000CB701AF061FAC8F8140104F5445020306C
:1032100092F024FE04F54550243092F01FFE594BE5
:103220001A680AB9C3F8009004F5BF47564BC5F8B1
:10323000583F203704F54650C8F88C71103083F0A1
:1032400089FB524B07934FF07E55514BC8F8C45140
:10325000C8F8D0510694009304F5475096E80C0046
:103260004FF400711C3016F0DDFD04F55D50103098
:1032700073F0C4F904F59A4003A97030039559F02E
:103280000FF804F59B4003A90430039558F0E2FFC2
:1032900004F59B4004F58045103019F059FE05F502
:1032A0005A6300261E605E609E6005F6AC5304F50E
:1032B0009B401E605E609E6004F598531033C5F815
:1032C000B83D002385F8D93D4FF400415C3017F03C
:1032D00095FB04F59C405C3064F086FD04F59D4050
:1032E000603071F019FB04F59E401C304EF04EFA30
:1032F000284BC5F81C3F04F59E40274B274930302A
:1033000004F59E48186008F150084DF0F3FAFF23C9
:1033100085F8603F85F8683F214940464DF0EAFA5C
:10332000204B1D6815B1204893F0A2FE04F59E4085
:103330007030C3F8008053F071FA1C4B1C481860C1
:1033400004F5B04214322B464FF0140C9DB20CFB26
:1033500005010133097C0029F8D1164B1D80164B5D
:10336000D3F80080B8F1000F2AD01448DCE700BF82
:10337000B06D0D0884650D08C4650D080000A040FF
:10338000D87B0E0850940020306E0D08AD27010840
:10339000A06D0D08D4650D08089A0020B4900E08A1
:1033A00084F00E089C9A002010660D08C090002042
:1033B00010B00D08BC9000207890002031660D08F8
:1033C00004F5B0401A6003A9584B0393283058F015
:1033D00041FF04F5B04004F5A045483006F024F85C
:1033E000534BC5F8483804F5B140083006F01CF8D6
:1033F00004F5B5494F4BC5F8883804F5B14009F1DB
:103400001C094430FFF7EAFD484606F00DF84A4B28
:10341000C5F89C3A09F13C0090F004FA474BC5F816
:10342000D83A04F5B8405C3005F0FEFF444BC5F8CF
:103430005C3C04F5B940203005F0F6FF414BC5F87F
:10344000A03C04F5B94085F8DC8C603005F0ECFF59
:103450003D4BC5F8E03C04F5BA401C3005F0E4FFF4
:103460003A4BC5F81C3D05F6585304F5BA401E60AA
:103470005E609E60703005F0D7FF354BC5F8AC8DAF
:1034800004F5BB40C5F8703D383005F0CDFF314B39
:10349000C5F8B83D04F5BB40C5F8F48D7C3005F0A7
:1034A000C3FF2D4BC5F8FC3D04F5BC40443005F08E
:1034B000BBFF2A4BC5F8443E04F5BD4005F0B4FF00
:1034C000274BC5F8803E05F6F86304F5BE401E6044
:1034D0005E601430FFF7DAFD384605F0A5FF214B9A
:1034E000C5F8A03F04F5BF405C3005F09DFF1E4BC2
:1034F000C5F8DC3F04F5C0452846A5F818802C30F7
:10350000FFF7C4FD194BEB6204F5C140012385F8B8
:10351000B530C5F8BC60C5F8C060C5F8C4604830B7
:103520000AF0C6FD204609B0BDE8F083CDCC4C3D85
:10353000B0BE0D0854BF0D085CC30D08ECC30D08E8
:10354000A8C40D0848C50D08E8C50D0880C60D08BB
:10355000BCC80D085CC90D08ECC90D0884CA0D086B
:1035600024CB0D08F8CD0D0894CF0D0854CD0D08CF
:1035700038B5054B1C6823680A461D68034B014695
:103580002046A847002038BD408E0020A02C0020F7
:1035900010B593F0A3F8064C064B18602046FFF7D1
:1035A00091FD2046044A0549BDE81040BBF0B2BD7C
:1035B000A02C0020408E002080F1002075280108FA
:1035C0000120704790F89C308B4286BF283150F81C
:1035D000210000207047000090F89C308B4286BF8D
:1035E000283150F82100002070470000FA20704771
:1035F000014B93F84E037047A04C0020034BD3F8C7
:10360000C001431E58425841704700BFA05C0020D3
:10361000034BD3F8C001831E58425841704700BF86
:10362000A05C0020034BD3F8B00108B18BF0CCBBF9
:1036300001487047A05C00201C6E0D0838B5C36AB5
:10364000374D43F4E052C262026B42F4E05202632F
:10365000426B42F4E0524263D5F8C42D0446E2B115
:1036600043F4F843C362D5F8C40D86F05DFE38B16B
:10367000236B43F480432363636B43F480436363AE
:10368000D5F8C40D86F072FF38B1236B43F40053B4
:103690002363636B43F400536363224B1D6845B19E
:1036A000192128464EF03AFB18B1E36A43F48073BF
:1036B000E3621D4B93F8903D6BB1236B43F4807331
:1036C000236345B1192128464EF060FB18B1636BA6
:1036D00043F480736363154B93F80838013B012B67
:1036E0000BD8D4E90B2343F480032363636B42F4C8
:1036F000800243F48003E2626363E36A43F0804341
:10370000E362236B43F080432363094BD3F8B0316A
:1037100093F8C1301BB9636B43F08043636338BDDA
:10372000A06C0020D0900020A04C0020A07C0020A5
:10373000A05C002013B54FF44470CDE9002119F0CE
:10374000BDFF044628B1DDE9002160F06FFA024BAD
:103750002360204602B010BD74700D080020704731
:10376000704700000320704708207047014B93F812
:1037700050037047A04C0020034B93F90804003815
:1037800018BF0120704700BFA04C0020014B93F9E7
:1037900052037047A04C00207047000070470000A3
:1037A00008B50C4BD3F8C40D70B910230A4AD2F8EF
:1037B000B02143F0400022B192F8CB200AB143F08F
:1037C000C00040F0010008BD86F0AEFD0028ECD03E
:1037D0001823EBE7A06C0020A05C002038B5C5786A
:1037E0000B46352D044628BF3525352200211846C5
:1037F000BEF0FEF92A4604F10C01BDE83840BEF0E7
:10380000ADB900001FB5184C94F8861104F13800CA
:1038100011F0ACFD78B194F8861104F1380011F084
:10382000A7FD40B194F8861104F1380004B0BDE85A
:10383000104011F09FBD002301930293039313F0F6
:10384000C7FC01A913F090FA20B101A82EF05EFE8A
:1038500004B010BD23F0D8F990F8F432B02202FB86
:10386000030090ED3B0AF3E7A04C002008B50D4B98
:10387000D3F8B001A8B1443058F0FAFB034693EDF9
:10388000000ADFED090A9F20B7EE001A2AF0EAFFCE
:10389000DFED067A20EE270ABDEEC00A10EE103AE0
:1038A00018B208BDA05C0020000000000000C84263
:1038B0002DE9F04FDFF8D880344F8DB00446042551
:1038C00008F5005617F8019BB8F9A83309F1FF3A3B
:1038D00043FA0AF3D90742D5207C5AF05DF88346B3
:1038E000207C5AF05DFF00F121039B4505D2207C2E
:1038F0000DB0BDE8F04F59F0A5BABAF1030F2ED8BC
:10390000DFE80AF00234393ED6F8BC0D03689B6844
:10391000984700F194035A69D3F800A0D3F804E063
:10392000D8681969D3F818C008925A6A1B6ACDF88A
:103930002520CDF8293062222123CDE900320690DE
:103940000791207CCDF80CA0192303AAC221CDF841
:1039500010E0CDF814C08DF824905AF087F8013D9E
:1039600015F0FF05AED10DB0BDE8F08FD6F8BC0D57
:103970000368DB68CCE7D6F8BC0D03681B69C7E7B2
:10398000D6F8C43D03F52A73C5E700BF48710D089A
:10399000A04C002013B504460748019109F034F803
:1039A00030B90199204602B0BDE810405BF038B94B
:1039B000042002B010BD00BF64850020014808F05B
:1039C000FFBD00BF6485002037B504460D4606489C
:1039D000019211468EF0EAFC019A2946204603B076
:1039E000BDE830405EF0F0BFD858002010B588B078
:1039F00004465CF013FB0C4BD3F8B00138B90B4A0A
:103A00000621204608B0BDE810405CF0EFBA6946D8
:103A10001E228BF0DDF9064A6B46062120465CF03B
:103A2000E5FA08B010BD00BFA05C0020686E0D086C
:103A30002EBC0D08034A92F8703D013382F8703DA8
:103A40005BF0B0BBA04C002007B50846019119F00F
:103A500087FB38B10448019902F026FD002003B02D
:103A60005DF804FB0420FAE74C8E0020F7B58B8B41
:103A7000CD2B06460C4617461DD1D1ED067AFCEE3D
:103A8000E77ACDED017A9DF80430022B13D10E4D6B
:103A900095F8D51E05F65C6064F0DCF958B195F830
:103AA000D51E05F65C6064F0DDF920B994ED020ADC
:103AB000064802F0D9FC3A462146304603B0BDE83C
:103AC000F0405BF001BC00BFA06C00204C8E0020D9
:103AD000162A10B40C4605D0542A03D05DF8044BC6
:103AE0005BF0BAB80323237001205DF8044B7047E4
:103AF00010B5074B93F9702F40F6CD3440F6CD1337
:103B0000002A08BF1C465BF003FB204310BD00BF2A
:103B1000A06C002010B5044619F0D8FD204610BD59
:103B200010B50C4C94F98031002B0FDBD4F88C01CC
:103B30000368DB6C984758B9D4F88C0103689B6C18
:103B4000984700280CBF0220032010BD0120FCE78D
:103B50000420FAE7A05C002010B44C69012C05D1C8
:103B600001465DF8044B034803F038B85DF8044B98
:103B70005BF032BBA02C00202DE9F341B1F90430F9
:103B8000002B06460C46154635DB4FF00008CDE904
:103B900000281A4FB1F902209FED190AD7F8741DB9
:103BA0004FF47A735FF0F8F90123CDE900539FEDEC
:103BB000140AB4F90020D7F8781D4FF47A73304610
:103BC0005FF0EAF99FED0F0AB4F90420D7F87C1DE5
:103BD00043463046CDE900585FF0DEF9CDE90058A4
:103BE0009FED070AB4F90620D7F8801D4FF47A73C9
:103BF00030465FF0D1F902B0BDE8F081A04C002062
:103C00000000FA4400007A44044B187820B9044BB1
:103C100093F88201C0F38010704700BFB88F002076
:103C2000A05C00200B4B93F84D277AB993F8A5219F
:103C300092060BD193F98021002A09DB93F8813198
:103C400013F0200F14BF0420012070470520704797
:103C500003207047A05C002008B5074B93F99C3304
:103C6000032B03D0BDE808405CF038BA034A0221B8
:103C70005CF0BCF9042008BDA04C0020806E0D084B
:103C8000094BD3F80C24920701D45AF0D9BF03F59D
:103C9000005303F6945393ED000ADFED047AB8EE77
:103CA000C00A20EE270A7047A04C00200AD7233C08
:103CB00010B594B0044603A819F04AF91C4BD3F888
:103CC0008C01036803A95B6D984778B3002103A8B2
:103CD00019F008FA50B3247C93F0F8F9059BDDED58
:103CE000047A0893069B09930023F8EEE77A9FED88
:103CF000117A0B930C930D930E930F9310931193D2
:103D000012934FF6F853ADF84C300023962267EE2D
:103D1000877A8DF84E303323CDE90032079007AA19
:103D200057212046CDED0A7A59F0A0FE14B010BDFF
:103D3000A05C00200AD7233C30B52DED0A8B774CD0
:103D40000546D4F88C01036899B05B6A984700284F
:103D50005BD004F50054D4F8F43D062B00F2C98082
:103D6000DFE803F00404045788AB53006C489FED70
:103D70006D8A0BF0DFFF9FED6C0A01684268836873
:103D80000D930BA80B910C922DF0C2FFF0EE489A08
:103D9000B0EE40CAF0EE60BAB0EE419AB0EE48AA7A
:103DA000F0EE488AF0EE48AAB0EE48BA40F6F85471
:103DB0002D7C93F08BF900231593169301238C220D
:103DC0008DF85E303323CDE900320B90B1EE499A85
:103DD000F1EE688AB1EE488A0BAA552128468DED8E
:103DE0000CCACDED0DBA8DED0E9A8DED0FBACDED5D
:103DF00010AACDED118A8DED12AACDED139A8DED9D
:103E0000148AADF85C4059F031FE19B0BDEC0A8B54
:103E100030BD43480BF08EFF9FED430A01684268B6
:103E200083680D930BA80B910C922DF071FF3C4809
:103E3000F0EE60BAB0EE419AB0EE40CA0BF07EFFF1
:103E40009FED390A2DF064FF3548B0EE40BAF0EE30
:103E500060AAF0EE418A0BF075FF9FED330A2DF05A
:103E600057FF4FF44064B0EE40AAF0EE609AB0EE17
:103E7000418A9DE72A489FED2B9A0BF05FFF9FED4B
:103E80002A0A2DF045FF2648B0EE40BAF0EE60AAAF
:103E9000F0EE418A0BF056FF9FED230A2DF038FF1C
:103EA000F0EE49BAB0EE40AAF0EE609AB0EE418A68
:103EB000B0EE49CA40F607447AE71948DFED198A9F
:103EC0000BF040FF9FED180A2DF022FFF0EE68AADC
:103ED000B0EE40AAF0EE609AB0EE418AB0EE68BA59
:103EE000B0EE689AF0EE68BAB0EE68CA40F63F44A9
:103EF0005EE79FED0C8A0024F0EE489AB0EE48AAE7
:103F0000F0EE488AF0EE48AAB0EE48BAB0EE489A11
:103F1000F0EE48BAB0EE48CA4AE700BFA05C002005
:103F2000588A0020000000000AD7233C2DE9F04108
:103F30002DED068B3B4D95F8813199068CB00446EA
:103F40006AD505F580579FED380AD7F8BC0DDFED2F
:103F5000378A6C302DF0DCFE8DED041A21EE281A24
:103F6000D5F88C618DED020ABDEEC11ACDED030AC4
:103F700011EE103A1DB2336894F810809B6D3046F4
:103F800060EE289A20EEA89A984707EE900AF8EE7D
:103F9000E77A304667EEA87AFDEEE77A17EE903AB8
:103FA0001CB23368DB6D984707EE900AB8EE678A5B
:103FB000D7F8C43DDFED1E7A93ED0FAA336828EEE3
:103FC000288A1B6EB4EEE78AF1EE10FA58BFB0EE05
:103FD000678A30469847BCEEC88A0023089318EEDB
:103FE000103AB7222AEE28AA20EE280AADF82C3083
:103FF0001A23CDE900323E2105AA4046CDED059AAF
:104000008DED069A8DED07AA8DED090AADF82850C1
:10401000ADF82A4059F02AFD0CB0BDEC068BBDE886
:10402000F08100BFA05C00209F0CB3450AD7233C61
:1040300000FF7F472DE9F04F2DED028B1A4B047CDA
:10404000D3F8BC3D8DB0D3F88480D3F88870D3F812
:104050008C60D3F8905093ED258AD3F898B0D3F8BC
:104060009CA0D3F8DC9093F031F800238DF82C302D
:1040700016222523CDE90032029002AA53212046C0
:104080008DED078ACDF820B0CDF824A0CDF828908A
:10409000CDF80C8004970596069559F0E7FC0DB015
:1040A000BDEC028BBDE8F08FA06C002070B58A7A61
:1040B0004B7A43EA0223CA7A43EA02439D2B06461F
:1040C0000C4621D1134D95F8D51E05F65C6063F0C2
:1040D000C1FEC8B195F8D51E05F65C6063F0CEFE52
:1040E000022811D195F8D51E05F65C6063F0BAFE82
:1040F00050B9D4ED057A9FED080A0848F8EEE77A42
:1041000027EE800A02F0B0F921463046BDE8704043
:104110005AF048BFA06C00200AD7233C4C8E0020E8
:10412000054BD3F8B0312BB193F8CA00002808BF73
:104130000220704702207047A05C002008B5034BA6
:10414000D3F88C0103681B68984708BDA05C002069
:10415000024B93F88101C0F340107047A05C00202F
:1041600070B52C4E2DED028B0546D6F88C0191EDE5
:10417000018A036886B05B6A0C46984750B9BDEE69
:10418000C88A18EE103ADB0704D4022006B0BDEC52
:10419000028B70BDD4E904012BF014FC0028F4D08C
:1041A00002A818F0D5FE02AA214628465EF064FE59
:1041B0000028EAD0184902A818F0DEFF03460028BC
:1041C000E3D1DFED160A00900246B0EE600A144813
:1041D00002A90BF0E7FBD8B1D6F88C0103685B6A43
:1041E0009847044608B10020D0E70E480222042177
:1041F00005F0B0FC60B1DFED090A094800942346E0
:10420000B0EE600A224602A90BF0CCFB0028EAD1EE
:104210000420BBE7A05C0020307A002000000000F2
:10422000588A0020A02C002008B591F82030032BDC
:104230001CD1D1ED027A9FED0E7A91ED060A0D4B5D
:10424000F0EEE77AF4EEC77ADFED0B7AD3F88C0163
:10425000F1EE10FA4CBF0121002120EE270A10F0E8
:10426000FDFA002814BF0020042008BD0220FCE74E
:1042700000000034A05C00200000C84210B52DED05
:10428000028BD1ED007AF5EEC07AF1EE10FA82B031
:104290000C4604DA042002B0BDEC028B10BD9FED89
:1042A000197AF4EEC77AF1EE10FAF3D891ED030A19
:1042B0009FED158AF0EEC07AF4EEC87AF1EE10FAAE
:1042C00019D5D4ED037A1148D4ED010A94ED000A12
:1042D000F4EEC87AD4ED027AFDEEE77AF1EE10FA48
:1042E000CDED017A9DF90410ACBF0122002202F04D
:1042F0001DF80020CFE7F7EE000A2AF0AFF90028FA
:10430000C8D0DEE70000B443000000344C8E00202B
:1043100091ED010AB5EEC00AF1EE10FA08B501DC24
:10432000042008BD9FED107A104BD1ED007AD3F830
:104330008C0120EE070A9FED0E7A0368F4EEC77A2F
:10434000F1EE10FA05DDDB6E98470028E8D000207A
:10435000E7E79FED087AF4EEC77AF1EE10FACCBFEA
:104360009B6E5B6EF0E700BF0000C842A05C0020BF
:104370009A9939403333F33F08B5D1ED007A9FED78
:10438000157AF0EEE77AF4EEC77AF1EE10FA1DD561
:10439000D1ED017AF0EEE77AF4EEC77AF1EE10FA99
:1043A00014D50D480222032105F0D4FB80B10A4840
:1043B0000121FDF715FF094890F80439012B03D0BE
:1043C00000F5106031F034F8002000E0022008BD54
:1043D0000420FCE700000034A02C0020A07C00207A
:1043E00010B5D1ED007AFCEEE77A17EE903A9CB268
:1043F000012C02D0022C06D04CB90648214669F0A7
:1044000043FC002010BD044803F0A8F9F9E704209C
:10441000F8E700BFD07B0020A02C00201FB5D1ED15
:10442000017A0B7CFCEEE77ACDED027AD1ED007AD1
:104430000093FCEEE77AD1ED030ACDED037A91ED1E
:10444000020A9DF808309DF80C20014602480EF043
:10445000B7FF05B05DF804FBA02C002010B50A4C96
:1044600094F8A531DB070CD402220521A4F54050B5
:1044700005F070FB28B902221146A4F5405005F062
:1044800069FB002010BD00BFA05C002010B5D1ED7D
:10449000007AFCEEE77A044617EE903A13F0FF0339
:1044A0000FD10F4BD3F88C0103689B6F984708B16D
:1044B000002010BD0B4A204606215BF097FD04202A
:1044C000F7E7012B09D1064BD3F88C010368DB6FAA
:1044D00098470028ECD1044AEDE70220E9E700BF45
:1044E000A05C0020A46E0D08B46E0D089FED0B7A41
:1044F00001F10C03F1EC017AF4EE677AF1EE10FAB7
:104500000AD6F0EEE77AF4EEC77AF1EE10FA03DCA1
:104510009942EFD1012070470020704700007A4493
:1045200030B52DED028B8DB0002305460393049327
:10453000059312F04DFE03A912F016FC58B312F0C9
:1045400047FE00F55A7393E8070006AC84E80700BD
:10455000DDED060A9DED070A2D7CF1EE600AB1EE55
:10456000400ABBF04FF92046B0EE408A2DF0CEFF56
:10457000DFED0B7A089B0B93012228EE278A0C2390
:10458000CDE90032A82109AA28468DED098A8DEDD2
:104590000A0A59F06BFA0DB0BDEC028B30BD00BFBA
:1045A000E02E6542272938B5054613D008D81B29C7
:1045B0000ED0242926D02846BDE838405EF048BEFB
:1045C000282914D0402903D0A1F14203012BF2D8AD
:1045D000012405E0122158F047FC044610B90024DC
:1045E000204638BD297C0C4851F04EFBF8E71621D7
:1045F00058F03AFC04460028F1D0297C064851F0D6
:104600001DFCEDE70C2158F02FFC04460028E6D0F5
:104610002846FFF785FFE3E7107C002038B5194CEA
:1046200094F8A531DB070D460AD4D4F8B03193F8DD
:10463000CB303BB901221146A4F5B470FDF726FC3E
:10464000002038BD94F98031002B4FF0020212DABD
:104650000521A4F5405005F07DFA0028F0D095ED35
:10466000000ADFED097AD4F88C0120EE270A012137
:1046700010F0F4F8E4E70921A4F5405005F06AFAD7
:10468000DEE700BFA05C00200000C84210B5214C4E
:1046900094F8A531DB070ED4D4F8B03193F8CB30C1
:1046A0004BB194F98031002B07DA01220821A4F5DF
:1046B000B470FDF79FFC002010BDD1ED007A9FED96
:1046C000167AF0EEE77AF4EEC77AF1EE10FA0BD52F
:1046D00012480222112105F03DFAA0B9022211462A
:1046E0000E4805F037FAE6E7D4F88C0103681B683A
:1046F00098470428DFD0D4F88C0103681B689847DA
:104700001428E5D1D7E7064840F6C41108F07EFE2C
:10471000D1E700BFA05C002000000034A02C0020E6
:10472000FC88002073B58B8BC12B05460C4644D802
:10473000BB2B0DD8202B63D02ED8113B99B2052965
:1047400018D92146284602B0BDE870405FF072BE1D
:10475000BC3B052BF5D801A151F823F09B4801087B
:10476000A5480108434701084347010833480108A9
:104770003F480108052BE4D801A151F823F000BF00
:10478000814801084347010843470108954801084B
:10479000A747010855480108732B2CD006D8542B85
:1047A00058D0552BCDD1022209216BE0B22BC8D1B4
:1047B00002B0BDE87040FFF7ABBD4AF21146B3420C
:1047C00054D00BD8D12B40D0B3F5967F53D0D02BFB
:1047D000B7D102B0BDE87040FFF702BE4AF2124600
:1047E000B3423ED04AF21346B342AAD102B0BDE86A
:1047F0007040FFF74BBF02B0BDE87040FFF73EBD11
:10480000D1ED007AF5EEC07AF1EE10FA4FDD9FEDB2
:10481000297AF4EEC77AF1EE10FA48D8FCEEE77A7E
:10482000254ACDED017A9DF80430A2F83A3C0020EB
:104830002EE0214602B0BDE87040FFF791BC214652
:1048400002B0BDE87040FFF721BE02B0BDE8704085
:10485000FFF7E4BD2146284602B0BDE87040FFF7EF
:10486000E3BC02B0BDE87040FFF7D8BE02B0BDE8BF
:104870007040FFF7F3BD02B0BDE87040FFF77CBDAC
:10488000022205210D4805F065F90028CFD104204A
:1048900002B070BD02220621F4E70221084806F0AA
:1048A000D7FAF2E70221064806F09CFAEDE702206B
:1048B000EEE700BF00007F43A04C0020A02C0020AA
:1048C0006485002008B591ED007AF6EE007AB4EE2A
:1048D000E77AF1EE10FA06DD044801220521FDF722
:1048E00089FB002008BD0420FCE700BF385B0020E6
:1048F00030B52DED028BCD7893B0272D28BF27251D
:104900000C462722002108A8BDF072F92A4604F1BE
:104910000C0108A8BDF022F9424BD3F88C010368C2
:104920005B6A9847002841D09DF8465068063DD400
:1049300000244FF07E5329060493079406940594AF
:1049400027D504A82CF08EFCEA0701940294039466
:1049500005F006032ED4002B2ED10D9B01930E9B48
:1049600002930F9B039330480AF0CAFD9DED100A95
:10497000044630B340F2ED40B7EE001AFFEE000AF5
:1049800029F070FF2848234601AA04A90AF0C0FDB7
:104990000CE0099B04930A9B05930B9B069304A8C8
:1049A0000C9B07932CF064FC0028CDD113B0BDEC18
:1049B000028B30BD062BD6D001211B480AF03CFDEE
:1049C000F4E7DFED1A0A4FF49E60B7EE001A29F003
:1049D00049FFF6EE000AB0EE408A29F03FFEE8B942
:1049E000B6EE000A124BB4EEC08AF1EE10FAD3F81C
:1049F000C83D08DD38EE400A30EE008A93ED070A24
:104A000028EE000ABEE730EE480AD3ED087A30EE11
:104A1000000AF0EEE77A27EEC00AB3E79FED030A3B
:104A2000B0E700BFA05C0020588A00200000000012
:104A3000A06C00202DE9F0439DB0814608460EA9E8
:104A4000FEF7CCFE844BD3F88C0103685B6A984771
:104A500050B19DF86C30012B09D0DA1F022A06D91B
:104A60007E4801210AF0E8FC1DB0BDE8F083BDF8E6
:104A70006840A20504F0070604F0380704F4E07566
:104A800001D5002DF0D04FF00008CDF81480CDF8FE
:104A90001880CDF81C803EBB9FED716A9DED107AA9
:104AA000DDED117ADDED0F6A27EE067A67EEC67A44
:104AB00066EE866A083B012BCDED056A8DED067A20
:104AC000CDED077A04D8674806AA05A9FDF704FDCD
:104AD0009DF86C30073B022B06D8634889F0CCF870
:104AE000014605A82DF034F9CDF82080CDF82480BA
:104AF000CDF82880F7B9DDED147A129B0893F1EE1A
:104B0000677A139B099308A94846CDED0A7AFFF707
:104B1000EDFC0028A4D09FED520A08A82DF04CF916
:104B20009DF86C30083B012B04D84E4809AA08A90F
:104B3000FDF7D2FCCDF82C80CDF83080CDF8348054
:104B4000EDB99FED476A9DED167ADDED177ADDED43
:104B5000156A9DF86C3027EE067A67EEC67A66EE27
:104B6000866A083B012BCDED0B6A8DED0C7ACDEDFD
:104B70000D7A04D83B480CAA0BA9FDF7ADFC14F440
:104B8000806233D1DFED397A9DED180A9DF86C1003
:104B900020EE270ADFED327A0839012920EE270AB4
:104BA0008CBF0021012114F4006305BFDFED2F7AD3
:104BB000DDED190ADFED2E0A60EEA70A04BFDFED76
:104BC000287A60EEA70AAEB9002F35D1B3FA83F385
:104BD000B2FA82F25B0952090291019300920BAB87
:104BE00008AA05A91D480AF095FD3DE79FED200A9A
:104BF0000021D8E77FB9B3FA83F35B090120009362
:104C0000B2FA82F3CDE901105B0914480BAA08A996
:104C10000BF018F828E7002D7FF422AF0120B3FA3B
:104C200083F3B2FA82F2CDE900105B090B48520916
:104C30000BA90AF0AFFF17E7002D3FF411AFB3FA4D
:104C400083F3B2FA82F2CDE900165B09520905A995
:104C500002480AF0E1FD07E7A05C0020588A002026
:104C60000000C842A02C0020407A0020E02E6542BF
:104C7000000000002DE9F047A2B08046084614A9C4
:104C8000FEF7ACFD7E4BD3F88C0103685B6A984756
:104C9000C0B1BDF88040A30504F0070904F4E07733
:104CA00000D57FB10CAE304618F052F9B9F1000FC3
:104CB00029D1DDE915012AF085FE30B971480121BD
:104CC0000AF0BAFB22B0BDE8F0879DF8841009AA6B
:104CD00040465EF0BBF80028F0D0DDED177A9FED7E
:104CE0006A7A099B009367EE877A10ADFDEEE77A4A
:104CF000DDE9151217EE903A284618F049F995E8C3
:104D00000F0086E80F00002514F0380A0695079575
:104D1000089514D1DDED1A7A189B0693F1EE677AA7
:104D2000199B079306A94046CDED087AFFF7DEFBF5
:104D30000028C3D09FED540A06A82DF03DF8099530
:104D40000A950B959FB99FED506A9DED1C7ADDED9C
:104D50001D7ADDED1B6A27EE067A67EEC67A66EEEF
:104D6000866A8DED0A7ACDED096ACDED0B7A14F4E1
:104D7000806805BFDFED457A9DED1E0A9FED440A70
:104D800020EE270A04BFDFED407A20EE270A14F454
:104D9000006405BFDFED3D7ADDED1F0ADFED3C0A63
:104DA00060EEA70A04BFDFED387A60EEA70AB9F11A
:104DB000000F31D1BAF1000F52D13046CDED050AC6
:104DC0008DED040A18F0F4F803289DED040ADDEDDA
:104DD000050A3FF473AF10A93046CDED050A8DEDFD
:104DE000040A10951195129518F074FA00283FF4F2
:104DF00065AFB4FA84F46409B8FA88F3DDED050A06
:104E00009DED040ACDF804A000945B0906AA10A940
:104E10001C480AF0EFFC55E7BAF1000F0FD101234F
:104E2000B4FA84F4CDE901A36409B8FA88F315480B
:104E300000945B0909AA06A90AF004FF42E7002FC3
:104E40007FF43CAF0123CDE90073B8FA88F2B4FADD
:104E500084F30C485B09520909A90AF09BFE31E76B
:104E6000002F3FF42BAFB4FA84F3B8FA88F2CDF8F0
:104E700000905B095209314602480AF093FD21E790
:104E8000A05C0020588A00200000C842E02E654245
:104E90000000000030B48D7A4B7A43EA0523CD7AC6
:104EA00043EA0543562B04460A461BD008D8522B2A
:104EB00012D0542B13D02046114630BC5EF096BC65
:104EC00003F18073863B23F07F43012BF3D8017CF1
:104ED000064830BC51F07AB830BCFFF709BD30BC91
:104EE000FFF7A8BD30BCFFF7C5BE00BF107C002097
:104EF0002DE9F0412DED028B044690B000F59E4067
:104F00000023012269467030009351F0D5FD08B9A5
:104F10004D4B009304F54056DFED4C8AD6F88C01DA
:104F200003685B69984704F58048002840F0878053
:104F3000D8F8C43DD3EDDE7A93EDD88AFDEEE77A5A
:104F400028EE288A17EE903A1DB204F5385720371C
:104F500001A938460FF01CF818B954F0CFFB3A4BB2
:104F600001933722002102A8BCF042FEA3238DF852
:104F7000083095238DF8093092F0B0F8D8F8BC3D90
:104F8000CDF80B00D6F8B001D3F8DC20D3F8E03030
:104F9000CDF80F104430CDF81320CDF8173057F06E
:104FA00067F80346DFED2A0A93ED000AB7EE001A10
:104FB0009F2029F057FC10EE103AD6F8B001CDF83A
:104FC0001B3003681B69984710EE103A04F59B46A6
:104FD000CDF81F30203618EE103A3046CDF8233089
:104FE00088F04EFE20EE280A384610EE103ACDF832
:104FF0002730D8F86C3DCDF82B30019BCDF82F3001
:105000000EF0E8FF10EE103A3046CDF83330009B3A
:10501000CDF83730ADF83B5088F03EFEBDEEC00A0B
:10502000372210EE103A02A904F57F60ADF83D304A
:1050300053F06CFB10B0BDEC028BBDE8F0819FED2E
:10504000048A002581E700BF2292CA7F0AD7233C49
:105050000000000010B500F58044D4F8BC0D81F0CC
:1050600093FCD4F8C41DD4F8BC0DBDE8104081F009
:10507000F1BC000070B54FF4805104460FF0D4F835
:1050800000284ED004F5804604F57F65D6F8BC0DA7
:1050900003689B689847692100F19402284653F001
:1050A000C1F9D6F8BC0D0368DB6898476A2100F1A6
:1050B0009402284653F0B6F9D6F8BC0D03681B6974
:1050C00098476B2100F19402284653F0ABF9D6F8CB
:1050D000C42D6C21284602F52A7253F0A3F9202131
:1050E00020460FF0A1F8E0B104F54053D3F88C014D
:1050F00003681B69984778B1D6F8C42D28469032CA
:105100006E2153F08FF9D6F8C42D2846BC32BDE885
:1051100070406F2153F086B920460BF0FDFA00284D
:10512000EAD170BD08B512F053F8BDE8084011F09F
:10513000CDBD00007FB50E464FF6FF710446154603
:105140000FF072F8E0B1102200216846BCF050FD6B
:10515000A3238DF8003095238DF8013003238DF8BB
:10516000023091F0BBFF1022CDF80300CDF80710FC
:1051700004F57F6069468DF80B60039553F046FB9C
:1051800004B070BD7FB50E464FF6FF71044615465C
:105190000FF04AF8E0B1102200216846BCF028FD6B
:1051A000A3238DF8003095238DF8013004238DF86A
:1051B000023091F093FF1022CDF80300CDF80710D4
:1051C00004F57F6069468DF80B60039553F01EFB74
:1051D00004B070BD30B52DED048B87B004460D468C
:1051E000182200216846B0EE409AF0EE608AB0EED8
:1051F000418ABCF0FDFCA3238DF8003095238DF887
:10520000013006238DF8023091F068FF1822CDF8A6
:105210000300CDF8071004F57F6069468DF80B5048
:105220008DED039ACDED048A8DED058A53F06EFA6B
:1052300007B0BDEC048B30BD10B54FF480110446AF
:105240000EF0F2FF30B104F598501030BDE8104078
:1052500010F026BA10BD00002DE9F0438FB01446BF
:10526000054689463122002101A8DDE916769846D7
:10527000BCF0BEFCA3238DF8043095238DF80530D7
:1052800008238DF8063091F029FF236804936368A2
:105290000593A36806933B68CDF81D307B68CDF875
:1052A0002130BB68CDF825303368CDF829307368DC
:1052B000CDF80700CDF80B10CDF82D303122B368B2
:1052C0008DF80F9001A905F57F608DF81C80CDF851
:1052D000313053F01BFA0FB0BDE8F08370B52DEDFF
:1052E000068B8CB0144605460E462C22002101A8E0
:1052F000B0EE409AF0EE608AB0EE418AB0EE61AA5C
:10530000F0EE429ABCF074FCA3238DF80430952390
:105310008DF805300B238DF8063091F0DFFEDFEDC0
:105320001A7A94ED007ACDF8070027EE277A29EE55
:10533000279A8DED077A94ED017ACDF80B1027EEC0
:10534000277A68EEA78A8DED087A94ED027A8DF8B7
:105350000F6028EE278A67EE277A2C2201A905F52F
:105360007F608DED049ACDED058A8DED068ACDED39
:10537000097A8DED0AAACDED0B9A53F0C7F90CB05E
:10538000BDEC068B70BD00BFE02E6542A0207047CB
:1053900030B5154B89B004466946D3F8B00104F521
:1053A0007F651E2289F014FD6A461049284653F095
:1053B00049FB04F54053D3F88C0103681B689847F8
:1053C00004F50053014693F80823284653F05EFB8A
:1053D00004F59850103012F061F904F5907020F047
:1053E0007DFC09B030BD00BFA05C00202EBC0D08C4
:1053F0002E4B2F4A70B54360002343618361C36124
:10540000C3632C4B426303644FF080422A4B4364D6
:105410000446826358305FF051FD284E284BA36547
:10542000A82560195FF000FF66513035B5F56A7F39
:10543000F7D1244D04F56A7061F0F8FB002104F205
:10544000BC708CF0B5F8C4F8705804F67800A5F577
:10545000BE658CF083FD9FED1C1ADFED1C0A9FEDED
:105460001C0AC4F8085904F61C1082F07FF89FED5E
:10547000161A9FED180AF0EE410A04F6341082F075
:1054800075F89FED111A9FED130AF0EE410A04F62C
:105490004C1082F06BF820460F494BF02BFA204657
:1054A0000E494BF027FA204670BD00BF103900208E
:1054B0000000C8410AD7233C0000E04098B90D081D
:1054C000ACB90D08688D0020000000009A99993E43
:1054D0000000B44300804A4300AD0D0880AF0D08C2
:1054E00070B54C4D4C49ADF50E7DD02206465AA8FC
:1054F000BCF034FB0FCD0EAC0FC40FCD0FC40FCDDD
:105500000FC495E80F0084E80F0000245AAB181967
:105510000021B7EE000A10344AF0A8FED02CF5D1D5
:105520003E4B0FCB02AC84E80F0001A920464AF0A5
:1055300051FE90B19DF90430DFED396AE06807EE65
:10554000103AB8EEC77AF0EE007AE7EE267AB7EEB8
:10555000000A80EE270A4BF06DFD00240EAB1819EF
:1055600000211034B7EE000A4AF080FE402CF5D13D
:105570002C49902236A8BCF0F1FA0022092136A865
:105580004AF020FF96F9A469D6B9274D0FCD1EAC7D
:105590000FC40FCD0FC40FCD0FC495E80F0084E8E2
:1055A0000F00324604211EA84AF00CFF9FED1F0A8F
:1055B0001F484BF03FFD1F48B7EE000A4BF03AFD85
:1055C0001D4C9FED1E0A0FCC06AD0FC594E80F00D1
:1055D00085E80F00002106A84AF048FE9FED170A53
:1055E000002128464AF042FE04F1100160221EA864
:1055F000BCF0B4FA00241EAB18190021B7EE000A63
:1056000010344AF033FE602CF5D161F09BF80DF5B3
:105610000E7D70BDEC5E0D081C5E0D082C5F0D0844
:10562000CDCCCC3D3C5F0D08CC5F0D0800000000E8
:10563000E8AB0D08F7AB0D080C600D080000344214
:105640002DE9F04790B00DF106011D2061F06EF9D3
:10565000002800F09E809DF80630614A0133DBB2DD
:1056600011210BA88DF8063090F088FD00220DF175
:1056700007010BA84AF0E0FA9DF80630594A1121BB
:1056800005460BA890F07AFD00220DF107010BA84A
:105690004AF0D2FA9DF80630534A112106460BA86B
:1056A00090F06CFD00220DF107010BA84AF0C4FA3E
:1056B0009DF806304D4A03F03F03112107460BA821
:1056C00090F05CFD00220DF107010BA84AF0B4FA3E
:1056D0008046002D5DD0002E5BD0002F59D00028D1
:1056E00057D028464AF0C0FC002852D130464AF034
:1056F000BBFC00284DD138464AF0B6FC002848D102
:1057000040464AF0B1FC002843D1394C94E80F00E0
:105710000DF10C0C10348CE80F0094E80F000DF123
:105720001C0989E80F0002A960464AF053FD98B3AE
:10573000BDF8084002A948464AF04CFD00284AD06E
:10574000BDF8083054BB23B340F2E2449C420FFA48
:1057500084FA0FFA83F927D80DF10A013046ADF823
:105760000A904BF05DFF0DF10A012846ADF80AA042
:105770004BF056FF0DF10A013846ADF80AA04BF088
:105780004FFF00230DF10A014046ADF80A304BF0FF
:1057900061FF10B0BDE8F0870024CBE740F2D6628D
:1057A000002B08BF1346D1E70DF10A013046ADF8D2
:1057B0000AA04BF035FF0DF10A012846ADF80A901A
:1057C0004BF02EFF0DF10A013846ADF80A904BF070
:1057D00027FF0123D6E7002CDBD040F2D663B5E7E4
:1057E00008AC0D0814AC0D0820AC0D082DAC0D084C
:1057F0008C600D0837B500F50D5178220C31044648
:1058000051F03EFB00220C2126484AF0DBFD2046E9
:10581000FFF716FF04F50D500022B7EE000A022133
:1058200020304AF057FE012504F507511E4A009525
:105830000023303145204AF0C9FD1C4A1368D907BE
:1058400009D41B49156004F5065318330B6004F5A1
:1058500088530433CB601649022204F50F5001250A
:105860004AF006FE134A0095002304F57F61FD20EF
:105870004AF0ACFD104B1A68D20705D40F4A1D60E0
:1058800004F59154143414600C4801214AF00CFEC4
:105890004BF036FA0A4A138843F00103138003B031
:1058A00030BD00BF40AC0D08DCEA0E08448E00207D
:1058B00000220020E0600E08488E00201822002000
:1058C000AC9000200F299DBF302303FB0100503016
:1058D00000207047014B93F993037047A04C0020C0
:1058E000024B93F8A50100F001007047A05C002076
:1058F000044BB3F85833DB075ABF0069C0F34010BC
:1059000000207047A04C0020014BD3F8800D704759
:10591000A04C002008B503689B68984730B9044B39
:1059200093F9A401B0FA80F0400908BD0020FCE71B
:10593000A05C002038B50D1E2DDB174C94F88C2D83
:10594000EBB29A4227D3D4F8883D0122595DA4F5E1
:10595000005004F0FFF8F0B15FF030FC032160F07C
:10596000A3FCC0B95FF02AFC0D2160F09DFC90B94A
:1059700094F97833EB40DB075CBF94F99213E9406C
:10598000A4F5005048BF0221BDE8384058BF01F0DF
:105990000101FCF73BBC38BDA04C0020022A10B529
:1059A0000C4605D1BDE810400948352204F0D2B8B4
:1059B000084BD3F88C0103681B689847A04205D1B7
:1059C0005FF0FCFBBDE810405FF082BB10BD00BF84
:1059D000A02C0020A05C002029B1022907D1044B93
:1059E000C3F884117047024B0122C3F88421704729
:1059F000A05C002031B1022907D1044B012283F8B9
:105A000088217047014B83F888117047A05C002003
:105A100010B500F50053DFED186AD3F8782DD3F8F0
:105A2000743DB2F90820B3F908309FED147A07EEFF
:105A3000902AF8EEE77A0446C7EEA60A00F59850D9
:105A40000121103007EE903AF8EEE77A60EE870A0F
:105A500087EEA60A20EE070A11F058FC53F04EFE1E
:105A6000262153F0E3FB04F53D50054ABDE8104004
:105A70000621183056F0C6BF0000C84235FA8E3CE9
:105A800068B70D0800F58042002382F8D83D044A2B
:105A900000F53D5013720621024A183056F0B2BF8D
:105AA0001D90002074B70D0870B500F580450446C0
:105AB00095F8D81D002957D02C4B2D4AD3F88C01CE
:105AC000904204D1D3F8B03193F8CB3023B92046BB
:105AD000BDE87040FFF7D6BF264E95F8D90D04F506
:105AE0004053012293F980313272D0BB002B3BDB53
:105AF00085F8D92D0139C9B204F5005385F8D81DB0
:105B0000D3F8782DD3F8743DB2F90820DFED1A6A86
:105B1000B3F908309FED197A07EE902AF8EEE77A8C
:105B2000B1FA81F1C7EEA60A04F598504909103080
:105B300007EE903AF8EEE77A60EE870A87EEA60A5B
:105B400020EE070A11F0E2FB95F8D83D63B904F5A1
:105B50003D5033720A4ABDE870400621183056F0B5
:105B600051BF002BC6DAB2E770BD00BFA05C0020B9
:105B7000408C00201D90002000007A4535FA8E3CB4
:105B800088B70D086D2900F3E380012901DC60F07E
:105B9000B5B98B1E6B2BFAD80FF2040C5CF823F00E
:105BA000AF5D0108A95D0108AF5D0108AF5D0108A7
:105BB0008F5B0108AF5D01088F5B01088F5B0108F7
:105BC000A95D01088F5B0108AF5D0108A95D0108AF
:105BD000A95D01088F5B0108AF5D0108AF5D010899
:105BE000AF5D01088F5B01088F5B0108A95D0108AB
:105BF000AF5D0108A95D01088F5B0108A95D01087F
:105C0000A95D01088F5B01088F5B01088F5B0108AC
:105C10008F5B01088F5B0108A95D0108AF5D01087A
:105C20008F5B01088F5B01088F5B0108AF5D010886
:105C30008F5B0108A95D01088F5B01088F5B01087C
:105C4000AF5D0108A95D01088F5B01088F5B01084A
:105C50008F5B0108AF5D0108AF5D0108AF5D010812
:105C60008F5B01088F5B0108AF5D01088F5B010846
:105C70008F5B0108AF5D0108AF5D0108AF5D0108F2
:105C80008F5B01088F5B0108AF5D0108AF5D010804
:105C90008F5B01088F5B01088F5B01088F5B010838
:105CA0008F5B01088F5B0108AF5D0108AF5D0108E4
:105CB000AF5D0108AF5D0108AF5D0108AF5D010890
:105CC0008F5B0108A95D0108A95D01088F5B0108D0
:105CD0008F5B01088F5B01088F5B01088F5B0108F8
:105CE0008F5B0108AF5D0108A95D01088F5B0108AA
:105CF0008F5B01088F5B01088F5B01088F5B0108D8
:105D00008F5B01088F5B01088F5B01088F5B0108C7
:105D10008F5B01088F5B01088F5B01088F5B0108B7
:105D20008F5B0108AF5D01088F5B01088F5B010885
:105D30008F5B01088F5B01088F5B01088F5B010897
:105D40008F5B01088F5B01088F5B0108A95D01086B
:105D5000A12921DC96297FF71AAFA1F197030A2B1D
:105D60003FF615AF0FF2040C5CF823F0AF5D0108AD
:105D7000AF5D01088F5B0108AF5D01088F5B010813
:105D80008F5B01088F5B01088F5B0108A95D01082B
:105D9000A95D0108AF5D0108B42908D0DB2903D053
:105DA000B2297FF4F4AE7047002360F079B87047F1
:105DB00070B563298AB0034668DC012973DD881E4B
:105DC000612870D8DFE810F07C008400940099000E
:105DD0006F00B3006F006F000D016F006F008B004C
:105DE00020016F000B013D0144016F006F004C0169
:105DF00053015A016F006B0174016F006F006F0057
:105E00006F006F007D018A016F006F006F008C01D1
:105E10006F006F006F006F008E016F006F006F00EA
:105E20006F006F006F006F006F006F0096016F00D2
:105E30006F00460148014A016F006F006F006F005C
:105E40006F006F006F006F006F006F009001920194
:105E5000940198019A019C016F00BD019E016F00A1
:105E60006F006F006F006F006F006F0003026F0024
:105E70006F006F006F006F006F006F006F006F00AA
:105E80006F006F006F006F006F000F02B22900F00B
:105E900069810EDC9A2900F0B2819F2900F09F8170
:105EA000982900F0A28118460AB0BDE870405FF062
:105EB00063BDB42900F0C780DB29F4D1012433E0AD
:105EC000022AFBD135220E21B04803F043FEF5E74C
:105ED000111E18BF0121AD48FCF798F9EEE7012A21
:105EE00004D0022A14BF00210221F4E71146F2E790
:105EF00006211846FFF752FDE0E7022ADED1A44D45
:105F0000D5F88C010368DB6A984704460028D5D091
:105F1000A5F58053D3F87C3DB3F90830002BCDD1E3
:105F2000A5F54050FFF774FD20460AB070BD022A67
:105F3000C4D1974E974AD6F88C119142BED0D6F86C
:105F4000B02192F8CB20002AB8D006F50054A6F56F
:105F50008056B4F934292AB9D6F87C3DB3F9083013
:105F6000002BABD01C22002103A805ADBBF040FEE6
:105F7000284616F0EDFFB4F93439874C9BB9162347
:105F8000ADF80E30D4F8943D642BB8BF642303A958
:105F900004F5C85006932CF065FE20B153F0AEFB1B
:105FA000272153F043F904F559630FCB85E80F001F
:105FB000D6F87C3D7948B3F90830002BCCBF1023CC
:105FC000152303A9ADF80E302CF04CFE00283FF449
:105FD00075AF53F093FB272153F028F96EE70321A7
:105FE00087E7022A6E4D03D0002385F8903D65E7D0
:105FF0001921A5F596504BF091FE04460028F3D0E8
:10600000012385F8903D8FE7012A0BD0022A11D099
:10601000002A7FF453AF624B83F8BC2353F06EFB2E
:106020002B21D9E75E4B019283F8BC2353F066FB2A
:106030002C21D1E75A4B83F8BC2353F05FFB2D2171
:10604000CAE70F2155E7574811468FF02BF935E77E
:1060500009214EE704214CE705214AE7172148E7CB
:10606000901E41424141504867F00EFE26E7022A49
:106070007FF424AF454801F071FB1FE7012A06D0E9
:10608000022A07D0002A7FF419AF1146EBE7114628
:106090000192E8E74448012167F0F6FDEAE73E4B4C
:1060A000911ED3F8BC3D4A424A4183F8202005E7BF
:1060B000931E59425941384BD3F8BC0D82F062FB14
:1060C000FCE6334B013A93F88211012A8CBF00227F
:1060D000012262F3041183F88211EFE6112108E72F
:1060E000122106E7152104E7002102E7102100E74D
:1060F0000221FEE60121FCE61621FAE60721F8E678
:106100000B21F6E6022A294B0ED1012483F82448FC
:1061100053F0F4FA4A2153F089F85DF047FB244A22
:10612000062156F06FFCFFE6002283F8242853F086
:10613000E5FA4B2153F07AF85DF038FB1D4A062151
:1061400021E0012A09D0022A0AD0002A7FF4B6AE43
:10615000012119480DF054FFB0E601920021F8E743
:106160001146F6E762B3022A7FF4A8AE084BD3F8D3
:106170008C0103689B6F984700287FF49FAE5DF009
:1061800015FB0E4A042156F03DFC97E6A02C00209A
:10619000A05C002064850020A06C0020A085002069
:1061A000A04C002078870020D07B0020A07C00201D
:1061B000A0B70D08B1B70D08C05A0020C3B70D082D
:1061C000184BD3F88C010368DB6F984776E61846C6
:1061D0001146FFF701FC144804F072F86EE6114610
:1061E000FFF708FC6AE61B2183E6022A7FF466AE0D
:1061F0000E48FCF709FE5DF0D9FA0D4A9FE71146FB
:106200005FF0A4FA0B487FF001F9044600283FF440
:1062100055AE044A92F8833143F0020382F8833189
:1062200082E600BFA05C0020E8840020A02C0020B3
:10623000DCB70D08385B002010B50446044887F031
:106240001DFD04F10801BDE8104029F039BB00BF75
:10625000407A002038B504462DED028B114887F0B6
:1062600013FD05462BF096FA0F48B0EE408A0DF06C
:1062700075FF90B1DFED0D7AB4EEE78AF1EE10FA1A
:106280000BDDD5ED000A95ED010AB9F0BBFADFEDA3
:10629000087A20EE270A84ED080ABDEC028B94ED03
:1062A000080A38BD407A0020A02C002000401C467F
:1062B000E02E6542074B93F97903022805D00328A5
:1062C00006D0003818BF0120704781F001007047E8
:1062D00004207047A04C002003688B4216D004298C
:1062E000C0E9001302D007290ED07047084B9FED7C
:1062F000097A03F5A263D3ED007AF8EEE77A67EE48
:10630000877AC0ED087A704700238362704700BF28
:10631000A03C00200AD7233C08B50246FFF7CAFF7D
:10632000BDE8084001461046FFF7D6BF70B52DED19
:10633000048B0446F0EE408AB0EE608A0D461646A5
:1063400090F0C4FE9FED329ADFED329AE06176B3B1
:10635000236843B9304B03F5A263D3ED007AF8EE1E
:10636000E77AC4ED097A68EE898A002DB7EE000A53
:10637000FFEE007AB8BFB0EE670A68EE808AC4ED1F
:10638000058A264BB4EEE98AF1EE10FAD3F8BC0D7B
:1063900030DA81F0D5F920EE090A84ED060ABDEC69
:1063A000048B20460321BDE87040FFF795BF94EDB4
:1063B000090A98EE890A28F0FFF9002D84ED050AF4
:1063C0000BDAB4EEE90AF1EE10FADADBDFED147A5B
:1063D00030EE670A84ED050AD3E7D2D0DFED117AFB
:1063E000B4EEE70AF1EE10FACBD8DFED0D7A30EE1D
:1063F000270AEFE781F0A4F9B4EE480AF1EE10FAAB
:1064000048BFB0EE408A28EE098A84ED068AC6E7C6
:106410000000C84200000034A03C0020A06C002016
:1064200000A00C47000000B410B52DED028B04460F
:10643000B0EE608AF0EE408A90F048FEDFED090A87
:10644000E06168EEA08A68EE200AC4ED098ABDEC1E
:10645000028BC4ED0A0A20460621BDE81040FFF772
:106460003BBF00BF0000C84210B52DED028B0446B3
:10647000B0EE408A90F02AFE94ED090ADFED097A29
:10648000E061A8EE270A28F081F9BDEC028B002319
:1064900084ED090AA36220460621BDE81040FFF7FB
:1064A0001BBF00BF0000C84270B54B68154D0646C3
:1064B0000C4673B98B6863B9C96851B91248FFF7C4
:1064C0002BFF95F8D51E05F65C60BDE8704061F0C5
:1064D00029BE95F8D51E0D4861F0C4FC48B906F1F7
:1064E0000801204616F0F6FE18B107480221FFF712
:1064F000F3FE95F8D51E05482246BDE8704061F0D0
:1065000005BE00BFA06C00204C8E0020FC7A00204D
:1065100008B50721FFF7E0FE80ED0A0A08BD00007C
:1065200008B50368032B23D1D0ED057A9FED127ACD
:10653000F0EEE77AF4EEC77AF1EE10FA1AD50F4BC7
:1065400090ED090A03F5A263D3ED007AF8EEE77A3D
:1065500037EEC00A28F030F9DFED097AB0EEC00A54
:10656000B4EEE70AF1EE10FA94BF0120002008BD56
:106570000120FCE70020FAE700000034A03C0020E6
:106580000000484330B50368023B85B00446082B41
:106590006DD8DFE803F0050D30374B613F616100D6
:1065A000FFF74AFE84ED090A94ED090A05B030BDF3
:1065B00090F08CFDE369DFED310AE061C31A07EE6C
:1065C000903AF8EE677A94ED050A67EEA07AD4ED7A
:1065D000060AF12020EEA71A67EEE00A28F042F939
:1065E000D4ED057A77EEC07AC4ED057AD4ED097A58
:1065F00037EE800AD6E7FFF72DFEDFED217A20EE99
:10660000270ACFE71F4BD3ED767AF8EEE77AC0ED95
:10661000097AC9E71C4DD5F8D00D85F065FC002836
:10662000C2D0D5F8D03D1B6B6362BDE790F04EFD44
:10663000E3699FED127AD4ED0A6AE061C31A07EEAE
:10664000903AF8EE677A67EE877A94ED097AA6EECB
:10665000A77A84ED097AA7E70B4B9FED0C0AD3F8D4
:10666000BC0D6C302BF054FB84ED091A9CE7064BF3
:10667000D3F8C43DD3F84433D6E700BF6F12833A52
:106680000000C842A05C0020A06C00209F0CB34515
:106690000368092B08D8DFE803F0050A050505059E
:1066A000070705100023836290ED0A0A7047044B28
:1066B000D3F8C43DD3F84833F5E7C36AF3E700BF26
:1066C000A06C0020F8B50023214FCB6297F8A531CC
:1066D000204E13F0010F04460D462DD1D7F88C0142
:1066E00003685B6F984738B3D7F88C0103F0ECFB75
:1066F000DFED197A85ED0B0AB0EEC00AB4EEE70AB9
:10670000F1EE10FA03D409213046FFF7E5FD1148F8
:10671000FFF738FF0F4884ED000AFFF7B9FF336831
:1067200084ED010A0A2B0FD8DFE803F00C101010DB
:106730001010100C100C0C003368092BE7D1054821
:106740000021E2E70223A3602046F8BD0123FAE717
:10675000A05C00204C8E002000000034034B01227E
:106760001A6000229A60DA601A6170474C8E00202D
:1067700013B501A904460DF089FB04F5804320B947
:10678000012283F8052F02B010BDDDED017ADFEDA7
:10679000096A03F6F862B8EEE77AD2ED007A67EE9E
:1067A000A67AB4EEE77AF1EE10FA54BF0122002285
:1067B000E7E700BF0000C8422DE9F04F2DED068B42
:1067C00000F500538DB000F59859019393F9CA3341
:1067D000054600F5A04409F1100933B100F5405811
:1067E000D8F8B03193F8CB707FB90021A4F818180D
:1067F000484610F07BFF94F8191848460DB0BDECE0
:10680000068BBDE8F04F10F07BBF90F05FFC05F504
:10681000804B0090DBF8C40D9FED958A90EDDBAACC
:1068200083F082FD09AE002800F0CD80DBF8C43D86
:1068300003F55C7393E8070086E8070030468DEDAA
:106840000B8A2BF063FEB0EE409A28460DF086FCD2
:1068500005F59B4A0AF1200A002800F0B78050464F
:1068600087F012FA07C886E8070030468DED0B8ADC
:106870002BF04CFEF0EE409AD8F88C0103681B68B0
:106880009847122840F0AB80002384F81838D8F8D5
:106890008C0103685B69984730B1019BD3F87C3D5C
:1068A000B3F90830002B0DDC98F98031002B09DAA0
:1068B000009BC4F81C38504687F0E2F904F50263E7
:1068C00083ED000A94F818385BB1009BD4F81C08DB
:1068D000181A41F28833984240F28F80002384F8DE
:1068E0001838DBF8BC0D9FED630A6C302BF010FA02
:1068F0008DED090ACDED0A0A8DED0B1A96E8070019
:1069000006AB03AE9FED5C0A83E8070086E807004C
:1069100030462BF0FDF92846B0EE408AF0EE608A52
:106920008DED060ACDED070A8DED081A0DF016FC67
:10693000002874D0DFED517AF4EEE79AF1EE10FA08
:1069400094BF01250025DBF8C40D83F0EDFC30B1C8
:10695000DFED4A7AB4EEE79AF1EE10FA09D9002D8C
:1069600064D1D8F88C0103681B689847022864D06A
:106970000027DBF8C40D83F0F9FD0546002873D02D
:10698000B5EEC0AAF1EE10FA6DD5DFED3D7AB4EEAA
:10699000E7AAF1EE10FAACBF01260026504687F0B8
:1069A0007BF95EB9DFED377AB0EEC00AB4EEE70AE4
:1069B000F1EE10FA5AD8002D08BF002794F81818E5
:1069C00084F8197814E7B0EE489A3EE728460DF0AF
:1069D00095FB00287FF443AFDFED259A4CE7D8F80C
:1069E000B03193F8CB30002B3FF451AF98F98031A0
:1069F000002BBFF64CAF012347E7504687F040F924
:106A000004F50263D3ED007A30EE670ADFED1E7AFB
:106A1000B4EEE70AF1EE10FA3FF760AF61E72846FF
:106A20000DF06CFB0546002884D18CE7DBF8C40D23
:106A300083F07AFC002894D19BE7B0EE680AB8F0A6
:106A40008FFCF0EE408AB0EE480AB8F089FCDFED2A
:106A50000F7A20EE280AB4EEE70AF1EE10FACCBF66
:106A60000127002785E700252E4697E73746A5E74B
:106A7000000000009F0CB345D30237390000FA42F2
:106A80000000C8C2000070420000484255CF7D3F60
:106A900038B504460DF062FB04F59855103548B939
:106AA00020460DF02BFB014620B92846BDE83840B2
:106AB00010F068B804F54054D4F88C0103689B6C5E
:106AC000984720B9D4F88C010368DB6C98470146DD
:106AD000EBE7000030B5044689B0684604F59855E8
:106AE00016F036FA103504A816F032FA6946284630
:106AF00010F002F998B104A9284610F04DF970B1D0
:106B0000059B019323680022DB6C69462046984769
:106B100028B104F52D5001213C308BF015F809B057
:106B200030BD000000F5805292F88C25D2070BD4BE
:106B300000F54052D2F8B02192F8CB1009B1FFF71E
:106B4000C9BF03689B6C18477047000030B587B019
:106B5000044602A8019116F0FBF904F5985002A929
:106B6000103010F0C9F8019A18B90025284607B06E
:106B700030BD236802A9DB6C2046984705460028F3
:106B8000F3D004F52D5001213C308AF0DDFFEDE714
:106B9000F0B5044685B004F59856684610360F46A1
:106BA000154616F0D5F96946304610F0F5F810B9DB
:106BB000002005B0F0BD394630460FF055FF0028E3
:106BC000F6D0002DF5D004F58054284694F88C3585
:106BD00043F0020384F88C35EBE700002DE9F04F19
:106BE0002DED0A8BBDB0044624220D4618A80021C5
:106BF000BAF0FEFF2422002121A8BAF0F9FF2422D6
:106C000000212AA8BAF0F4FF04F5405624220021FE
:106C100033A8BAF0EDFF0023CDE90D330F9396F8BA
:106C2000813113F0080839D104F5005943F0080305
:106C300099F8702D079286F8813117F013FB90F9BF
:106C4000213003B390F84033EBB104F28457384657
:106C500017F018FAC34694F8A6355FFA8BF18B4209
:106C60001FD9384617F0ECF90BF1010B82460028CA
:106C7000F1D1C94A0221284659F0B8F996F8813174
:106C80006AF3C30308E0C54A0221284659F0AEF969
:106C900096F881316FF3C30386F881314FF0010814
:106CA0003EE304F53A531833012118460BEE903AAF
:106CB000FAF788FF824608B9B94ADBE720460CF0AC
:106CC00069FFD9F87C3DB3F908A0BAF1000F01D0F3
:106CD000B44AD9E796F98031002B01DBB24AC9E703
:106CE000204601F0BBFE04F547531C3318465246BC
:106CF0000CA90CEE103A13F033FA002814BF02234B
:106D000001230393F123CDE9133A8F210A23CDE91F
:106D1000003113AA287CADF854A003234D2156F06E
:106D2000A5FEA24B9FEDA28A01225A720621A14A1A
:106D3000284659F05BF9039B022B0CBF9E4A9F4AE1
:106D4000062128464FF0000A59F050F989F886A329
:106D50005146384617F0E0F894F8A6355FFA8AF104
:106D60008B420CD913AA38468DED138A8DED148A07
:106D70008DED158A0AF1010A16F050FFECE738464E
:106D800017F080F94FF0000A4FF07C0B94F8A6251D
:106D90005FFA8AF94A4519D94946384616F030FE55
:106DA000C0B20BFB00403CAA0C2300F2146003FBB2
:106DB000092C07C8ACF1900C8CE807003CAA02EB48
:106DC000890909ED2F8A0AF1010ADFE741F28831CA
:106DD0000AA824F02BF8D6F8B0019FED759A036845
:106DE0009FED77AA9B6ADFED77AA9847D6F8B001A6
:106DF000012187F0F1FE744B1B680293D86A036887
:106E000001211B68984790F061F9059090F05EF9B8
:106E1000F0EE499A0690002604F50059079A99F871
:106E2000703D934240F0D88094F8C618384617F069
:106E300007F9002800F0D08004F5405BDBF8B031A2
:106E400093F8CB300493002B00F0C68041F28831D8
:106E50000BA823F0EBFF90F039F9059BC01A13281B
:106E600040F2D98090F032F9059020460CF092FE65
:106E700060F004F882465FF097FFD9F87C3DDBF8BC
:106E8000B001B3F9083000EE103AB8EEC00A20EEB7
:106E90000A0A89F013FB50465FF08EFF384617F060
:106EA000F1F81CEE100A13F077FBD9F87C3DDFED0A
:106EB000400AB3F9083000EE103AB8EEC00AA2203A
:106EC00020EE0A0AB7EE001A27F0CCFCB4EEE90A6D
:106ED000F1EE10FA1CEE100A4FF000020CA958BF98
:106EE000F0EE409AF0EE408A13F03AF908B9002328
:106EF0000C939DED0C8ADFED357AB4EE498AF1EE04
:106F000010FAF4EEE78A48BFB0EE498AF1EE10FAC3
:106F100080F28F809FED2E9ADFED2E8A4FF0000ACF
:106F200094F8A6355FFA8AFB5B4540F296814FF0F4
:106F30000C0918AB09FB0BF903EB0900B0EE490A89
:106F40002AF0E6FE59463846CDED110A8DED121AAB
:106F50008DED100A16F054FD7C23C0B203FB0040F7
:106F6000B0EE680A00F214602AF0D2FE3CAB13A91E
:106F700010A899448DED130ACDED140A8DED151A64
:106F80002AF09AFE0AF1010A09ED240A49ED230AC2
:106F900009ED221AC4E700BFD9B90D08C8B90D0818
:106FA0004BD00D08E7B90D08F9B90D081D90002068
:106FB0000000000004BA0D0819BA0D08AB620D08F4
:106FC0006F12833A0000C842408E00200000003457
:106FD000A4707D3F0AD7233C04F54059D9F8B0018D
:106FE00003689B6A9847D9F8B001002187F0F4FD47
:106FF000029BD86A036800211B689847002E40F066
:107000005F812846C94A052158F0F0FF31463846CD
:1070100016F082FF70E1029B986A036805215B68A5
:1070200098470BA823F00EFFB0EE498AB0EE489ABD
:10703000F2E64FF000094FF00C0B04F5B86A94F833
:10704000A6255FFA89F39A4222D919463846089351
:1070500016F0D6FC089B0BFB03F13CAB5A18A2F1CF
:107060006C034FF07C0CC0B2CDE908320CFB00A0E1
:1070700018AB194454302AF035FE089B099A09F1DF
:10708000010902ED1B0AC3ED010A83ED021AD6E7DE
:10709000039B012B4FF0000A46D19FEDA5BA9FED4F
:1070A000A59A4FF00C0B94F8A6355FFA8AF6B34216
:1070B00040F286800BFB06F63CAB03EB0609A9F118
:1070C0004803089321ABB0EE680A98192AF030FE05
:1070D000089B09ED120AC3ED010A83ED021A33ABD6
:1070E000B0EE4B0A98192AF013FE2AAB98198DEDD1
:1070F000100AB0EE490ACDED110A8DED121A2AF0F0
:1071000007FE13A910A88DED130ACDED140A8DED1D
:10711000151A2AF0E7FD0AF1010A09ED090A49EDFD
:10712000080A09ED071ABEE79FED819A9FED81BA23
:10713000F0EE088A94F8A6355FFA8AF94B4564D9CF
:107140009DED0C0AB4EEE80AF1EE10FA35DB0C23E3
:1071500003FB09F93CAB03EB090621AB03EB090088
:107160002AF0E6FD33AB46ED110A06ED101A06EDE6
:10717000120A03EB0900B0EE490A2AF0C9FD2AAB56
:1071800003EB09008DED100AB0EE4B0ACDED110AAC
:107190008DED121A2AF0BCFD13A910A88DED130A6B
:1071A000CDED140A8DED151A2AF09CFD06ED090AA5
:1071B00046ED080A06ED071A049E0AF1010AB9E72E
:1071C0004FF000094FF00C0A94F8A6355FFA89F6E3
:1071D000B34241D933AB0AFB06302BF097F91BEED3
:1071E000900AF0EE408A7EF00DF907EE900AB8EEB4
:1071F000677A3CABC8EE877A03EB860609F1010992
:1072000067EEAA7A46ED2F7ADEE74FF0000A4FF0DC
:107210000C0B94F8A6355FFA8AF94B451DD933ABB0
:107220000BFB09302BF072F9C8EE297A0AF1010A3A
:107230001BEE900A67EE808A7EF0E4F807EE900A73
:10724000B8EE677A3CABC8EE877A03EB890967EE44
:10725000AA7A49ED2F7ADCE7049E8FF037FF069B70
:10726000C01AB0F5FA7F27D98FF030FF04F500532C
:10727000DDED0D7AD3F87C3D0C9A1B891392FCEE60
:10728000E77A339A1492ADF85C30349A159217EE7F
:10729000903A359A1692ADF85E30F0221423CDE97B
:1072A0000032B121069013AA287C56F0DFFB78F05B
:1072B000A1F8297C77F090FF0BA823F0C3FDB5E679
:1072C0000399384616F028FE00264FF00C0A94F871
:1072D000A635F1B28B4207D933AB0AFB01323846EF
:1072E00016F09CFC0136F2E7384616F0A9FC124A6B
:1072F0000621284658F07AFE104B002520465D7284
:1073000001F09EFB04F50E50063049F0C9FB99F8D8
:10731000813165F3C30389F881310AA823F092FD16
:1073200040463DB0BDEC0A8BBDE8F08F653E0F08CE
:10733000A4707D3F0AD7233C21BA0D081D90002080
:10734000F0B5544FD7F8383DDA0785B0044600F160
:107350009F8000F54055D5F8B03193F8C120002A40
:1073600040F0968093F8CB30002B00F08E8095F99A
:107370008031002BC0F2898000F5A04393F82438B7
:10738000002B40F0858000F580469FED430AD6F83B
:10739000BC0D6C302AF0BCFCCDED020A60EEA00AF8
:1073A000DFED3E7A8DED010AE0EE000A8DED031A65
:1073B000F4EEE70AF1EE10FA67DCD6F8BC3D9FED7B
:1073C000387AD3ED377AF4EEC77AF1EE10FA04D5B5
:1073D000D5F8B0311B7A002B57D0B5EE007AF4EE19
:1073E000C77AF1EE10FA50D404F59B40203086F0B5
:1073F00053FCDFED2C7AB4EEE70AF1EE10FA44D834
:10740000D6F8BC3D9FED287AD3ED367A67EE877AC1
:10741000B3EE0E7AF4EEC77AF1EE10FA35DA234ABB
:10742000B4F9A410138801339BB2138019B9B4F8CE
:10743000A210A4F8A410B4F8A410994228D80026E9
:10744000168052F05BF90122192151F00FFFD5F897
:10745000B00103685B699847431C04F53D50144A2A
:107460003146183055F0CEFAD5F8B031012283F804
:10747000C120D7F8383D5B070AD504F588500430A1
:1074800005B0BDE8F0406AF093BD084B00221A80B9
:1074900005B0F0BDA04C00209F0CB3454054094AF4
:1074A0006666663F000000B4E02E6542868E0020CE
:1074B00038BA0D08F0B52DED028B4B4BD3F8383DA3
:1074C0009B0785B004461FD400F58046DFED478A50
:1074D000D6F8BC0D03681B699847D0ED017AF4EE2D
:1074E000E87AF1EE10FA0FDB04F5405304F5B045ED
:1074F000D3F8B02192F8C110283549B1002303A96F
:107500002846039354F0B6FD05B0BDEC028BF0BDE8
:1075100092F8CB20002AF1D093F98031002BEDDBDB
:1075200004F5A04797F82438002BE7D1D6F8BC0D16
:1075300003681B699847D0F8A430D6F8BC0D0393B4
:1075400003681B69984704F58C7200F1A401284672
:1075500054F08EFEDDED037AB0EEC08AF0EEE77AED
:10756000F4EEC87AF1EE10FA03D503A9284654F0D8
:1075700081FDD6F8BC0D03681B699847D0ED040A5D
:10758000F4EEE80AF1EE10FABEDBF6EE087A60EEF1
:10759000A77AF4EEC87AF1EE10FA1DD58FF096FDB9
:1075A000D7F8343842F21072C31A9342ACD9DFEDE7
:1075B000107AC7F8340868EE277A04F53D5417EEC0
:1075C000900AF8F7A9FF1834CDE90001094A002113
:1075D000204655F017FA97E79DED030A27F03EF88D
:1075E0000028DBD190E700BFA04C00200000003451
:1075F0000000C84254BA0D0810B5044600F59E407C
:10760000303066F053FB04F59E400121BDE8104088
:1076100050306EF0AFBE0000F8B500F5804504466E
:1076200095F9303F5BB300F5405695F8442F96F836
:107630008031DB43C3F3C01363F3C30200F59E47FD
:1076400000F59B4085F8442F203086F025FBDFEDC8
:107650003F7A303720EE670A384666F0A7FB04F51C
:10766000A04393F8243853B9384666F04BFBD6F85C
:10767000B03193F8CB301BB9354B00221A80F8BDDE
:1076800095F8443FDB07FAD4D6F88C0103689B6B6E
:1076900098470028F0D096F98031002BECDB2C4E77
:1076A00033884BB9B5F9363F33B1642213FB02F38B
:1076B000D5F8942D9A42E2DB384666F093FBD5F874
:1076C000BC3D9FED247AD3ED367A67EE877AB3EE30
:1076D0000E7AF4EEC77AF1EE10FA05D83388002B53
:1076E000CDD0013B3380CAE7B4F9A4301BB9B4F85C
:1076F000A230A4F8A4303388B4F8A420B4F9A400CC
:10770000154993423CBF013333803388D5F86C2D43
:10771000012B01D10A60B2E709689142ACDD18B9CA
:10772000B4F8A220A4F8A420B4F8A4209A42A6D8C1
:107730000023338051F0E2FF02220C2151F096FD2C
:107740002046BDE8F840FFF757BF00BF0AD7233CEB
:10775000848E0020E02E6542808E002008B500F562
:10776000804292F9303F6BB300F5405393F980317A
:10777000002B0EDA00F53D50134A0621183055F063
:1077800041F951F0BBFF0322BDE808400F2151F041
:107790006DBDB2F9363F8BB1D2F8942D642113FB45
:1077A00001F39A420ADA00F53D50084A01211830E7
:1077B00055F028F951F0A2FF0222E5E7BDE80840A4
:1077C000FFF71ABF08BD00BF6CBA0D087EBA0D08DE
:1077D00070B52DED028B00F540555D4ED5F8B031FA
:1077E00093F8CB308CB0044643B195F98031002B2F
:1077F00004DB00F5005393F9A2332BB90023338047
:107800000CB0BDEC028B70BD00F5A04393F824389A
:10781000002BF3D101F08AFB00287FD1D5F88C0131
:1078200003689B6B98470028E8D004F59A407030B5
:1078300054F076FC2AF06AFEF0EE087AB4EEE70A1D
:10784000F1EE10FAF0EE408AD8DA04F5805303F531
:10785000AB6203F25C53D3ED007A92ED000A20EEA6
:10786000270AB7F067FFDFED3B7A20EE270AB2EE7A
:107870000E7AB4EEC70AF1EE10FABFD904F58043D0
:10788000D3F8BC3D93ED368A28EE278AF3EE0E7AC4
:10789000B4EEE78AF1EE10FAB0D904F5985000235F
:1078A00009A9103009930A930B930FF081FA00286D
:1078B0003DD13388B4F9A42001339BB23380002A30
:1078C00040D0B4F8A420B3EB420F99DB51F016FF7F
:1078D00001220C2151F0CAFC1F4B002218EE900A25
:1078E000CDE90623F8F718FE1C4BCDE90401002270
:1078F00018EE100ACDE90223F8F70EFE04F53D5408
:107900001834CDE90001164A2046002155F07AF8D6
:1079100001220C211348FAF76DFB71E7D5F88C01B1
:107920000368DB6C984700287FF478AF66E709A806
:107930002AF0ECFDF2EE047AB4EEE70AF1EE10FA6A
:10794000B7DB5BE7B4F8A220A4F8A420B9E700BF36
:107950007C8E0020E02E65420000084000003E4082
:1079600094BA0D08385B0020F0B52DED028B8BB07A
:10797000002307930893099305AB0446019300F590
:10798000985007AB009302AA04AB03A910300FF084
:1079900027F904F50056054686F84C0F28B900254E
:1079A00028460BB0BDEC028BF0BD8FF087FBD6F8FC
:1079B000503F9FED327AC31A07EE903AF8EE677A9D
:1079C000074667EE877A04F53C5006AA02A92830DC
:1079D000CDED067A54F04CFC04F53C5006AA03A900
:1079E00034308DED020A54F043FC06AA04A904F5D4
:1079F0003D508DED030A54F03BFC96EDE98AC6F844
:107A0000507FB5EEC08AF1EE10FAC8D9DDED080A54
:107A10009DED070AB7F02AFDDDED090AB7F026FD56
:107A2000D6F8D02EDDED037AB4EEC08AF1EE10FA6E
:107A300094BF012300231AB196F8D42ED20712D492
:107A400038EE087AB4EEE77AF1EE10FA0BD802338A
:107A5000DBB2DDED027AB4EEE78AF1EE10FA09D876
:107A6000002B9CD09CE7B4EEE78AF1EE10FAF0D838
:107A70000133EDE7012B93D891E700BFBD37863581
:107A800070B500F54055044695F8A53143F0040360
:107A900085F8A53151F032FE0122112151F0E6FBAB
:107AA000D5F8B03193F8CB30002B43D0D5F88C010A
:107AB00003681B68984709280AD1204608F02CFE65
:107AC00030B104F5BB407C30BDE8704008F00CBE1E
:107AD000194BD3F88C0103681B69984704F50053D0
:107AE00040B993F9A133032B24D10621204608F095
:107AF000FFFD0DE093F9A1130229F6D195F8A53108
:107B0000DB07F2D40622204602F024F80028ECD04D
:107B10000A4BD5F88C0101225A7303681B6C9847F5
:107B2000034604F53D50064ABDE870400221183076
:107B300054F068BF70BD00BFA05C00201D90002005
:107B4000C8BA0D0808B500F5405292F8A53159079A
:107B500017D56FF3820382F8A5310A4B5A7B42B1E5
:107B6000002200F53D505A730221074A183054F0A4
:107B700049FF51F0C3FDBDE808400022112151F03A
:107B800075BB08BD1D900020ECBA0D08F0B5054688
:107B900085B005F598576846103715F0D9F969464C
:107BA00038460FF0F9F880B105F50053D3EDE97AC6
:107BB000374CF5EEC07AF1EE10FA08D8354A0023BA
:107BC00028462380D373FFF7BDFF05B0F0BD2846DC
:107BD000FFF7CAFE064628460CF090FA10B9284670
:107BE0000CF066FAA378002E18BF00200343DBB226
:107BF000A370002BE9D06378A8BB83BB2378013343
:107C0000DBB2082B237003D14EB338460FF054F883
:107C10002378092B02D138460FF046F82378092B38
:107C20001DD94FF48573238051F068FD0222102185
:107C300051F01CFB8FF04AFA6368C01A47F23053C8
:107C4000984209D905F53D50134A0221183054F0E5
:107C5000D9FE8FF03BFA60602846FFF711FF0D4B0D
:107C60006278DA73B1E72678002EF8D0013EF6B2DA
:107C70002670002BF3D0002EF1D1667051F03EFD3E
:107C80003246102151F0F2FA2846FFF75BFFE6E793
:107C9000888E00201D90002004BB0D0800F5405385
:107CA00093F8A5315B0701D5FFF7EABE70470000E6
:107CB00073B5044600F5985001A9103004F500553D
:107CC0000EF0D8FDD5F8143F834206460CD004F5DB
:107CD0008043D3F8BC0D81F0F7F8C5F8146F51F06C
:107CE0000DFD3E2151F0A2FA04F5805695F9181FBA
:107CF00096F9202696F8203691421BD0FF2B19D0FA
:107D000004F58043D3F8BC0D81F0DEF896F82036F8
:107D100085F8183F51F0F2FC95F8182F182151F012
:107D2000A5FA04F53D5095F9183F034A042118308F
:107D300054F068FE02B070BD14BB0D082DE9F0438D
:107D40008FB005468FF0C2F9002305930693079381
:107D5000089309930A930B930C930D9305F5985888
:107D600004AB019308F1100803AB009306460BAB7C
:107D700008AA05A940460EF013FFDFED487A9DEDF5
:107D8000077AB4EEE77AF1EE10FA074632DB9DEDA2
:107D90000A7AB4EEE77AF1EE10FAACBF01240024BF
:107DA00005F50059404699F84C3F002B08BF0027C5
:107DB0000EF008FF8046FFB9444699F9D43C012BE8
:107DC0002BD174B105F54053D3F8B02192F8CB40D4
:107DD0003CB1D3F88C0103685B69984780F00100DF
:107DE000C4B299F81C3FCBBBCCB9C9F8206F0FB017
:107DF000BDE8F0830024D3E7002CDDD005F53C502E
:107E0000343054F035F990ED007AF7EE007AB4EEA4
:107E1000E77AF1EE10FAD0DCCEE70024E1E7D9F8FA
:107E2000200F301AB0F57A7FE1D9C9F8243F012438
:107E300005F5804389F81C4FD3F8C43D83F80C4402
:107E400051F05CFC22461D2151F010FA144A05F550
:107E50003D500221183054F0D5FDC8E714B1C9F8DF
:107E6000246FC4E7D9F8240F43F69823361A9E42AC
:107E7000BDD905F58043C9F8204F89F81C4FD3F8C8
:107E8000C43D83F80C44C9F8244F51F037FC224616
:107E90001D2151F0EBF9034AD9E700BF000000347F
:107EA0002CBB0D0846BB0D080B4B10B50122044638
:107EB0005A728FF00BF904F5A042D2F81038C31AA9
:107EC000142B08D9C2F8100804F595501C30BDE8F1
:107ED000104045F01FB810BD1D9000202DE9F7435C
:107EE000044604F5405600F50E5000231C300DF1F9
:107EF00007018DF8073049F041FBD6F8B00190F941
:107F0000C030026883B3083BDBB2012B95692BD9E3
:107F10003221A84704F1100012F0DAFC204B04F5DE
:107F20003D581F684FF0000908F11808F86A036807
:107F3000DB69984701281ED18FF0C8F841F28733DA
:107F4000A0EB09029A42054605D9164A0621404689
:107F500054F058FDA9462046FFF7A6FFB86A03680B
:107F600003215B689847E1E704F500539269B3F891
:107F7000B0139047CEE70121D6F8B00186F02CFE71
:107F8000D6F8B0010368DB6A98475EF075FBF86AC3
:107F900003681B68012103B0BDE8F043184700BF28
:107FA000408E002064BB0D0870B5044600F53D50BE
:107FB0002DED028B184A194E9FED198A06211830B3
:107FC00054F020FD2046FFF789FF2046FFF76CFFA5
:107FD00020460BF0DFFD3368986A036803215B6875
:107FE00098475EF04BFF05465EF0DEFE04F5005359
:107FF000D3F87C3DB3F9083000EE103A04F5405355
:10800000B8EEC00AD3F8B00120EE080A88F056FA9C
:1080100028465EF0D1FED8E788BB0D08408E0020D0
:108020006F12833A2DE9F047044600F53D502DEDDF
:10803000028B2A4ADFF8AC900621183054F0E2FC9B
:108040002046FFF74BFF5EF019FF04F5405605464A
:108050005EF0AAFEB7EE000AD6F8B00188F02EFA5C
:1080600028465EF0A9FE8FF031F841F2873A0746C4
:108070008FF02CF8C01B5045D9F8008017D99FED20
:10808000188A28465EF090FEB0EE480AD6F8B00195
:1080900088F014FA28465EF08FFE2046FFF704FFB2
:1080A000D8F82800036803215B689847E9E7284669
:1080B0005EF07AFEB7EE000AD6F8B00188F0FEF95D
:1080C00028465EF079FE2046FFF7EEFED8F828003D
:1080D000036803215B689847CAE700BFB8BB0D0877
:1080E00000000000408E0020F7B500F54053044624
:1080F000D3F8B03193F9C030032B2BD0364E652521
:1081000000F5A047013D15F0FF050CD0D7F80C385D
:108110004BB93368986A036814215B689847204616
:108120000BF038FDEEE704F53A5001211830F9F76D
:1081300049FD04F5005378B993F99C3353B1092BE9
:1081400008D08DF8070004F50E500DF107011C3022
:1081500049F014FA03B0F0BD93F99C23032A34D8F4
:10816000DFE802F002252D30D3F87C3DB3F908207A
:1081700040F2B5339A422ADD04F50E5001250DF187
:1081800007011C308DF8075049F0F8F904F53D500F
:10819000124A0221183054F035FC114B5D720E4B1F
:1081A0001C68A06A036805215B689847F9E7D3F863
:1081B0007C3DB3F9082040F2B5339A4207DD2046F2
:1081C000FFF7F2FE2046FFF72DFF092AC2D0002359
:1081D0008DF80730B7E700BF408E0020DCBB0D08EC
:1081E0001D90002000F53D500B46024A0421183036
:1081F00054F008BCFCBB0D0810B5044651F07EFAE3
:108200000022052151F032F804F53D50034ABDE843
:1082100010400421183054F0F5BB00BF08BC0D0815
:1082200013B50B464AB100F53D5000920421054AB2
:10823000183054F0E7FB02B010BD02B0BDE81040AA
:10824000FFF7D0BF20BC0D0808B500F53D50064A29
:108250000421183054F0D6FB51F050FABDE8084024
:108260000022082151F002B834BC0D0838B504468C
:108270000D468EF02BFF04F540533DB9D3F89C21F9
:10828000C3F8A0010AB9C3F89C0138BDD3F8A021F6
:10829000801A642884BF0022C3E96722F5E7000042
:1082A00037B5044600F59B40203085F0DBFC04F533
:1082B0004052C0F3803592F88231C3F34001A942A5
:1082C0001DD065F3410304F53D5482F88231183422
:1082D0006DB151F013FA02220B2150F0C7FF094A89
:1082E0000221204603B0BDE8304054F08BBB51F072
:1082F00005FA2A460B2150F0B9FF034AF0E703B014
:1083000030BD00BF4CBC0D0868BC0D0838B50A462E
:108310000C460621054601F01DFC28B1054A1378DC
:1083200043F00803137038BD21462846BDE83840A5
:1083300008F0DEB93C90002038B50A460D461521FC
:10834000044601F007FC28B1094A137843F00803FA
:10835000137038BD04F53D5004211830054A54F01F
:1083600051FB29462046BDE8384008F0C1B900BF9E
:108370003C90002078BC0D0838B50A460D46152102
:10838000044601F0E7FB28B1094A137843F00803DB
:10839000137038BD04F53D5004211830054A54F0DF
:1083A00031FB29462046BDE83840FFF7AFBF00BF8C
:1083B0003C900020A0BC0D0838B50A460D461B2194
:1083C000044601F0C7FB28B1094A137843F00803BB
:1083D000137038BD04F53D5004211830054A54F09F
:1083E00011FB29462046BDE83840FFF78FBF00BF8C
:1083F0003C900020B6BC0D0838B50A460D46112148
:10840000044601F0A7FB28B1094A137843F008039A
:10841000137038BD04F53D5004211830054A54F05E
:10842000F1FA29462046BDE8384008F061B900BF9E
:108430003C900020C8BC0D0810B500F5405494F8DD
:1084400082319A0623D4D4F88C0103681B689847BC
:10845000032808D005D802280ED194F88001C0095D
:1084600014E01B28F9D194F8800100F0A000A0F1DD
:1084700080035842584109E0B4F8800120F4FE40DE
:1084800020F07F0080B2003818BF012010BD01200D
:10849000FCE7000038B500F54055044695F8A531D5
:1084A000184A43F0080300F53D5085F8A531022134
:1084B000183054F0A7FA51F021F90122172150F099
:1084C000D5FE2046FFF7B8FF40B104F53A5001222F
:1084D000BDE8384015211830F9F78CBDD5F88C016E
:1084E00003681B689847062806D104F5BE4014307F
:1084F000BDE8384009F008BB20460B21BDE83840F4
:10850000FFF704BFDCBC0D0870B500F54055D5E998
:1085100067239B1A41F288329342064611D9D5F857
:108520008C0103681B6D9847044695F8A531C3F389
:10853000C003A34213D034B13046BDE87040FFF70A
:10854000A9BF0024F1E751F0D9F82246172150F0D5
:108550008DFE95F8A53164F3C30385F8A53170BD90
:108560000B4610B511460446072B07D8DFE803F089
:108570002A041316191C242708F0BAF804F500532E
:10858000D3F8D83C9B061DD504F588500430BDE8CF
:10859000104069F00DBDFFF7B9FEEFE7FFF7ECFE05
:1085A000ECE7FFF7C9FEE9E700F53A500122142194
:1085B0001830F9F71FFDE1E7FFF7FEFEDEE7FFF7F2
:1085C0001BFFDBE710BD0000F8B5044604F50057BB
:1085D00051F094F80122052150F048FE97F88633B7
:1085E000072B98BF304A204694BFD55C0125FFF782
:1085F00023FF68B12D4A2E492046FFF711FE04F5EE
:108600003A50012210211830F9F7F4FC002514E04B
:1086100004F54056D6F88C010368DB6C984798B196
:1086200096F84D3783B196F94C37012B0CDC214A73
:1086300021492046FFF7F4FD012529462046032263
:10864000BDE8F840FFF78CBFD6F88C010368DB6CFF
:10865000984718B1D7F8D83C190715D4D6F88C012B
:1086600003681B689847032803D1D7F8D83CDA077A
:108670000DD4D6F88C0103685B6A984768B90C4939
:108680002046FFF7AFFDD8E70A4A0949D1E70B4A70
:1086900007492046FFF7C4FDB8E7D7F8D83C5B0789
:1086A000EDD5074AF4E700BFBCBD0D08FCBC0D08C2
:1086B0006A910E0806BD0D0819BD0D0829BD0D08EB
:1086C00039BD0D0838B50446154651F017F801229A
:1086D000062150F0CBFD2046FFF7AEFE98B104F521
:1086E0003A50012207211830F9F784FC144A154941
:1086F0002046FFF795FD0025294620460422BDE8C7
:108700003840FFF72DBF04F54053EDB2D3F88C018C
:108710000368DB6C984768B104F50053D3F8D83C84
:108720001B0707D535B1084A06492046FFF778FDF3
:108730000125E1E703492046FFF754FDDCE700BFD0
:10874000FCBC0D0856BD0D0806BD0D082DE9F04115
:10875000044604F5005750F0D1FF0122082150F0E3
:1087600085FD5CF02BFC97F87533072B98BF384AD2
:1087700004F5405698BFD55CD6F8B03193F8CB805D
:1087800088BF0225B8F1000F0BD132492046FFF710
:1087900029FD0025294620460522BDE8F041FFF7C6
:1087A000DFBE2046FFF748FE60B104F53A500122D3
:1087B00012211830F9F71EFC274A26492046FFF7F8
:1087C0002FFDE6E7D6F88C010368DB6C984768B1AB
:1087D00096F84D3753B196F94C37012B06DC1F4AFA
:1087E0001F492046FFF71CFD0125D3E7D6F88C0171
:1087F0000368DB6C984718B1D7F8D83C190713D435
:10880000D6F88C0103681B689847032803D1D7F872
:10881000D83C9A070BD4D7F8D83CDB0609D40D49CD
:108820002046FFF7DFFCB5E70C4A0A49D9E70D4AB5
:10883000C3E7D6F88C010368DB6998470646002831
:10884000EDD1094A03492046FFF7EAFC3546A1E786
:10885000C4BD0D08E1A80D08FCBC0D0806BD0D083F
:1088600050BD0D085EBD0D0873BD0D08F8B500F5CF
:108870000055044695F97533BBB300F54056D6F85C
:10888000107197B38EF022FC05F5536595ED000A43
:10889000DFED167A9FED161ADFED160AC71B20EEE4
:1088A000270A8D2025F0DEFFBCEEC00A10EE103A3C
:1088B0009F420CD296F8A5319A0716D52046002182
:1088C000F9F7F2FC2046BDE8F840FFF7BDBC0CD933
:1088D00096F8A5319B0708D420460121F9F7E4FC5E
:1088E0002046BDE8F840FFF731BFF8BD00007A44EC
:1088F0000000804F000000002DE9F341074600F51D
:108900009B40203085F0AEF907F54054C0F3804815
:1089100001908EF0DBFB94F8A831434545460646AE
:108920000DD007F53D5084F8A8811830002D41D0B6
:108930003B4B3C4AC4F8AC61022154F063F894F814
:10894000A83107F5005843B394F8A9312BBBB8F907
:10895000463D9FED350A9FED351ADFED350A07EEEE
:10896000903AF8EEE77A40F2571027EE800A25F0A9
:1089700079FFBCEEC00AD4F8AC0110EE103A361AFA
:108980009E420AD9012307F53D5084F8A931294AAE
:10899000234B0221183054F035F898F9453D002B4F
:1089A00094F8A5310DDC6FF3451384F8A53102B0BE
:1089B000BDE8F0811A4B204AC4F8AC8184F8A98143
:1089C000BAE7C3F34012AA42F1D065F3451384F825
:1089D000A5319B06EBD5194BD3F88C0103681B69B5
:1089E00098470028E3D050F089FE01221F2150F063
:1089F0003DFC3846FFF720FD48B107F53A5001220B
:108A00002121183002B0BDE8F041F9F7F3BA98F827
:108A1000451D3222384602B0BDE8F041FFF7A0BD47
:108A20008CBD0D089BBD0D0800007A440000804FEE
:108A300000000000B1BD0D08A6BD0D08A05C00201F
:108A400008B5044B01221A708EF038FB024B1860F7
:108A500008BD00BF918E0020948E0020014B0022A3
:108A60001A707047918E00202DE9F04104468EF077
:108A700025FB2A4BB4F8BE201988294E91420546A1
:108A80000ED01A80274B18603378A3B100243470BD
:108A900050F034FE22461321BDE8F04150F0E6BB11
:108AA0003378214FDBB93B782BB11E4B1F4A1B6833
:108AB000C31A934201D8BDE8F0810123337004F555
:108AC0004053D3F8B00190F8CB3013B103689B6AE0
:108AD000984750F013FE0122132150F0C7FB3B785A
:108AE000002BE8D03378002BE5D00E4A10491368EC
:108AF000EB1A8B42DFD904F540541560D4F8B0016D
:108B000090F8CB30002BD6D0002186F065F8D4F851
:108B1000B0010368BDE8F0415B6A1847928E0020FF
:108B2000908E0020948E0020918E002080841E0064
:108B300040420F002DE9F84300F5405500F500587C
:108B40000446D5F88C0198F82C720368DB6C9847C2
:108B5000014650B995F98031002BA5BFD5F8B03149
:108B600093F8CB00012180F0010104F5075909F1C8
:108B7000300948466AF024FAD5F8B03193F8CB3082
:108B80000646002B7BD0002865D03E4B93F9803100
:108B9000002B04DB02463C49484669F0EBFD98F99E
:108BA000F67157B195F98031002B0EDA04F53A5081
:108BB00001220F211830F9F71DFA50F09FFD3246BF
:108BC000BDE8F843092150F051BBD5F88C0103688A
:108BD0005B69984758B195F98131002B07DA95F810
:108BE000A531DA0703D498F82C32DB07DED53146FD
:108BF00048466AF04BFADFED257AB4EEE70AF1EE6B
:108C000010FA05DD0A220921204600F0A3FFD4E76F
:108C1000023F032F11D801A353F827F0058C010858
:108C20002D8C01084B8C0108518C01080A2215215A
:108C3000204600F08FFF0028BFD10A2206212046DF
:108C400000F088FF0028B8D1DCE70A221121F6E7FE
:108C50000A221521F3E797B198F82C327BB9094B1A
:108C600093F98031002B06DB04F53D50084A0521BD
:108C7000183053F0C7FE50F041FD0022A0E7BDE8D8
:108C8000F88300BFA05C0020CCBD0D080000C842E6
:108C9000D5BD0D0870B500F5005300F59B45203596
:108CA00086B093F81C1F0446284684F089FF02A86A
:108CB00014F04EF904F5985002A910300EF01CF88B
:108CC00004F58043049AC3F8982D059AC3F89C2DA7
:108CD000284684F0C7FF82061AD5284684F0D0FFC4
:108CE00004F59B45FDEEC07A103504F5805417EE6F
:108CF000901A0222284617EE906A14F02FF994F881
:108D00008C35DB0706D401223146284614F026F9BB
:108D100006B070BD0121284614F0E4F90028F2D015
:108D2000F6E7000070B500F5A04486B0B4F840380E
:108D30008B420D46164603D1D4F83C38934221D0DD
:108D40008EF0C4F9D4F83838C31A132B1AD9C4F8E2
:108D50003C68A4F84058C4F8380850F0CFFC0446EA
:108D60008EF0BCF9084B094A1B68CDE90453084B47
:108D70000193084B0093CDE90201074B07492046B8
:108D800050F0FEF806B070BD988E0020ECBD0D08C6
:108D900004BE0D0862930D08A8760D08FFBD0D08EE
:108DA00038B500F540540D4694F88131C3F3801373
:108DB0008B420BD021B150F0A1FC112150F036FABA
:108DC00094F8813165F3861384F8813138BD000051
:108DD000F0B52DED048B00F540568BB0D6F8B031D0
:108DE00093F8CB30054600F58044002B67D096F908
:108DF0008031002B63DBD6F88C0103685B699847F0
:108E0000002861D1D4F8BC0D9FED440A6C3028F0E5
:108E10007FFF0AAACDED080A8DED091A8DED070A2C
:108E200012E9070004AB01AF83E8070087E80700F9
:108E3000384628F0B9FCD4F8BC3D05F59A407030AE
:108E4000D3ED368AB0EE409A53F06AF929F05EFB12
:108E5000D4F8C43DD6F88C01D3EDDB9A0368DB6C03
:108E6000B0EE408A9847DFED2E7AB4EEE79AF1EE45
:108E700010FA02DC96F888310BB100283AD0DFED09
:108E8000297A68EEA78AF3EE0E7AF4EEE78AF1EE1D
:108E900010FA2FDCF0EE087AB4EEE78AF1EE10FA61
:108EA00028DCF5EEC09AF1EE10FA23DAD4F8BC0D06
:108EB00003689B6F98470BB0BDEC048BF0BDD4F8F2
:108EC000BC0D03689B6F0FE005F50055D4F8BC0D91
:108ED000D5F87C2D0368B2F90820002A03DCD6F807
:108EE0008421022AEED1DB6F0BB0BDEC048BBDE810
:108EF000F0401847D4F8BC5DDFED0B0A2B68D3F8BF
:108F00008060D4F8C43D40F2AB1093EDC90AB7EECF
:108F1000001A25F0A7FC2846B047CCE79F0CB345C4
:108F20000080BB44E02E65420000000000F5405088
:108F300090F88801704700002DE9F04100F5405598
:108F4000064695F88031B1EBD31F0C4648D0254B2F
:108F500000221A6000293FD050F0D0FB122150F0BF
:108F600065F995F8803164F3C71385F8803184F092
:108F7000010876F07FFB414676F058FB06F5005776
:108F8000B8F1000F06D097F80A331BB98EF09EF89F
:108F9000C7F80C0387F80A8314B3B7F858335B0794
:108FA0001ED5D5F8B03193F8CB30CBB1D5F88C01C4
:108FB00003685B69984798B9D5F88C01036820214C
:108FC0009B69984760B106F53A500122BDE8F0412F
:108FD0000D211830F9F70EB850F090FB1C21BEE7B8
:108FE000BDE8F081988E00202DE9F04F2DED0A8B21
:108FF00000F540558DB0D5F8B03193F8CB6000F551
:10900000A042044601921EB90121FFF795FF0BE033
:1090100095F98021002A66DAD5F88C0103689B6CEB
:1090200098470646002842D04FF0000B95F9802162
:10903000B44E002AC0F25981D6ED007AB4F9A420CA
:10904000B8EE677A1AB9B4F8A220A4F8A420B4F84C
:10905000A430DFEDAD6A07EE903AF8EEE77A67EEFE
:10906000A67AB4EEE77AF1EE10FAACBF0121002146
:109070002046FFF795FE95F98021002A95F8812179
:10908000B8BF4BF0010B5306019B93F8242848BF4F
:109090004BF0020B0AB14BF0080B326859462046E0
:1090A0000DB0BDEC0A8BBDE8F04FFFF73BBED5F825
:1090B000B031204693ED0C8AF9F7C8F9B4EEC80A2E
:1090C000F1EE10FAB0D5D5F8B03193F8A130032BFA
:1090D000AAD14EF0C9FC4FF4801142224EF07CFC24
:1090E0003146204691E7019A92F82498B9F1000F91
:1090F00003D0844A0023136096E700F5804A93F872
:109100000780DAF8BC0D03685B6F9847074600904C
:10911000D5F88C0103685B69984720B1D5F8843194
:10912000022B00F0E480B8F1000F0CBF4FF0000BF1
:109130004FF4007BB7EE00BA17B14BF4806B00968A
:1091400004F59E47503738466DF034F90130DAF8AF
:10915000BC0D9FED6E0A9FED6ECADFED6E8A0CBFEF
:10916000012302236C3008EE103A28F0D1FD0CAB3D
:10917000CDED0A0A8DED0B1A8DED090A13E90700F2
:109180000DF10C0E0DF1180C8CE807008EE80700AD
:10919000704628F009FB04F58042DFED5F7AD2F8D3
:1091A000BC2D92ED36AA2AEE27AAB4EECC0AF3EE35
:1091B0000EBAF1EE10FA04F59A40B4EEEBAAC8BF6D
:1091C0004BF4807B7030F1EE10FAC8BF4BF4807B1B
:1091D000F0EE40AA52F0A4FF29F098F9B8EEC88A40
:1091E00004F59B40B4EEC80AF1EE10FA00F120003D
:1091F00098BF4BF0800BF0EE409A84F04DFD68EE86
:10920000288AB0EEC09AB4EEE89AF1EE10FA204641
:1092100048BF4BF0400B0AF0A9FD002847D14BF0A6
:10922000200BB24638466DF0C5F8012850D14BF0FE
:10923000100BB1463349B8F1000F54D0009B002BFE
:1092400051D0F4EECCAAF1EE10FA4CDCB4EEEBAA5D
:10925000F1EE10FA47DCF4EEC89AF1EE10FA42D8BB
:10926000B4EEE89AF1EE10FA3DD5BAF1000F3AD01B
:10927000B9F1000F37D00A68B4F9A40007EE902ABC
:10928000B8EE677A18B9B4F8A200A4F8A400B4F84C
:10929000A43007EE903AF8EEE77A67EE8B7AB4EEF8
:1092A000E77AF1EE10FA19D501320A60BEE604F54C
:1092B0003650183052F0DCFEDFED187A90ED007A6F
:1092C000B4EEE77AF1EE10FAA9D44FF0000AA9E75C
:1092D00038466DF06FF80130ACD1A8E70121204687
:1092E000FFF72AFEA2E60022DFE70121C0E6B8F17F
:1092F000000FB0EE08BA0CBF4FF0000B4FF4007B2C
:109300001BE700BF988E0020CDCC4C3E9F0CB34590
:109310000080BB440000C842E02E65420000484384
:1093200010B500F5B352044607CA88B002AB83E813
:1093300007009FED1D7ADDED047A77EE877A9FEDC9
:109340001B7ACDED047AD4ED2B7AF0EEE77AF4EEC9
:10935000C77A04F59A40F1EE10FA00F170000BD5CF
:10936000B4F9A22007EE902AF8EEE77AF7EE006A49
:1093700086EEA77A84ED2B7AD4F8AC2001921946B8
:1093800001AA52F09BFF2046FFF72EFE2046FEF773
:1093900043F92046FEF71CFA2046FDF7D1FF204690
:1093A000FEF788F808B010BD0AE81C410000003440
:1093B00010B504462DED028B1D205DF01DFB60B342
:1093C00004F54053D3F88C0100F0C2FA192108EEDD
:1093D000100A04F5546048F097FC02281AD00338AC
:1093E000012808D804F53650183052F041FE90EDAF
:1093F000008ABDEEC88AB8EEC88A9FED090A28EE39
:10940000000ABDEC028B04F59E405030BDE81040D0
:109410006DF056B89FED038AEDE7BDEC028B10BDF1
:109420000AD7233C00000000124A0260124A426040
:1094300002F1740181601149C16002F52A51016194
:1094400008394161243981610D49C1610D490162C9
:1094500002F66461416202F62821816202F62C2143
:10946000C16202F5236102F634224263064A0163B7
:1094700082637047B4D10D08EC4F0020687A002059
:10948000B03F00205C7A0020B82D0020172951D869
:10949000DFE801F0100C1418221F2A1C5026502E51
:1094A00050503236393C40505043474C00F5B040A4
:1094B0004830704700F5BF402030704700F5B1409C
:1094C0000830704700F5B1404430704700F5B940AE
:1094D000F2E700F5BC40F7E700F5BB4038307047D5
:1094E00000F5BB407C30704700F5BE40143070473B
:1094F00000F5B9406030704700F5BA401C30704745
:1095000000F5B540FAE700F5BD40704700F5B840FA
:109510005C30704700F5BF40FAE700F5C0402C30E2
:10952000704700F50050D0F8300C704700F5BA4095
:10953000703070470020704773B50B6805461B6C90
:1095400008460C4616469847034605F53D500F4A17
:1095500000960421183053F055FA50F0CFF82368E4
:1095600005461B68204698470A21024628464FF0C8
:109570007DFE074B93F881319B0641BF054A137866
:1095800043F00403137002B070BD00BF08BE0D08A5
:10959000A05C00203C90002038B50C4A18230546FA
:1095A0000C464EF0ADF878B121462846FFF76EFF25
:1095B00030B10146064A2846FFF7BEFF002038BDFD
:1095C00028464DF0E3FFF9E70120F8E788BE0D08D3
:1095D00028BE0D0810B500F50053002283F82C2E8C
:1095E000094B044693F8801100F5804304F540547C
:1095F000D3F8BC0DC9097EF013F9D4F88C010368C7
:10960000BDE81040DB681847A05C002070B5054637
:10961000086803685B690C461646984790B1306845
:1096200003685B69984768B905F54053D3F8B021E2
:1096300092F8CB2032B193F98031002B02DB28461F
:10964000F8F71AFF04480BF065F920680368BDE8D5
:1096500070409B68184700BF748F002070B500F5FC
:1096600040550446D5F88C010B4E0368DB699847DA
:109670003074D5F88C0103681B689847F070D5F8F2
:109680008C0103685B6C9847014604F595501C30CB
:10969000BDE8704043F058BC1D90002070B52DED22
:1096A000028B244B93F8A531DB0782B006460D46AA
:1096B0001446B0EE408AF0EE608A06D500232B6097
:1096C000236002B0BDEC028B70BD5BF077FD037FC1
:1096D000002BF3D0F36A9FED181A1B689FED170A51
:1096E000B3F9083007EE103AB36A1B68B3F90830D3
:1096F00007EE903AB8EEC77AF8EEE77A67EE000A1E
:1097000068EE811A27EE800A28EE011A01A9684640
:1097100025F09CFFDFED0A6A9DED007ADDED017A10
:1097200027EE267A67EEA67A85ED007AC4ED007AF8
:10973000C7E700BFA05C00200AD7233C5304693967
:109740000000C84270B52DED028B88B00023029353
:109750000393364B93F8A53113F0010F0646B0EE94
:10976000408A06AD02AC03D15BF028FD037F5BB9F4
:1097700094E8030085E803009DED060ADDED070A85
:1097800008B0BDEC028B70BDB36ADFED296A1B68BF
:10979000B3F9083007EE903AF36A1B68B3F9083062
:1097A00007EE103AB8EEC77AF8EEE77A27EE267A97
:1097B00067EEA67AF1EE476ACDED026ADFED1D6A2B
:1097C000CDED037AB0EEC77AB4EEE67AF1EE10FA98
:1097D00006D5F0EEE77AF4EEE67AF1EE10FAC7D4A9
:1097E00003AA21461448F8F777FEDDED027A9DEDD5
:1097F000037AF0EEE77AB0EEC77AF4EE477AF1EE4C
:1098000010FACCBFB0EE670AB0EE470A204627F048
:1098100019FF04A88DED040ACDED050A27F0C4FF59
:10982000204688EE000A27F03DFFA1E7A05C00205B
:109830005304693900000034A02C0020094B93F92F
:109840008021002A0CDAB5EEC00AF1EE10FA07D931
:10985000D3F8B03193F8A100C31E58425841704765
:1098600000207047A05C0020436A1B6893F8CB304F
:1098700043B1054B93F8800100F0A000203818BFD9
:109880000120704701207047A05C002010B5436A9A
:1098900004461868D1B1022185F0AEF9236A9FED24
:1098A0000C1A18680368F0EE410ADB6AB0EE410A50
:1098B0009847236A074A1868D2EDD50A03689FEDD6
:1098C000040A5B6EBDE81040002118470121E3E760
:1098D00000000000A04C002010B5436A0446186840
:1098E000002930D0022185F087F9236A18687DF0BD
:1098F00067FF636A1B6893F8A130012B04D8236AC1
:10990000012118687EF0F6FC6369186881F002FE98
:109910006369186881F05EFE63699FED0C0A186840
:1099200082F084F86369186882F0F2F8236A9FED88
:10993000071A18680368BDE81040DB6AF0EE410AB8
:10994000B0EE410A18470121CDE700BF000000003A
:1099500013B5044601A90C480AF098FA10B1019811
:1099600002B010BD6369186880F0DEFC18B9074BBF
:10997000D3F8940DF4E7064801AA032113F024FB61
:109980000028F4D0EBE700BFA02C0020A06C002042
:10999000307A002070B504462DED028B00296AD183
:1099A0008368B3F96E58642DB8BF6425FFF7D0FF04
:1099B000A8426268A4BF324B93F88151B2F93430A7
:1099C000ACBFC5F380150125002BDBBF63691B68A5
:1099D0005B4293EDC48AC8BF07EE903AB2F93230C9
:1099E000C8BFB8EEE78A002BB8BF5B429BB25B42B0
:1099F00007EE903AA368F8EEE77AB3F96E68F4EEF2
:109A0000C87AF1EE10FAD8BFB0EE678A2046642E0D
:109A1000B8BF6426FFF79CFF6369A26B1B68D2ED99
:109A2000001A93EDC61AD3ED0E0A311A00EE101A81
:109A3000B8EEC00A25F0F8F96368B3F93230002BAC
:109A4000B8BF5B429BB25B4201EE103A40F29720F6
:109A5000B8EEC11AF0EE480A24F004FF6369294603
:109A6000186880F005FDBDEC028B6369BDE87040AD
:109A7000186882F04DB89FED030A0025EEE700BF9D
:109A8000A05C002000000000436A186803681B699E
:109A90001847000038B52DED028B03680446D3F853
:109AA00080309847236B2A481B68F0EE408AB3F950
:109AB00008500AF0FBF84FF47A72041E4FF00001D0
:109AC0002846D8BF4FF4FA7424F00AFF8442B6EE59
:109AD000000A2ADD07EE900AB8EEE77A07EE904A10
:109AE00027EE007AF8EEE77A87EE278A4FF46D705A
:109AF00038EEC00AF5EE087AB1EE400A80EE270A89
:109B0000B7EE001AFEEE000A24F0ACFEF7EE007A83
:109B100077EEC07A28EE000A20EE080A20EE080A46
:109B2000A7EE880ABDEC028B38BD031B07EE103A86
:109B3000C4F57A74B8EEC77A07EE904A27EE007A39
:109B4000F8EEE77A87EE278A38EE008ACEE700BF84
:109B5000A02C00202DE9F0472DED028B00F5A0434D
:109B600000F5405893F8444883F844280546D8F84F
:109B70008C01036882B01B680F4616469847B842AE
:109B800023D105F500531A2E83F8086309D140B993
:109B900005F5804503F60C53D5F8BC2D1B68C2F8BB
:109BA000FC308D4B93F88131980606D40124204671
:109BB00002B0BDEC028BBDE8F087B442F6D0874A14
:109BC000137843F002031370F0E7022E0CD01B2F22
:109BD00012D105F5B1403146443002B0BDEC028BE4
:109BE000BDE8F04701F06AB939462846FFF7D4FCD2
:109BF00004460028EBD1DAE739462846FFF746FC51
:109C00000446019018B928464DF0C0FCCFE7D8F8BB
:109C1000B03193F8CBA003685B699847019A05F5CA
:109C2000B94360338AF001099A4208BF0120BAF1B2
:109C3000000F08D10198036849465B6898470446BD
:109C400048BB674A22E098F98031002B80F2B5804A
:109C5000002800F0B280DFF880A1DAF88C010368F8
:109C60005B6998470446002840F0A7800198FFF7F9
:109C700011FFAAF54050B0EE408AF8F7E7FBB4EECA
:109C8000C08AF1EE10FA40F39880564A01992846AE
:109C9000FFF752FC8BE705F5465101AA0C31284627
:109CA00005F50054FFF7B2FC0198C8F88C0184F860
:109CB000086303681B6898473246014605F57F60D4
:109CC0004EF0E4FE05F53D50002118305AF08AFBB5
:109CD00094F9F63123B105F50750303069F0FAF9FF
:109CE000D8F88C0103681B689847C21E05F58043AD
:109CF0005042504104F6DC4183F84C0ED3F8BC2DA1
:109D00000968C2F8F81004F60C51D3F8BC2D0968A4
:109D1000C2F8FC10012F01D00B2F06D104F6F44439
:109D2000D3F8BC3D2268C3F8FC202846FFF796FC18
:109D3000294B93F881319B063FF541AF36E705F596
:109D4000005393F8F021002A3FF474AFB3F80C22CB
:109D5000D1077FF56FAF93F82C22002A3FF46AAF4A
:109D6000D8F8B02192F8CB20002A3FF463AF93F8E3
:109D700008330A2B7FF45EAF98F98031002BFFF691
:109D800059AF194A01992846FFF7D6FB00240EE780
:109D900016480AF0F5F90028D1D1D8F88C010368EB
:109DA0005B6998470028CAD0019803685B699847A7
:109DB00004460028C3D10E4A68E7019803681B696E
:109DC00098470028E4D009480AF0C8F9044600285A
:109DD000DED1084A5AE700BFA05C00203C9000207A
:109DE00006390F0850BE0D0874BE0D08A02C0020C7
:109DF00062BE0D08EEE90E080148FFF7ABBE00BFDA
:109E0000A02C002013B504468DED010A6CF06AFA0F
:109E10006369A26B1B6892ED001A93ED0E0AD3EDF5
:109E2000C60A01A96BF0ECF89DED010A02B010BD65
:109E3000436A186803685B6A1847000038B5436ACC
:109E40001C6894F8CB10054661B9204684F0D4FE16
:109E50006B6A1B6893F8A10018B1012814BF032096
:109E6000022038BD164803783BBBFFF7E7FC20BB58
:109E7000144A92F8803103F0A003202B17D0B5EEDE
:109E8000C00AF1EE10FA10D592F882315B070CD4BB
:109E90000121204684F0B0FE6B6A1B6893F8A13064
:109EA000012B0CBF02200320DBE70221F1E7204653
:109EB000022184F0A1FE0420D3E70120D1E700BFF6
:109EC000748F0020A05C002010B52DED028B134B89
:109ED00093F8A531DB07044604D59FED110ABDECCC
:109EE000028B10BD5BF06AF9037F002BF5D0636B2A
:109EF00018685BF08DFAA368DFED0A7A03F5156246
:109F000092ED008A03F65413D3ED000A28EE278A57
:109F100025F056FB28EE000AE1E700BFA05C002018
:109F2000000000000000C8420148F8F7FFBA00BF77
:109F3000A02C00200148F8F797BF00BFA02C0020FC
:109F40000148FFF707BE00BFA02C002070B52DED23
:109F5000028B7D4D95F881318CB000260446580661
:109F60000496059603D56369186880F051F895F852
:109F7000A531D9075DD463689B899A071BD57348BF
:109F800052F076F8DFED727A90ED007AB4EEE77A6F
:109F9000F1EE10FA0FDD4FF0B1FB3D214FF046F925
:109FA0006C4809220521FFF7D5FD20B909220221BD
:109FB0002046FFF7C5FF636893F95430CBB365487B
:109FC0009FED658AF8F750FFE3689FED647A1B68A0
:109FD000D3ED0A7AF4EEC87AF1EE10FAB8BFF0EEDB
:109FE000477AB6EE000A27EE800A2046FFF7AAFB62
:109FF0008DED040AB0EEC00AB4EEC80AF1EE10FA14
:10A00000CDED050A06D5F0EEE00AF4EEC80AF1EE51
:10A0100010FA0ED495F882311B0704D44FF06EFB72
:10A0200049214FF003F995F8823143F0080385F890
:10A03000823195F883316FF3820385F8833160694B
:10A0400009960A9609AD2A4604A90068012380F002
:10A0500049F86369186881F0BDFA6369186880F08F
:10A0600095FBA3688DED060ACDED070A8DED081A64
:10A07000D3ED007AF5EEC07AF1EE10FA52DD384BEE
:10A080009FED388AB3F9483300EE903AF8EEE00AD3
:10A090002046CDED030AFFF75BFCA368DDED030A64
:10A0A000D3ED001A9FED2A0AB7EE002A07EE900AB8
:10A0B00031EE822AB8EEE71A22EE082A61EE881AFB
:10A0C00024F010FBDFED287A20EE270ADFED277A57
:10A0D00020EE270AB5F0CAFADFED257A20EE270A2E
:10A0E00006A820EE088A27F05FFBB4EEC08AF1EEE6
:10A0F00010FA17D5C8EE006A63699DED067ADDEDAA
:10A10000077A27EE267A67EEA67A8DED067ACDEDF0
:10A11000077A1B68D3F88823C3F89423D3F88C23D9
:10A12000C3F89823236A13491C682846FCF7CAFA27
:10A130000B9B009395E80C0006A920467DF0F2FBEE
:10A140000CB0BDEC028B70BDA05C0020247A002016
:10A1500000002F44A02C00200000003400007A43AF
:10A16000A04C00200000C8420AD7233C35FA8E3CA0
:10A170000AE81C414C8E002013B504460191FFF7FC
:10A18000E5FE0199204602B0BDE81040FFF702BC91
:10A190000148FEF7D1BE00BFA02C00200048704748
:10A1A000F85B00200148F8F7AFB900BFA02C0020F1
:10A1B00030B50F4D87B0002304466946D5F8C40D6D
:10A1C00000930193029380F0F9FAD5F8C40D02A927
:10A1D00080F048FB009B0393019B04930222029BA7
:10A1E000059303A9204613F0F1F9204607B030BDCE
:10A1F000A06C0020014B01221A7070479C8E002039
:10A2000000207047002070470020704700207047F2
:10A2100000207047002070470020704700207047E2
:10A2200000207047002070479FED010A704700BF73
:10A230000000000000207047002070470020704799
:10A2400001207047002070470020704701207047B0
:10A2500000207047012070470120704700207047A0
:10A260000120704701207047002070470048704768
:10A27000A0BE0D0800487047A0BE0D08836893F883
:10A280006439DB0706D5002380F83C30024B0222FC
:10A29000C3F8842101207047A05C002090F83C3076
:10A2A00043B9836893F86439DB0742BF034B01224B
:10A2B000C3F88421002380F83C307047A05C002064
:10A2C000012380F83C3070472DE9F0432DED0C8BD5
:10A2D000F0EE409A20EE000A97B00025A0EEA00A0A
:10A2E00004468946B0EE41CAF0EE60AA90461F4689
:10A2F000019502950395049505950695B5F0CCFB5F
:10A30000F7EE00CAB4EEEC0AF1EE10FAC8BFCCEEDC
:10A31000807AA36803F5126203F6241392ED009A83
:10A320009FEDC5DAD3ED000AC4BF69EEA79A6AEEC5
:10A33000A7AAB0EE690A25F043F9A36829EE0D9AA1
:10A3400003F5126203F62413D2ED008AD3ED000A5E
:10A3500029EE009AB0EE6A0A25F032F9A36868EE99
:10A360008D8A03F6381203F63C13D3ED000A92ED02
:10A37000008A68EE808AB0EE4C0A25F021F9636805
:10A3800028EE0D8A93F9703028EE008A002B00F039
:10A39000D980236A9FEDA90A18686C3027F0B8FCB1
:10A3A000B0EE60AACDED080A8DED091A8DED070A11
:10A3B00024F002FABDEEC0BAA14940F6B8321BEE55
:10A3C000100A24F07DFA434207EE903A6368F8EEF3
:10A3D000E77A93ED1A7A67EE877AB0EE4A0ACDED06
:10A3E000017A24F0E9F9FDEEC0BA40F6B83294499A
:10A3F0001BEE900A24F064FA42426368039507EE6C
:10A40000902A93ED1B7A93F97030F8EEE77A022BDD
:10A4100067EE877ACDED027A6ED18A4BB3F9483375
:10A420000AEE103AB8EECBBAB8EECAAA236AB4EE76
:10A43000CABAF1EE10FA1A683DDDA368DFED820AB0
:10A44000A16B92ED051AD1ED001A03F5126393ED9D
:10A45000007A27EE0D7A3AEE4B0AC7EE200A24F076
:10A46000E3FCDDED017A37EE800A8DED010AB8EEEE
:10A47000EB0A236AB4EECA0AF1EE10FA1A6834DD68
:10A48000A368A16B92ED061AD1ED001A03F51263D1
:10A49000D3ED000A20EE8DDADFED6B0A3AEE400ACA
:10A4A000CDEE200A24F0C0FCDDED027A37EE800A02
:10A4B0008DED020A20E0B1EE4A0AB4EEC0BAF1EE28
:10A4C00010FAD4D5A368A16BDFED5F0AD1ED001AB5
:10A4D00092ED051A03F5126393ED007A27EE0D7ADB
:10A4E00030EE4B0AC7EE200AB9E7B1EE4AAAB4EE45
:10A4F000CA0AF1EE10FAC3D4236AD3F800C00CF1F3
:10A5000084030FCB12AD85E80F000EAE0AAD86E8CE
:10A510000F0085E80F0004AB01AA294660467DF0D4
:10A520009DFE636893F97030022B16D1DDED047A3D
:10A5300039EE279ADDED057A78EEA78ADDED067A09
:10A5400038EE278A89ED009AC8ED008A87ED008AE7
:10A5500017B0BDEC0C8BBDE8F083F0EEE99AF0EE9D
:10A56000EAAAF4EEE9AAF1EE10FA48BF6D46CDED85
:10A57000009ACDED0AAAD5ED007ADFED340AB0EEEF
:10A58000CCCAF4EECC7AF1EE10FAD8BF35468DED98
:10A590000ECA95ED007ADFED2E7A87EE270AAD2000
:10A5A000B7EE001A3CEEC00A24F05CF9E369D3ED83
:10A5B000937A04A820EE270A27F0AAFBF0EEC07ACF
:10A5C0008DED061AB0EEC91A31EE671A8DED040A48
:10A5D000B0EEC11A39EE000ACDED050AB520F1EE54
:10A5E000410A24F03FF9B0EE409A9DED050AB0EE25
:10A5F000E81AF0EEC07A31EE671A38EE800AB0EE53
:10A60000C11AF1EE410ABA2024F02CF9F0EE408A8A
:10A610009DED060AB0EEC81AF0EEC07A31EE671A68
:10A6200038EE000AB0EEC11ABF20F1EE410A24F064
:10A6300019F9B0EE408A85E70000C8429F0CB34587
:10A6400048F4FFFFA04C002000007A440000000006
:10A6500000A08C4510B52DED028B836A044686B0B0
:10A6600018685AF0D5FEE36A1868B0EE408A5AF0CE
:10A67000CFFE636B8DED010A18685AF0C9FE05AB79
:10A68000B0EE401A03A92046DDED010A04AAB0EE9F
:10A69000480AFFF719FE636A186890F8CB10002982
:10A6A0003AD184F0A9FA2046FFF7F4F9636A1B68EF
:10A6B00093F8A1100129B0EE408A3DD0032944D07F
:10A6C00051B9236A012118687EF0CAFC236A186810
:10A6D0007DF060F89FED208A236AA268186892F8DE
:10A6E000642903689DED030ADDED040A9DED051A5A
:10A6F00092074CBFDB6B9B6B9847236A174A18681D
:10A70000D2EDD50A036800215B6EB0EE480A984787
:10A7100006B0BDEC028B10BD114B93F98121002ACC
:10A7200006DBD3F88431022B04D190F8A1300BB9A9
:10A730000121B6E70221B4E7236A18687EF090FC95
:10A74000236A18687DF03CF8C4E7D9790029C3D1A1
:10A750002046FFF71DFDBFE700000000A04C0020D1
:10A76000A05C0020836893ED140AB5EEC00AF1EEF8
:10A7700010FA01DCFFF788B970470000704700004D
:10A78000002070470120704702207047002070476A
:10A7900000207047012070470020704781F00100C1
:10A7A0007047000001207047012070470048704743
:10A7B00038BF0D080048704744BF0D0838B54369DD
:10A7C000044618687FF0D2FE18B96369186881F0F2
:10A7D00051F8636920461D68FFF7E4FC6368B3F92C
:10A7E0003820B3F9363000EE903A434201EE102A99
:10A7F00000EE103AB8EEC11AF8EEE00AB8EEC00A60
:10A8000028467FF09FFD636920461D68FFF7CAFC5C
:10A810006368B3F93820B3F9363000EE903A43421A
:10A8200001EE102A00EE103A2846B8EEC11AF8EEF2
:10A83000E00AB8EEC00A7FF0FFFD012038BD00003D
:10A8400030B52DED028B0446436985B01D68FFF7D6
:10A85000A9FC6368B3F93820B3F9363000EE903ABA
:10A86000434201EE102A00EE103AB8EEC11AF8EE9B
:10A87000E00AB8EEC00A28465B4D7FF063FD204633
:10A88000FFF758FBB5F9483308EE103A236A186809
:10A8900003689B6E9847B8EEC88AF0EE400A02AA99
:10A8A00001A9B0EE480A2046FEF7F8FE2046FFF761
:10A8B0000BFB236B1B68B3F90830F0EE408A00EE07
:10A8C000103A2046B8EEC00AFFF72EFB2046B0EE45
:10A8D000408A8DED030AFFF765FC6368B3F93630F3
:10A8E00001EE103A434200EE903AB8EEC11AF8EE8B
:10A8F000E00A2B20B0EE480A23F0B4FF20468DED8D
:10A90000030AFFF79BFA042813D8DFE800F0032FAF
:10A91000252A4B00236A18687CF03CFF236A00213B
:10A9200018687DF0E7FC63699FED300A186881F0D4
:10A930007DF8236ADDED020A18689DED010A0368BF
:10A94000B0EE681ADB6A98476369186881F0E0F82E
:10A9500005B0BDEC028B30BD236A012118687DF083
:10A96000C9FC236A18687CF02BFFDCE7204D2B78AC
:10A9700063B963689FED1F1ADFED1C0A93ED040AAB
:10A98000452023F06FFF284609F0ACFF20469DEDDF
:10A99000030AFFF737FA16488DED030A03A909F0F9
:10A9A000DBFFC6E7636A0221186884F025F9B5F970
:10A9B0004833114800EE103A02AA01A9B8EEC00AC5
:10A9C0006AF04EF820469DED030AFFF71BFA0B488C
:10A9D0008DED030A09F078FA63699DED030A1868A2
:10A9E0007FF036FDA5E700BFA04C0020000000006E
:10A9F000748F002000007A44807B0020C05A002021
:10AA00000020704790F8B931002B14BF1B200320A1
:10AA100070470000002070470120704790F89001B7
:10AA2000062804D0A0F10A0358425841704701207B
:10AA300070470000012070470120704790F8B9016D
:10AA4000034A044B002814BF10461846704700BF45
:10AA5000DCBF0D0822FD0E0890F8B901034A044B33
:10AA6000002814BF10461846704700BFE8BF0D0805
:10AA700022FD0E0890F890010B3818BF0120704796
:10AA800090F8B9312BB9044BD3F8280D00F0010030
:10AA900070470020704700BFA04C002090F8903114
:10AAA00023B9034B187880F00100704700207047ED
:10AAB000588F002038B590F89041012C054601D000
:10AAC000002038BDC368186803681B6998470028D0
:10AAD000F6D1EB681B68204683F8B848F1E7000020
:10AAE000C3681B68002283F8B82801207047000063
:10AAF00070B52DED028B002380F8B931B0F87030BD
:10AB0000012B84B004460D4601D8002946D0636A63
:10AB1000254E1B6893F8CB3073BB2448072384F879
:10AB200090310368022B02D10021FBF7D5FB9FED8A
:10AB3000208AE368F0EE480A1868B0EE481AF0EE92
:10AB4000481AB0EE480A012582F0CCFA84ED738AE7
:10AB500084ED748A84ED758A84F8B85104F59A708E
:10AB600027F0BEFD134805F0DBF896F882316FF34D
:10AB7000C30386F8823111E096F98031002BCCDADC
:10AB800004F13C0029F0B6FE05460028C5D1204658
:10AB9000FFF704FB084A022151F034FF284604B0B5
:10ABA000BDEC028B70BD00BFA05C00204C8E00206D
:10ABB00000000000588A0020F0BF0D0810B50446C0
:10ABC000094890F80439012B03D100F5106027F0F3
:10ABD000EFFD064890F8D51E00F65C605DF058F970
:10ABE000002384F8B93110BDA07C0020A06C0020A7
:10ABF00010B52DED028B094B0446D3F8C80DB0EE0D
:10AC0000408A81F0E5FD9FED060A28EE008A0120CA
:10AC100084ED748ABDEC028B10BD00BFA06C0020D7
:10AC20000AD7233C10B52DED028B094B0446D3F80F
:10AC3000C80DB0EE408A81F0DBFD9FED060A28EEDC
:10AC4000008A012084ED758ABDEC028B10BD00BF27
:10AC5000A06C00200AD7233C10B52DED028B094BC8
:10AC60000446D3F8C80DB0EE408A81F0CFFD9FEDC9
:10AC7000060A28EE008A012084ED738ABDEC028B5F
:10AC800010BD00BFA06C00200AD7233CC3681B681E
:10AC900018697FF0ADBE000038B5D0F89431044695
:10ACA0000D461BB98CF012FAC4F894018CF00EFA20
:10ACB000D4F89431C01A4FF47A73B0FBF3F0B4F8BF
:10ACC0009231984209D32046FFF768FA2B88044A4C
:10ACD000062151F097FE012038BD0020FCE700BF9F
:10ACE0000CC00D0890F89031052B05D1054BD3F819
:10ACF000D03DD8687FF0F4BDC36818680368DB688E
:10AD0000184700BFA06C002008B590F89031052BC3
:10AD10000BD1094BD3F8D03DD868243026F044FD40
:10AD2000BCEEC00A10EE100A08BDC36818680368BC
:10AD30009B689847F4E700BFA06C002090F8903122
:10AD40008B4206D00B2B80F8901102D10148FCF702
:10AD5000A5BF7047A02C002073B501231E4E80F8BC
:10AD60007530D6F88C31834205460A4614D1012449
:10AD700085F8B941D6F88C01019203681B689847A1
:10AD8000019A014615484DF081FE96F881319A06E8
:10AD90001BD4204602B070BD01910321FFF7D0F80B
:10ADA000019A04460028E2D185F875004EF0A6FC11
:10ADB0001B220A214EF05AFA96F881319B06E8D5FB
:10ADC000074A137843F0040303E0054A137843F07D
:10ADD00002031370DDE700BFA05C0020903C002060
:10ADE0003C90002030B585B004460D4601466846CB
:10ADF000FFF7DEF9694604F13C002AF02DFBC8B9E3
:10AE00004EF07CFC1B220A214EF030FA0D4B93F8D9
:10AE100081319B0604D50C4A137843F00403137068
:10AE20002046FFF7BBF9094A042151F0EBFD002051
:10AE300005B030BD2946204605B0BDE83040FFF7DB
:10AE40008BBF00BFA05C00203C90002020C00D08FC
:10AE500030B585B004460D4601466846FFF7A8F9AF
:10AE6000694604F13C002AF01BFBC8B94EF046FCD1
:10AE70001B220A214EF0FAF90D4B93F881319B0603
:10AE800004D50C4A137843F0040313702046FFF7EF
:10AE900085F9094A042151F0B5FD002005B030BD07
:10AEA0002946204605B0BDE83040FFF755BF00BF3A
:10AEB000A05C00203C9000205CC00D087FB50546DA
:10AEC0000E4605F13C0401466846FFF771F96946F4
:10AED00020462AF0E5FAC0B9204669462AF0BCFAB5
:10AEE000044690B94EF00AFC1B220A214EF0BEF92E
:10AEF0000D4B93F881319B060FD42846FFF74EF98E
:10AF00000A4A042151F07EFD04E031462846FFF74D
:10AF100023FF0446204604B070BD054A137843F071
:10AF200004031370E9E700BFA05C002094C00D0883
:10AF30003C90002030B5044685B00F4809F00EF96A
:10AF40000546B0B1072384F89031002301930293A2
:10AF50000393E36801A9186881F0D4FBE3681868DB
:10AF6000036801A95B680022984704480021FBF7A9
:10AF7000B3F9284605B030BDA02C00204C8E00202F
:10AF8000F0B5424FD7F89C2DD7F8983D2DED028BA8
:10AF90001343D7F8942D134387B005460C460CD1C4
:10AFA0004CF062FD40F275124FF4801107B0BDEC19
:10AFB000028BBDE8F0404CF00FBD806982F060FE6E
:10AFC0002046B0EE408A11F0F3FF03283AD1EB6837
:10AFD00001A9186881F072FC064698B3DDED017A8C
:10AFE0006368009338EE678A294BDFED2A7A93F97C
:10AFF00080319FED290A2948002BA8BFB0EE670ACF
:10B0000038EE008A009BBDEEC88A002118EE102A97
:10B010009342ACBF00930092FBF75EF96B6918682E
:10B0200080F028FCDDED007A1D48B8EEE70A3146D5
:10B0300009F012FF00212846FFF780FE07B0BDECA3
:10B04000028BF0BD94E80F0002AE86E80F00D7F83F
:10B05000983D04936A46D7F89C3D059302213046FB
:10B0600011F0B2FF78B94EF049FB022215214EF0E3
:10B07000FDF8DDED037AF8EEE77A77EE887AFDEEFB
:10B08000E77ACDED007A0026AEE700BFA06C002085
:10B09000A05C0020000000000000C8424C8E002090
:10B0A000588F002030B52DED028BC36887B0044661
:10B0B00018680D4681F0F6FB00284BD194F89021DA
:10B0C00000230093019302936AB93148039303A9C3
:10B0D0000493059309F0F2FE28B1039B0093049BAF
:10B0E0000193059B029394ED730A9FED2A8AE3680E
:10B0F000DDED000A9DED011ADDED021A1868B4EECF
:10B10000C80AF1EE10FAAABFDFED237A9FED230AF9
:10B1100020EE270A81F0E6FFD4ED747AF4EEC87AC7
:10B12000F1EE10FA07DBE3689FED1B0A186827EEC3
:10B13000800A81F04DFBD4ED757AF4EEC87AF1EE19
:10B1400010FA07DBE3689FED140A186827EE800AFF
:10B1500081F04EFBE3682946186881F0EBFE054656
:10B1600088B10F4B1B68022B09D0032B03D10D4B69
:10B1700093F979331BB10A480021FBF7CDF801217F
:10B180002046FFF7DBFD284607B0BDEC028B30BD43
:10B19000588F0020000000340000C842000000006A
:10B1A0004C8E0020A04C002010B52DED028BC36802
:10B1B000DFED348A1B684269D3ED0A0A9FED328ABB
:10B1C00093ED060AF4EEE80A0446F1EE10FA106870
:10B1D000B8BFF0EE480A7EF09BFEE36862691B6828
:10B1E0001068D3ED0A0A93ED060AF4EEE80AF1EED0
:10B1F00010FAB8BFF0EE480A7EF002FF63691868E3
:10B200007FF092F818B96369186880F0CDF8E368A8
:10B2100062691B68106893ED080A93ED0C1AD3ED70
:10B22000070AB0EEC00A7FF08DF8E36862691B6818
:10B23000106893ED080A93ED0C1AD3ED070AB0EEEF
:10B24000C00A7FF0F9F8636918687FF08FF918B9C0
:10B250006369186880F00EFB00210C48FBF73CF88E
:10B260000B486BF0C5F90B4AB2F8823123F48163C5
:10B27000A2F88231BDEC028B20460221BDE81040CD
:10B28000FFF75CBD0000003400007A434C8E0020C4
:10B29000F07B0020A05C002010B50C4B0446D3F8D6
:10B2A000D00D90ED0B0A90F8502000F11C0180F0B9
:10B2B0002FFF07480368022B02D00821FBF70CF888
:10B2C00020460521BDE81040FFF738BDA06C0020E6
:10B2D0004C8E0020F0B52DED028B4A4DDFED4A8AF1
:10B2E000B0EE408A8FB00446D5F8D00D0E46174612
:10B2F00080F084FDF0EEC87AF4EEE87AF1EE10FA10
:10B3000007D49FED420AD5F8D00D28EE000A80F050
:10B31000DBFDD5F8D00D90ED0B0AB0EEC00A0FB1F1
:10B32000B1EE400A80F0C0FD0023D5F8D00D0793A0
:10B3300002AA07A90893099380F0E2FDDFED347AB1
:10B340009DED027AB4EEE77AF1EE10FA56DD0222B4
:10B3500007A90AA812F03AF971680191304611F074
:10B3600027FE019902460AA811F0F8FDE3680AA930
:10B37000186881F0DFFD10B92648FDF78BF8A06949
:10B3800082F07CFC02684368D5F8D00D049303A9D1
:10B390001C30039226F03AF905A88DED050ACDED93
:10B3A000060A26F001FA1C4B1B68022B1BD0D5F8AD
:10B3B000D03D1948D3ED0A7AF4EEE87AF1EE10FAAE
:10B3C000B8BFD3ED047AF4EEC07AF1EE10FA4FF084
:10B3D000000110D5DFED117AB4EEE70AF1EE10FAB4
:10B3E00009DDFAF799FF04212046FFF7A7FC0FB00B
:10B3F000BDEC028BF0BDFAF76FFFF4E72046FFF7D4
:10B400004BFFF4E7A06C0020000000340000C842AD
:10B4100000009643A02C00204C8E00200000FA4330
:10B4200070B52DED028B294BDFED298AD3F8C84D7D
:10B43000D3F8C45DD4ED0A0A9FED268A94ED060A7E
:10B44000F4EEE80AF1EE10FAB8BFF0EE480A06464C
:10B4500028467EF05DFDD4ED0A0A94ED060AF4EE6E
:10B46000E80AF1EE10FAB8BFF0EE480A28467EF07E
:10B47000C7FD28467EF058FF10B928467FF094FF9C
:10B4800094ED080A94ED0C1AD4ED070AB0EEC00A48
:10B4900028467EF057FF94ED080A94ED0C1AD4ED7F
:10B4A000070A2846B0EEC00A7EF0C6FF28467FF0A5
:10B4B0005DF810B9284680F0DDF907480021FAF759
:10B4C0000BFFBDEC028B0123337070BDA06C00201C
:10B4D0000000003400007A434C8E002008B5074875
:10B4E000D0F8283D9B0704D50121A0F50050F6F7C0
:10B4F00077FEBDE80840024809F00EBBA04C0020D2
:10B50000588F002030B589B00446FEF7ADF930B150
:10B510000021204609B0BDE83040FEF7DDB9636A7E
:10B520000221186883F068FBE368186803685B69A8
:10B53000984701461048FCF799FE6369186880F047
:10B54000E7FA236A1D68636918687FF01FF905AC84
:10B5500020460A498DED020ACDED030A8DED041A4D
:10B56000FBF7B0F8079B009394E80C0002A928466B
:10B570007CF0D8F909B030BDA02C00204C8E002002
:10B5800038B50446FEF770F9054628B1204600217B
:10B59000BDE83840FEF7A0B9636A0221186883F05D
:10B5A0002BFB29462046BDE83840FEF7E5BD0000EC
:10B5B0000148002106F0C2BEB48B002030B5174D03
:10B5C0009FED170A05F5804389B00446D3F8D00DE6
:10B5D00080F038FE01462846FCF748FE636918688B
:10B5E00080F096FA236A1D68636918687FF0CEF8C8
:10B5F00005AC20460B498DED020ACDED030A8DED19
:10B60000041AFBF75FF8079B009394E80C0002A96B
:10B6100028467CF087F909B030BD00BFA02C00207F
:10B62000000000004C8E002030B589B00446FEF7C3
:10B630001BF930B10021204609B0BDE83040FEF7CB
:10B640004BB9636A0221186883F0D6FAE368186878
:10B6500003685B69984701461048FCF707FE636979
:10B66000186880F055FA236A1D68636918687FF0CE
:10B670008DF805AC20460A498DED020ACDED030A8E
:10B680008DED041AFBF71EF8079B009394E80C005D
:10B6900002A928467CF046F909B030BDA02C002054
:10B6A0004C8E002030B52DED028B83B00446FEF7A2
:10B6B000DBF820B9636A1B6893F8CC3043B90021EA
:10B6C000204603B0BDEC028BBDE83040FEF704B964
:10B6D00094F89831DA071DD4E3681D682B68284672
:10B6E0009B689847D5ED097A94F89831B4EEE70A4B
:10B6F000F1EE10FA4CBF0122002262F3000384F83D
:10B70000983107D4204603B0BDEC028BBDE8304031
:10B71000FFF7F8BE94F898319B0734D4E368DFED67
:10B72000458A1B686269D3ED0A0A9FED438A93ED4F
:10B73000060A1068F4EEE80AF1EE10FAB8BFF0EE6F
:10B74000480A7EF0E5FBE36862691B681068D3ED88
:10B750000A0A93ED060AF4EEE80AF1EE10FAB8BF11
:10B76000F0EE480A7EF04CFC636918687EF0DCFD60
:10B7700018B9636918687FF017FE94F8983143F0A0
:10B78000020384F898312D4BD4F8A021D3F8943DCE
:10B790009B1A07EE903AB8EEE78AF1EE047AB0EE23
:10B7A000C87AB4EEE77AF1EE10FA38D594F8983109
:10B7B00043F0040384F89831204684ED678AFEF74D
:10B7C000C5FB6369A26B1B68D2ED001A93EDC61A24
:10B7D000D3ED0E0AB1EE480A23F026FB63691B681D
:10B7E00040F2AA4093EDC31AD3EDC40A23F03AF80D
:10B7F0002046FEF707FB12488DED010A08F064FBB6
:10B8000063699DED010A18687EF022FE636918687D
:10B8100003B0BDEC028BBDE8304080F079B9D4EDC7
:10B82000677A68EE277AF5EEC07AF1EE10FAC3D5A2
:10B83000BCE700BF0000003400007A43A06C002089
:10B84000C05A002030B52DED028B83B00446FEF7C0
:10B850000BF820B9636A1B6893F8CC3043B9002118
:10B86000204603B0BDEC028BBDE83040FEF734B893
:10B870006369DFED347A1B6894ED710A93EDC31AA6
:10B88000D3EDC40A20EE270A40F2C44022F0EAFFBA
:10B890002046FEF7B7FA236A186803689B6EB0EE7D
:10B8A000408A9847284BB3F9483307EE903AB4F8EA
:10B8B000BC316425F8EEE77A13FB05F3B4EEE70A32
:10B8C00007EE103A94F9BE31F1EE10FAD8BFF0EE5F
:10B8D000407A13FB05F39FED1D0AF8EEC76A07EEE9
:10B8E000103AF4EE407AB8EEC77AF1EE10FA58BF8B
:10B8F000B0EE670A6846CDED006A8DED017A25F05D
:10B90000A5FF236ADDED010A1868B4F8C0310268AA
:10B910009DED000A126B13FB05F301EE103A0121B5
:10B92000B8EEC11A90476369B0EE480A18687EF015
:10B930008FFD6369186880F0EBF803B0BDEC028BF3
:10B9400030BD00BF0000C842A04C002000007A4477
:10B950002DE9F0432DED028BB64F85B00446D7F8A4
:10B960008C01FDF781FF48B1D7F88C01002105B0AB
:10B97000BDEC028BBDE8F043FDF7AEBF07F5805686
:10B98000D7F8B001022183F037F9D6F8BC3D93ED2A
:10B99000378A8BF09BFBB7F8803103F4814305466F
:10B9A0007BB1D6F8C40D7EF033FB2378022B08D18F
:10B9B00057F0FCFEA04BA14A062151F023F80323C7
:10B9C000237066F01BFB66F005FB48B166F016FBC2
:10B9D00066F00AFB20B12378012B10D9022B1DD071
:10B9E0002378082B00F28581DFE813F0210039006D
:10B9F00063000A013E0145015A015C012A0057F02B
:10BA0000D5FE8D4B8E4A062150F0FCFFD6F8C43D82
:10BA1000D3F85433636108232370E1E757F0C6FE7F
:10BA2000854B884A062150F0EDFF0323F4E7D6F852
:10BA3000C80D03681B69984710B12046FFF7F0FC5A
:10BA40002378082B00F27381DFE813F05C016401B6
:10BA500064017A017A017A017A0182018201A5608A
:10BA6000D6F8C43D9FED787AD3F854336361774BB1
:10BA700003F66852D2ED007AF4EEC77AF1EE10FACE
:10BA80004EDB9FED737A67EE877AD6F8C83D93ED6B
:10BA9000087AB0EEC77AF4EE477A4FF07E53F1EEB3
:10BAA00010FA48BFB0EE677A2361022384ED067A6C
:10BAB0002370D4ED016A9FED647AD6F8C43DF0EEB0
:10BAC000E67AF4EEC77AF1EE10FA0AD4D4ED057AEC
:10BAD00093EDD56A77EEC67AF4EEE76AF1EE10FAE6
:10BAE00029D4DFED5C6AD4ED067A67EEA67AD3ED51
:10BAF000DB6AF4EEE76AF1EE10FA26DCA368D4ED17
:10BB0000047AEB1AB3F5FA6F21D2B4EE678AF1EE3C
:10BB100010FAC8BFB0EE678A84ED048AE5608FE74B
:10BB2000B3F97E33002BB8BF5B429BB207EE903A6D
:10BB3000F8EEE77AA9E70623237057F037FE3E4B6D
:10BB4000454A042150F05EFF7AE7A56078E7DFF808
:10BB5000FC8008F65C53D3ED006A67EEA67AF4EE3B
:10BB6000C87AF1EE10FAD9D408F55669D9ED007A01
:10BB7000F4EEC77AF1EE10FA22DB98F8903D33B973
:10BB80000623237057F012FE2B4B344AD9E7A8F551
:10BB9000005008F0EBF898B198F9A63D83B9B8F9D0
:10BBA000923DD9ED007ADFED2A6A07EE103A67EE92
:10BBB000A67AB8EEC77AB4EEE77AF1EE10FAADDC09
:10BBC000E068281AB0F5FA7F7FF63AAF03232370B6
:10BBD00008F65C5857F0EAFD98ED007AD4ED047A47
:10BBE00067EE277A054617EE900AF4F795FC124B9C
:10BBF0001B4ACDE900010621284650F003FF1FE74C
:10BC0000D6F8C40D7FF0B2FE66F0F8F966F0E2F9FE
:10BC100068B157F0CBFD084B124A062150F0F2FEF6
:10BC200066F0ECF966F0C4F90423237008E70523F5
:10BC3000FBE700BFA05C0020E0C00D08EEC00D08CF
:10BC4000F8C00D080FC10D0800000034A04C002002
:10BC50000000C842333373BF21C10D083CC10D0839
:10BC60006CC10D0894C10D0866F0C8F966F0B2F910
:10BC7000C0BB05232370404BE068DFED407AD3ED75
:10BC8000006A9FED3F7A2D1AA6EEA77A07EE905A2A
:10BC9000F8EE677AF4EEC77AF1EE10FA3FF5D0AE1F
:10BCA00007232370D6F8C43D9FED367AD3EDC37ACF
:10BCB000D3EDC66A67EE877AB6EE007A67EEA77AAA
:10BCC00067EE877A87EEA67AD4ED057A77EEC77AA3
:10BCD00093EDD57AF4EEC77AF1EE10FA3FF6B0AEF6
:10BCE0000823A2E766F08AF966F07EF90028C0D141
:10BCF000A6E64BF0B9FE40F29C524FF480114BF097
:10BD00006BFE9DE6204805B0BDEC028BBDE8F0431C
:10BD1000FFF7F8BBD7F88C01FEF718F994ED060A87
:10BD20000121B1EE400AD6F8C40D7EF0A1FBD6F891
:10BD3000C40D05B0BDEC028BBDE8F0437FF0E8BE5A
:10BD4000D7F88C01FEF702F99FED100A0021EAE70F
:10BD50009FED0E8AD7F88C018DED038AFEF7F6F879
:10BD6000D6F8C40D0123B0EE480A03AA04F1140169
:10BD70007FF084F9DBE700BF045A002000007A441A
:10BD80000000FA43CDCCCC3D6485002000000000CB
:10BD900030B590F8B83185B00446F3B1684611F07B
:10BDA000D7F8414869460AF0F7FF50B104F13C006A
:10BDB00029F03EFB002384F8B83104F59A7026F090
:10BDC0008FFC94F890310B2B2DD8DFE803F0294B32
:10BDD0004F534B572C5B5F632C6700F59A7026F02E
:10BDE0007FFC04F13C0590B194F84030012B0ED15A
:10BDF00094F89031012B0AD1284629F087F950B1E7
:10BE00002046FEF7CBF9294A022150F0FBFD2846D7
:10BE100029F0AAF9D5E72046FEF7C0F9244AF3E74E
:10BE20002046FFF75BFB94F844303BB994F846306A
:10BE300023B994F840309A1E5342534194F8B921E3
:10BE400082B37BBB84F8B9311A4BD3F88C010368F9
:10BE50001B689847014618482D2205B0BDE83040C0
:10BE60004CF014BE2046FFF74DFBDCE72046FFF701
:10BE700087FBD8E72046FFF79BFBD4E72046FFF778
:10BE80009DFBD0E72046FFF7CFFBCCE72046FFF72E
:10BE900009FCC8E70948FFF75BFDC4E72046FFF748
:10BEA000D1FCC0E705B030BDB03F0020B0C10D08E7
:10BEB000D8C10D08A05C0020903C00209C8E002082
:10BEC0002DE9F0412DED028B074684B008460E4661
:10BED00011F06EF8032880466D4628D1FB6818687B
:10BEE00080F03EFB012822D12148294607F0CEFFF1
:10BEF0000446B0B17B69DDED007A1B68F8EEE77AA5
:10BF000093EDF27A77EEC77A4246FDEEE77A17EEC6
:10BF1000901AC829CDED007AB8BFC821304611F07B
:10BF20001DF8204604B0BDEC028BBDE8F081114B3A
:10BF30000FCB85E80F00304611F03AF8014628464D
:10BF400011F0D0F804460028EBD07B69DDED017AD2
:10BF50001B68B8EEE78AD3EDF27A284638EE678A96
:10BF600011F026F8BDEEC88A024618EE101AD5E781
:10BF7000A02C0020307A002010B543699FED126A92
:10BF80001B68D3EDF06A93EDF17AD3EDF27A86B0C7
:10BF900066EE866A27EE067A67EEC67A68460C4633
:10BFA000CDED006A8DED017ACDED027A25F074FEBB
:10BFB00003A920468DED030ACDED040A8DED051A87
:10BFC00011F058FB06B010BD0AD7233C30B508323B
:10BFD00004461D460FCA84E80F00134301BFAB6837
:10BFE000A360EB68E360636885B093B9204610F006
:10BFF000DFFF03AA0146284610F0E6FF60B103996F
:10C000000191204610F0D4FF01990246204610F01D
:10C01000A5FF204605B030BD696801912846F1E7CB
:10C0200030B50B6985B004460BB94B6953B3002397
:10C03000C4F8B43108310FC96D4685E80F002946B0
:10C040002046FFF73DFF98B9124B0122D3F8941D0B
:10C05000284610F083FF4DF051FB022215214DF0D0
:10C0600005F92046FEF79AF80B4A022150F0CAFC67
:10C0700029462046FFF716F810B90848FCF70AFAD7
:10C0800005B030BD0123C0F8B43105B0BDE8304083
:10C09000FFF78AB8A06C00200CC20D08A02C00206D
:10C0A00070B51A4B04460E460FCB88B06D4685E836
:10C0B0000F0020462946FFF75FFFE368186880F00D
:10C0C000F1FB98B1E368186803681B69984768B189
:10C0D000E3682946186880F057FA38B94BF0C4FC79
:10C0E00040F295624FF480114BF076FC214604A893
:10C0F0002B463246FFF76AFF04A92046FEF7D2FF1F
:10C1000010B90348FCF7C6F908B070BD307A0020BA
:10C11000A02C002070B5154B0C4606460FCB88B0FE
:10C120006D4685E80F0029463046FFF725FF2B4670
:10C130002246314604A8FFF749FF6288A388122AE5
:10C140004FEA132305D1227ED20744BF03EB8303BA
:10C150005B00227A07EE903AC2F34002B8EE670A1B
:10C1600004A93046FFF7B6F808B070BD307A002059
:10C1700038B504460D46FFF793FF0023C4F8943109
:10C18000AB88A4F8923138BD7FB50D460446FFF761
:10C1900087FF05F108010FC96E4686E80F001343BB
:10C1A00006D1234BD3F8982DD3F89C3D02920393EC
:10C1B00004F5D0720121304610F006FF94F8983152
:10C1C00070B923F0050343F0050384F89831204645
:10C1D000FDF7E4FF174A062150F014FC04B070BDCF
:10C1E00023F0070384F898310023C4F89C31E368F6
:10C1F00062691B68106893ED080A93ED0C1AD3ED81
:10C20000070AB0EEC00A7EF09DF8E36862691B6819
:10C21000106893ED080A93ED0C1AD3ED070AB0EEFF
:10C22000C00A7EF009F908212046FEF787FDD5E710
:10C23000A06C002038C20D082DE9F0438DB06D468A
:10C2400088461C46074613460A4601462846DDE94D
:10C250001469FFF7BBFE95E80F0084E80F0007A8FC
:10C2600010F076FEB8F80430F3B9B8F800100131D8
:10C2700005AA89B207F13C0028F0F4FAA0B12346E0
:10C2800005AA39462846FFF7A1FE95E80F0086E883
:10C290000F00BDF81630A3F152025342534189F802
:10C2A00000300DB0BDE8F08394E80F0086E80F0081
:10C2B0000023F4E770B58B8892B004460D4616460D
:10C2C000002B47D10DA810F043FE298801310BAA9D
:10C2D00089B204F13C0028F0C5FA00283AD0BDF834
:10C2E0002E1052291CD019D8112913D80F2913D96F
:10C2F00033462A46214603A8FFF768FE03AB2146D2
:10C3000007A80BAAFFF762FEE36807A9186880F088
:10C3100051FE01E01329EBD012B070BD5E29FAE79F
:10C3200007AD03A810F014FE284610F011FE0DF121
:10C330000B03CDE90053324603AB0BA92046FFF7B0
:10C340007BFFE0689DF80B3000682A4603A980F067
:10C3500007FEE1E70120DFE770B5214B04460E46FA
:10C360000FCB88B06D4685E80F0020462946FFF7C1
:10C3700003FEE368186880F095FA98B1E3681868DE
:10C3800003681B69984768B1E3682946186880F01C
:10C39000FBF838B94BF068FB40F216624FF480119D
:10C3A0004BF01AFB214604A82B463246FFF70EFE3F
:10C3B00004A92046FEF776FE20B90A48FCF76AF881
:10C3C00008B070BD0023C4F89431B388A4F892314A
:10C3D00004AA31462046FFF76DFF0028F0D1ECE7B4
:10C3E000307A0020A02C0020F0B5324B04460E46D7
:10C3F0000FCB91B004AD85E80F0020462946FFF72A
:10C40000BBFDE368186880F04DFA98B1E3681868DE
:10C4100003681B69984768B1E3682946186880F08B
:10C42000B3F838B94BF020FB4FF4DF624FF48011C2
:10C430004BF0D2FA0CAF08A810F08AFD384610F085
:10C4400087FD0DF10F03CDE900732A4608AB314695
:10C450002046FFF7F1FEE0689DF80F3000683A468D
:10C4600008A981F0C3F820B91348FCF713F811B0FC
:10C47000F0BD0023C4F89431B388A4F8923108AA1F
:10C4800031462046FFF716FF0028EDD00B4B1B6806
:10C49000022B09D0032B03D1094B93F979331BB13C
:10C4A00006480021F9F738FF01212046FEF746FC37
:10C4B000DDE700BF307A0020A02C00204C8E002049
:10C4C000A04C002037B504460D468AF0FFFDC4F8A5
:10C4D000A801D5ED027AF5EEC07AF1EE10FA17DD7B
:10C4E0009FED137A67EE877AFCEEE77AC4ED697AFE
:10C4F0002046FDF753FED4F8A4214FF47A73B2FB23
:10C50000F3F30C4A062103B0BDE8304050F07ABA8C
:10C5100066F064F80023009395F90D2095F90E302C
:10C5200095F90C1065F0F6FFC4F8A401E0E700BF30
:10C5300000007A4450C20D0810B5B1F90A30A0F8D5
:10C54000BC3191F90C3080F8BE31B1F90D30A0F852
:10C55000C031B1F90F3007EE903AF8EEE77A0446B1
:10C56000C0ED717A8AF0B2FD0B21C4F8C8012046F3
:10C57000BDE81040FEF7E2BB38B504460D468AF030
:10C58000A5FDC4F8B001D5ED027A9FED047A67EEFF
:10C59000877AFDEEE77AC4ED6B7A38BD00007A4405
:10C5A0004A7C06480B46003A91F91010D3ED030A75
:10C5B00093ED020A18BF0122F9F7B8BE4C8E002095
:10C5C00070B51B4E0446D6F88C01036886B01B6814
:10C5D0000D469847042806D16B88102B0FD0732B7B
:10C5E00020D000201CE0D6F88C0103681B68984717
:10C5F0000328F6D194F89031062BF2D1ECE705F13F
:10C6000008010FC902ACDFED0B0A84E80F0000231C
:10C6100009480093B0EE600A1A46214603F0C2F9B9
:10C6200006B070BD20462946FFF7BAFF0120F7E7A4
:10C63000A05C002000000000588A002038B5D1F826
:10C64000093007EE903AF5EEC07AF1EE10FA0546A1
:10C650000C4605DD0B7A022B03D01ED9032B0ED01E
:10C6600038BD154B9FED150AD3F8C80D27EE800A8B
:10C6700080F0AEF8D4F80930C5F8D031F0E70E4BB1
:10C680009FED0E0AD3F8C80D27EE800A80F0B0F8AF
:10C69000D4F80930C5F8D431E2E7074B9FED070A1B
:10C6A000D3F8C80D27EE800A80F0B0F8D4F809302E
:10C6B000C5F8CC31D4E700BFA06C00200000C84210
:10C6C00038B5114D0C4605F65C6095F8D51E5BF04B
:10C6D000C1FB58B195F8D51E05F65C605BF0C2FB56
:10C6E00020B994ED040A0948F9F7BEFE94ED041A46
:10C6F000D4ED020A94ED030A95F8D51E0448BDE86E
:10C70000384000225BF0E6BBA06C00204C8E00207D
:10C71000FC7A0020F0B50B69214F85B005460E4626
:10C720000BB94B6953B300233B7006F108030FCBE1
:10C730006C4684E80F0021462846FFF7C1FB98B9F4
:10C74000184B0122D3F8941D204610F007FC4CF042
:10C75000D5FF022215214CF089FD2846FDF71EFD6C
:10C76000114A022150F04EF921462846FEF79AFC64
:10C7700038B90E48FBF78EFE05B0F0BD3846FEF71F
:10C780004FFEB38807EE903AF8EE677A0921284603
:10C79000C7ED017A05B0BDE8F040FEF7CFBA00BFA3
:10C7A0009C8E0020A06C002060C20D08A02C0020F0
:10C7B00010B5044C237813B1034869F013FF2078B7
:10C7C00010BD00BF588F0020F07B002000780728A4
:10C7D00094BF00200120704713B5094B0191044616
:10C7E000D3F8C80D03681B69984730B101992046FA
:10C7F00002B0BDE81040FEF74FBA02B010BD00BF56
:10C80000A06C002090F8983113F0010018BFC3F31A
:10C8100080007047094A034692F8510F68B192F8B8
:10C82000502F043A012A07D85B6A1B6893F8A100CD
:10C83000431E58425841704700207047A07C00209A
:10C8400010B504468AF042FCD4F8B031C01AD4F8CE
:10C85000AC3123EAE37398424FF0000084BFC4F880
:10C86000AC01012010BD000010B503680446DB6D6B
:10C870009847D4F8AC3123EAE37398424FF00000B4
:10C880003CBFC4F8AC01012010BD000008B504484D
:10C890000321F9F721FDBDE808400148F9F740BE42
:10C8A0004C8E002070B51C4B0446D3F8C80D0368AD
:10C8B0001B690E469847054610B90025284670BDED
:10C8C000D4F894315BB98AF001FCB4F89231C4F821
:10C8D000940123B1114A537843F0010353708AF055
:10C8E000F5FBD4F89421B4F89231801A4FF47A729F
:10C8F000B0FBF2F09842E0D323B9084A537843F0F2
:10C90000010353702046FDF749FC3388044A062191
:10C9100050F078F8D2E700BFA06C00203C900020D7
:10C920000CC00D0810B590F89031042B0446164B3E
:10C930000AD1D3F8C80D03681B69984718B120467F
:10C94000FEF7AAFC002010BD0A79D3F8D03DDFED38
:10C950000F6A93ED0E6A07EE902A0A7E920748BF8F
:10C960009FED0B7AF8EE677A48BF67EE877A86EE1E
:10C97000267AB0EEC77AB4EEE77AF1EE10FAACBFE1
:10C9800001200020DFE700BFA06C0020DB0FC940C2
:10C990000000803B13B5094B01910446D3F8C80D44
:10C9A00003681B69984730B10199204602B0BDE881
:10C9B0001040FEF771B902B010BD00BFA06C00209E
:10C9C00010B504468AF082FBD4F8A831C01AD4F816
:10C9D000A43198424FF0000084BFC4F8A4010120A4
:10C9E00010BD000038B505460C468AF06FFBD5F83F
:10C9F000C831C01A23894FF47A725343984294BFC6
:10CA00000020012038BD0000C368186808B190F804
:10CA1000B808704710B5012104460A4805F00EF821
:10CA200028B120460321BDE81040FEF787B94BF03E
:10CA30001BF8BDE8104040F26B124FF480114AF031
:10CA4000CBBF00BFB48B002090F89031022B04D0F4
:10CA5000032B04D1034804F0C1BF0120704700201C
:10CA6000704700BFB48B002038B50C4BD3F8285D5D
:10CA700090F89031032B044605F004050AD10848CC
:10CA800004F0C4FF94F8903135B110B9023B58421C
:10CA9000584138BD0020F5E70120FAE7A04C0020FE
:10CAA000B48B002010B50F4A137843F08003137045
:10CAB0000D4B93F98021002A044609DBFEF73AFA70
:10CAC00070B920460822BDE810400921FDF738BAA8
:10CAD000BDE8104001220E21A3F5B470F5F78ABA23
:10CAE00010BD00BF3C900020A05C0020F8B5D0F83D
:10CAF000B44105465CB1012C1AD04AF0B5FF40F6AE
:10CB000043024FF480114AF067FF012407E0184BFD
:10CB1000D3F8C80D03681B69984710B90024204654
:10CB2000F8BD2846FEF740FB0123C5F8B431F6E70F
:10CB3000104F97F98031002BF0DA436A1B6893F8A5
:10CB4000A160012EEAD13C3027F0E2FE0446002825
:10CB5000E5D1D7F8B03193F8CB3033B132460D215F
:10CB6000A7F5B470F5F746FAD9E73446D7E700BF22
:10CB7000A06C0020A05C002038B56E4BD3F88C214F
:10CB80006D4B9A4204460D4601D0002072E04B885E
:10CB90005E2B55D8512B0CD8103B9AB20F2A29D9AD
:10CBA0002046FDF7FBFA6B88644A04214FF02AFF08
:10CBB00059E0523B0C2BF3D801A252F823F000BFEE
:10CBC00017CD0108A1CB0108D9CC0108EDCC010893
:10CBD000A1CB0108A1CB0108A1CB0108A1CB010881
:10CBE000A1CB0108A1CB0108A1CB01081DCD0108F3
:10CBF000F5CC01080F2BD3D801A252F823F000BFC7
:10CC0000E7CC01088BCB0108FDCC010803CD01085E
:10CC100011CD0108EDCC0108D9CC0108A1CB010848
:10CC2000A1CB0108A1CB0108A1CB0108A1CB010830
:10CC3000A1CB0108A1CB0108A1CB010809CD0108B6
:10CC4000732B74D006D8702B6ED0722BA8D1FFF73F
:10CC50000BFE44E04AF2CF62934262D0A0D8B32BDD
:10CC600009D8B12B9CD92046FDF798FA298854F0B1
:10CC7000B5F8012038BDBC3B9AB2132A90D8132BCB
:10CC80008ED801A252F823F067CC010867CC0108C6
:10CC9000A1CB0108A1CB0108A1CB0108A1CB0108C0
:10CCA000A1CB010867CC0108A1CB010867CC010822
:10CCB000A1CB0108A1CB0108A1CB010867CC0108D9
:10CCC000A1CB0108A1CB0108A1CB010867CC0108C9
:10CCD000A1CB010867CC01082046FFF769FD0028B9
:10CCE0003FF453AFBFE7FFF7DDFDF8E72046FFF75E
:10CCF000FDFEF4E71248FFF769FDF0E7FFF712FECB
:10CD0000EDE7FFF769FDEAE7BDE83840FFF77ABDD8
:10CD1000FFF780FDE3E7FFF73DFEE0E7FFF750FE9A
:10CD2000DDE7FFF75FFEDAE7FFF78AFDD7E7FFF7FA
:10CD3000ADFDD4E7A05C00206485002094C20D08FE
:10CD40009C8E002090F89031032B0BD0062B06D040
:10CD5000012B0AD1C368186803681B681847044888
:10CD600002F012BA034804F0C3BE0020704700BFAF
:10CD7000588A0020B48B00208B88012B05D00B69CA
:10CD80003BB94B692BB9CB681BB904480021F9F7B3
:10CD9000DDBE024800220831F9F7FABEA02C0020BF
:10CDA00010B54B885E2B04460A464DD8512B05D84A
:10CDB000103B99B20F2921D900209DE0523B0C2B4A
:10CDC000FAD801A151F823F033CF0108B9CD0108F9
:10CDD000EDCE010803CF0108B9CD0108B9CD010896
:10CDE000B9CD0108B9CD0108B9CD0108B9CD010807
:10CDF000B9CD01083BCF010843CF01080F2BDBD889
:10CE000001A151F823F000BFFBCE01080DCF0108AE
:10CE100015CF01081DCF01082DCF010803CF010850
:10CE2000EDCE0108B9CD0108B9CD0108B9CD010891
:10CE3000B9CD0108B9CD0108B9CD0108B9CD0108B6
:10CE4000B9CD010825CF0108B32B00F0848016D896
:10CE5000732B7DD00ED8702B77D0722BACD1D1ED47
:10CE6000027A9FED447A67EE877AFDEEE77AC0EDAD
:10CE70006B7A40E0B22B9FD1FFF7E0FB3BE0CD2B7C
:10CE80002CD8BB2B98D9BC3B112B95D801A151F8BC
:10CE900023F000BFF7CE0108F7CE0108B9CD010895
:10CEA000B9CD0108B9CD0108B9CD0108B9CD010846
:10CEB0005DCF0108B9CD01085DCF0108B9CD0108EA
:10CEC000B9CD0108B9CD01085DCF0108B9CD010880
:10CED000B9CD0108B9CD010869CF01084AF2CF6286
:10CEE00093427FF469AFFFF727FB04E002F10801EA
:10CEF0002046FEF745F8012010BD1146FFF72CFA39
:10CF0000F9E711462046FFF78BF8F4E71146FFF7E3
:10CF1000C7F8F0E71146FFF7FDF8ECE71146FFF719
:10CF200027F9E8E71146FFF72FF9E4E7FFF772FD6D
:10CF3000E1E71146FFF758FADDE71146FFF7C2FABD
:10CF4000D9E71146FFF7E6FBD5E7FFF715FBD2E778
:10CF5000FFF726FBCFE7FFF70FFFCCE7064802F10C
:10CF60000801F9F7A1FAC6E711462046FFF7A8FB2A
:10CF7000C1E700BF0000C8424C8E0020704700008F
:10CF8000704700007047000090F8280080F0010012
:10CF900070470000024B436040F605030381704771
:10CFA0000001020490F85501704700000F207047FF
:10CFB0000020704700207047002070470020704715
:10CFC0000048704740C30D08004870474CC30D0827
:10CFD00008B5094800F50053D3F87C3DB3F9083093
:10CFE00000EE103AB8EEC00AF5F7A0FABDE8084026
:10CFF0000248FCF707BF00BFA02C00203C870020A0
:10D0000010B514482DED028B1C4600F5005300F5B9
:10D010008040B3F94833D0F8BC0D08EE103A0368ED
:10D0200082B09B6ECDE900219847B8EEC88AF0EE39
:10D03000400ADDE90021B0EE480A0748FCF72EFB64
:10D040000548FCF741FF84ED000A02B0BDEC028BFD
:10D0500010BD00BFA02C00203C870020F8B51C4D5F
:10D0600005F5005405F580462846D6F8C47DF5F749
:10D070004BFAB4F9843301EE103AB4F9823300EE7E
:10D08000903A434200EE103AB8EEC11AF8EEE00AC8
:10D09000B8EEC00A38467DF055F92846D6F8C46D7A
:10D0A000F5F732FAB4F9843301EE103AB4F9823369
:10D0B00000EE903A434200EE103A3046B8EEC11A04
:10D0C000BDE8F840F8EEE00AB8EEC00A7DF0B4B969
:10D0D000A02C002038B5144C04F5804504F57F647D
:10D0E000D5F8BC0D03689B689847692100F194024C
:10D0F00020464BF097F9D5F8BC0D0368DB689847DC
:10D100006A2100F1940220464BF08CF9D5F8BC0D51
:10D1100003681B6998476B2100F194022046BDE823
:10D1200038404BF07FB900BFA02C0020014807F029
:10D1300015B800BFA02C00203C3088F09FB800003C
:10D1400008B54AF091FCBDE8084072224FF4801106
:10D150004AF042BC08B54AF087FCBDE808406622A8
:10D160004FF480114AF038BC08B54AF07DFCBDE8A8
:10D17000084080224FF480114AF02EBC73B51F4D39
:10D180000646D5F88C0103681B6B9847044680B3AC
:10D1900095F98131002B2FDBD5F8B03193F8CB40D6
:10D1A0003CB395F8803103F0A003202B24D1D5F8AF
:10D1B0008C0103681B689847052808D0D5F88C01B6
:10D1C00003681B689847A0F110035C425C410C4A5D
:10D1D00002F55A630193A2F500532146D3F8943E19
:10D1E0000093D2F8C43DD2F8BC2D304687F0F4FF4E
:10D1F0000446204602B070BD0024FAE7A05C00207F
:10D20000A06C00203C30FFF7B9BF000038B5114DCD
:10D2100004461148F5F728FE95F98031002B14DA01
:10D22000236A93F8A120012A06D0D5F88C010021A9
:10D23000BDE83840FCF750BB0D21A5F5B470F4F7FC
:10D24000D9FE95F98031002BEFDB2046BDE8384050
:10D2500088F0FEBAA05C0020A02C00203C30FFF734
:10D26000D5BF0000012070470120704701207047A2
:10D27000012070471120704701207047002070473F
:10D2800000207047002070470048704790C40D0888
:10D290000048704798C40D0838B5436904461D68B6
:10D2A000806980F0F1FC25F031F9DFED1B0A28469A
:10D2B0007CF02EFE6369A0691D6880F0E5FC25F016
:10D2C00025F9DFED150A28467CF09AFE6369186897
:10D2D0007EF06AF86369DFED110A18689FED0E1A97
:10D2E000B0EE600A7DF02EF86369DFED0C0A186875
:10D2F0009FED091AB0EE600A7DF09EF86369186828
:10D300007DF034F918B9636918687EF0B3FA002328
:10D310002364012038BD00BF00803B4400007A43F5
:10D3200070B52DED028B88B00446FCF79DFA70B104
:10D3300020460021FCF7D0FA63699FED310A186896
:10D3400008B0BDEC028BBDE870407EF06FBB636A35
:10D350000221186881F050FC2A4B93F881315B065A
:10D3600003D5636918687CF053FE9FED258A6069D8
:10D370008DED018A8DED028A8DED038A8DED048A93
:10D3800003AA01A9006801237CF0ACFE6369186858
:10D390007EF020F9236A1D682B68DE6C63691868CB
:10D3A0007DF0F4F90122CDED060A8DED071A05A9ED
:10D3B0008DED050A2846B0EE480AB0476369B0EE25
:10D3C000480A18687DF044F8636918687EF0A0FB8D
:10D3D000236C8BB189F07AFEE36BC01A236C984200
:10D3E0000AD309480C220521FCF7B4FB20B90648F2
:10D3F0000C220221FCF7AEFB08B0BDEC028B70BD25
:10D4000000000000A05C0020A02C002038B50446DD
:10D410000D4689F05BFEC4E90F0538BD0720704753
:10D42000012070470020704700207047012070479E
:10D430000048704730C50D080048704738C50D08D2
:10D4400070B52DED028B0025C36880F83C501B6839
:10D45000DFED488AD3ED0A0A42699FED478A93EDD2
:10D46000060AF4EEE80A0446F1EE10FA88B01068F5
:10D47000B8BFF0EE480A7CF04BFDE36862691B68B8
:10D480001068D3ED0A0A93ED060AF4EEE80AF1EE0D
:10D4900010FAB8BFF0EE480A7CF0B2FD636920468E
:10D4A0001E68FCF77FFE6368B3F93820B3F93630A5
:10D4B00000EE903A434201EE102A00EE103AB8EE28
:10D4C000C11AF8EEE00AB8EEC00A30467CF03AFF26
:10D4D000636920461E68FCF765FE6368274CB3F954
:10D4E0003820B3F9363000EE903A434200EE103A5D
:10D4F00001EE102A3046B8EEC11AF8EEE00AB8EE96
:10D50000C00A7CF099FFD4F8D00D7EF01DFED4F84F
:10D51000D06D338B1B0723D504A80FF019FD09F03C
:10D5200057FE9FED170A044606F11C0024F0F0FB9D
:10D5300001AA04A920468DED010ACDED020A8DED68
:10D54000031A09F013FE80B10322294604A80FF044
:10D5500005FD0C4B186804AA90F879105AF0D6FD16
:10D5600009480821F8F7B8FE012008B0BDEC028B8D
:10D5700070BD00BF0000003400007A43A06C0020A2
:10D580000AD7233CCC9900204C8E002030B52DEDDD
:10D59000048BC3689FED898A1B684269D3ED0A7AC0
:10D5A000DFED870A93ED060AF4EEC87AF1EE10FA81
:10D5B0000446A8BFF0EE670A106889B07CF0A8FCAA
:10D5C000636920461D68FCF7EDFD6368B3F93820F8
:10D5D000B3F9363000EE903A434200EE103A01EED5
:10D5E000102A2846774DB8EEC11AF8EEE00AB8EED8
:10D5F000C00A7CF0A7FED5F8D00D7EF021FFA5F57E
:10D60000805393F8A531D90747D4D5F8D03D1A8B6C
:10D61000D20742D593ED0A9AB4EEC89AF1EE10FA09
:10D62000B8BF93ED049AE36A186857F0F1FED5F895
:10D63000C83DD3ED067AA36B20EE270AD3ED007A1E
:10D64000F0EE498AE0EE278AB0EE490AF5EEC08A8C
:10D65000F1EE10FAD8BFDFED5C8AF0EE680A20F038
:10D66000FDFF28B9D5F8D00DB0EE680A7EF02CFC8D
:10D67000636893F95130272B0FD0A36A186857F0CD
:10D68000C7FEF0EEC07AF4EEC87AF1EE10FAB0EE12
:10D69000407A20D5002384F83C30236B1B68B3F913
:10D6A000083000EE103A2046B8EEC00AFCF73CFC09
:10D6B0002046FCF7A7FB2046B0EE408AFCF7D4F8E2
:10D6C000002848D00021204609B0BDEC048BBDE8FD
:10D6D0003040FCF701B9D5F8D03D9FED3C0AD3EDC1
:10D6E0000F7AD3ED0B6AA36B27EE800AF4EEC86ABB
:10D6F000D3ED007AF1EE10FA67EE277A10DB9FED9A
:10D70000341ADFED310A552037EE800A21F0AAF8ED
:10D71000012384F83C30D5F8D00D7EF0C5FBBCE782
:10D720009FED2C7AF4EEC76AF1EE10FA05D89FED62
:10D73000261ADFED290A5920E6E7F0EEE66AF4EE54
:10D74000C86AF1EE10FAE3D594F83C30002B08BF1C
:10D75000B0EE670ADCE7636A0221186881F04CFAD0
:10D760001E4806F0B1FBB0EE480AD5F8D00D7EF0A9
:10D7700069FD01461A48FAF779FD636918687EF079
:10D78000C7F9236A1D68636918687CF0FFFF05AC60
:10D79000204614498DED020ACDED030A8DED041AE1
:10D7A000F8F790FF079B009394E80C0002A9284625
:10D7B0007AF0B8F809B0BDEC048B30BD000000343D
:10D7C00000007A43A06C002000000000E02E6542BB
:10D7D0000000B442000000B40000B4C2C05A0020EF
:10D7E000A02C00204C8E002008B5064BD3F8D03D6D
:10D7F000D868243023F0D8FFFCEEC07A17EE900AE8
:10D8000008BD00BFA06C0020024BD3F8D03DD86803
:10D810007DF066B8A06C00200B2070470120704797
:10D820000020704701207047002070470048704773
:10D83000D0C50D0800487047D8C50D0801207047B5
:10D8400008B5DFED237AF4EEE70AF1EE10FA2DEDDC
:10D85000028BF0EE408AB0EE608A35DDDFED1D7A96
:10D86000F4EEE70AF1EE10FA2ED5F6EE007A70EE3D
:10D87000E77ADFED196A9FED190ADFED190AF0EE7C
:10D88000E77A87EEA67A8720B7EE001A30EE470ACD
:10D8900020F0E8FFDFED137A9FED131ADFED130A96
:10D8A00020EE270A8A2020EE280A20F0DBFF30EE47
:10D8B000080ABDEC028BDFED0A0ABDE808408D20A6
:10D8C000B7EE001A20F0CEBF9FED050AEFE700BFCC
:10D8D000AC1C5A3ED578493F8FC2753E9A99993F04
:10D8E00000000000FAEDEBBA9A99993E9A9999BE18
:10D8F00030B52DED048B7D4BB3F9483300EE903AF3
:10D90000F8EEE00A83B0044601AA6946B0EE600A68
:10D91000FBF7C4FEA06980F0B7F9E369D0ED008A97
:10D92000D3ED946AD3ED977A90ED016AA3689FEDE9
:10D93000701ADFED700A27EEE80A68EEA68A03F691
:10D940003813E6EE278A05463B20DFED6B7AB0EE12
:10D95000E87AB4EEE77AF1EE10FA58BFB0EE677AE3
:10D96000DFED667AC7EE275AF7EE007A77EEE57AB2
:10D970009DED007A67EE877A93ED007A67EE877AFD
:10D980009FED5F7AA6EE260A87EE879A20F06AFF5F
:10D990003C209FED571ADFED570AB0EE408AB0EEFB
:10D9A000680A20F05FFF626B564B1268DFED567A13
:10D9B000B2F90820D3ED006A9FED541ADFED540A46
:10D9C00007EE102AB8EEC77AF0EE408A27EE277AE3
:10D9D000DFED507AA6EEA77A4520F4EE007AA7EEA6
:10D9E000678ABAEE000A28EE000A83ED007A8DED10
:10D9F000000A20F037FFDDED017A9FED477A474BB3
:10DA00008DED000AF0EEE77AF4EEC77AF1EE10FA47
:10DA100051D593ED007ADFED427A77EE277AB2EEB8
:10DA2000007AF4EEC77AF1EE10FA58BFF0EE477ABA
:10DA3000C3ED007A67EEA87ACDED017A636A1868C3
:10DA400090F8CB10002939D181F0D6F8636A1B68B1
:10DA500093F8A110012939D0032940D039B9236A9C
:10DA600018687AF047FC236A186879F093FE236AF5
:10DA7000DDED010A18689DED000A0368B0EE491A51
:10DA8000DB6A9847204695ED028AFCF703F82046AA
:10DA9000F0EE400AB0EE480AFFF7D2FE236A626851
:10DAA0001868D2ED020A036801215B6E984703B043
:10DAB000BDEC048B30BD00221A60BFE7194B93F90F
:10DAC0008131002BB4BF01210221BDE7236A186810
:10DAD0007AF010FC236A186879F072FEC7E7D979EA
:10DAE0000029C4D12046FCF753FBC0E7A04C00201E
:10DAF00000000C4400000CC40000FA4400409C45A7
:10DB000000003442B88E00200AD7233D00A08C4587
:10DB100000A08CC58FC2753F00000034BC8E002071
:10DB20008FC2F53CA05C00200E207047002070479B
:10DB30000020704700207047002070470020704789
:10DB40000048704770C60D080048704770C60D0841
:10DB500070B52DED028B436A1B6893F8CB300446F9
:10DB6000FBB9052384F848302046FBF793FF636A2E
:10DB700002211868B0EE408A81F03EF894F95030E6
:10DB8000E2696BB3D2F8F8515D4394F84820052A56
:10DB90004FD8DFE812F02B005F008400B100DF00F7
:10DBA0001E01836A1B68B3F90830002BB8BF5B42C3
:10DBB0009BB2B3F57A6FD4D2C36A1B68B3F908304D
:10DBC000002BB8BF5B429BB2B3F57A6FC9D289F024
:10DBD0007DFAE36CC01A40F6C4139842C1D8C3E77B
:10DBE00094F95150D2F8FC215543CEE7226A94F9BA
:10DBF000511010689FED801A49F64042534351433B
:10DC000000EE103A00EE901A0268F8EEE00A926B0D
:10DC1000B8EEC00A9047DFED797A41F293139D4246
:10DC200038EE278A05DD94F950308BB1012384F852
:10DC30004830236A62681868D2ED020A0368B0EEC1
:10DC4000480ABDEC028B5B6EBDE8704000211847AE
:10DC50000223ECE7226A9FED681A106849F64042F9
:10DC6000534300EE103A0268B8EEC00A926BF0EE31
:10DC7000410A9047DFED627A38EE678A05F50C5568
:10DC8000B5EEC08AF1EE10FA05F1270543F2BA436A
:10DC9000D8BF9FED598A9D42CBD80423C7E7236A9A
:10DCA0009FED551A186894F9513049F64042534394
:10DCB00000EE903A0268F8EEE00A926BB0EE410A8C
:10DCC0009047DFED4F7AE36938EE678AD3F8F83191
:10DCD000B5EEC08AF1EE10FAD8BF9FED478A002B4F
:10DCE000B8BF5B4242F228329342A2DD41F2941364
:10DCF0009D429EDD03239AE7236A9FED3F1A186831
:10DD000094F9513049F64042534300EE903A02688C
:10DD1000F8EEE00A926BB0EE410A9047DFED387AF8
:10DD2000E36938EE678AD3F8F831B5EEC08A03F5B7
:10DD30000C53F1EE10FA03F1270344F24E62D8BF00
:10DD40009FED2D8A93423FF674AF2E4B9D42FFF616
:10DD500070AFA2E7236A94ED111A1868D4ED100A87
:10DD6000036894ED0F0A1B6B00219847DFED237ABF
:10DD700094F95020E36938EE278A1AB393ED7E7A3E
:10DD8000D4ED0F7AB8EEC77A77EEC77A9FED1E7A98
:10DD9000F0EEE77AF4EEC77AF1EE10FA3FF649AF0B
:10DDA0000D2294F849101948FBF7D4FE024618B921
:10DDB00001461648FBF7CEFE4BF0A0FC16214BF0B7
:10DDC00035FA36E793ED7F7AD4ED107AB8EEC77A5C
:10DDD000DAE70D2294F849100C48FBF7BBFE024627
:10DDE00018B901460948FBF7B5FE4BF087FC022243
:10DDF0000D214BF03BFA1CE700000000CDCC4C3E5F
:10DE00008FC2753E6DEEFFFF0000FA43A02C00208C
:10DE100073B5474D0446D5F88C0103685B6B984792
:10DE200018B90026304602B070BD95F98131002B3B
:10DE30005FDBA36A1B68B3F90830002BB8BF5B42F5
:10DE40009BB2B3F57A6FECD2636A1B6893F8CB6030
:10DE5000002EE6D095F98031002BE2DBD5F88C015D
:10DE600003681B689847002584F8490084F84850E7
:10DE700089F02CF9E36AE064A4F850501B68B3F908
:10DE80000830B3F5967F43DD012384F851304BF021
:10DE900035FC15214BF0CAF9264BB3F9483301EE96
:10DEA000103AE369B8EEC11A93ED7E0A8DED011ABE
:10DEB000F1EE410A5320B8EEC00ACDED000A20F081
:10DEC000D1FCE36984ED0F0A93ED7F0A9DED011A01
:10DED000DDED000AB8EEC00A542020F0C3FCE3696F
:10DEE00084ED100AD3ED807AF8EEE77AC4ED117A6A
:10DEF00098E7D5F88C0103681B689847012890D0F3
:10DF0000D5F88C0103681B689847002891D188E7F1
:10DF100013F5967F01DAFF23B7E7A36A1B68B3F90D
:10DF20000830002BACBF0123FF2384F85030AEE74C
:10DF3000A05C0020A04C00201620704700207047F5
:10DF400000207047012070470020704781F00100D9
:10DF500070470000012070470048704708C70D084F
:10DF600000487047BCA70D0803681BB1007900F09A
:10DF70000100704718467047F0B5494D95F9D56EC8
:10DF800085B00446A5F50055002E00F08580454873
:10DF9000FFF7EAFF064600287ED0636920461F6827
:10DFA000FCF700F96368B3F93820B3F9363000EEB6
:10DFB000903A434201EE102A00EE103AB8EEC11A30
:10DFC000F8EEE00AB8EEC00A38467CF0BBF96369A7
:10DFD00020461F68FCF7E6F86368B3F93820B3F908
:10DFE000363000EE903A434200EE103A01EE102A2D
:10DFF0003846B8EEC11AF8EEE00AB8EEC00A7CF076
:10E000001BFA05F58043D3F8C40D7CF0AFFA18B9BC
:10E01000636918687DF02EFCB5F9A43004F13C006A
:10E020001BB9B5F8A230A5F8A430B5F8A43007EEB6
:10E03000903AF8EE677A04F1980203A90027CDED33
:10E04000037A4EF0A7F804F15C00C4F8A0700190C8
:10E0500070F05EFB002384F8A530B5F9A430019878
:10E060001BB9B5F8A230A5F8A430B5F8A43007EE76
:10E07000903AF8EEE77AB7EE000A80EE270A70F0E1
:10E080006BFB09487FF0FCFDC4F8C870DFED077A30
:10E0900020EE270A84ED310A304605B0F0BD00BFFE
:10E0A000A04C0020705B0020407A00200AD7233C5F
:10E0B00010B50446FBF7B8F92046154B40F83C3B39
:10E0C0004DF0F4FF134B2365134B9FED142A9FED86
:10E0D000141ADFED140A9FED140A6365F1EE041AB9
:10E0E00004F15C0070F04EFB002320460F49C4F899
:10E0F000A830C4F8AC30C4F8B030C4F8B430C4F8B8
:10E10000B830C4F8BC3042F0F5FB204610BD00BF6B
:10E1100010C80D08CDCCCC3D000040400AD7233BB1
:10E1200000803B459A99993ECDCC4C3EA8C70D083E
:10E130002DE9F0432DED028B9BB0914604460D4630
:10E1400088F0C4FFB8499FEDB98A0646A1F10800DE
:10E1500023F05CFA94ED161ACDED110A7E20F1EE53
:10E16000410A8DED100A20F07DFB94ED161A8DED1D
:10E17000100AF1EE410A7F209DED110A20F072FB9A
:10E1800010A904F13C008DED110A4EF021F8A848C9
:10E19000CDED130A8DED120A7FF072FDD4ED327AC7
:10E1A000D4ED140A94ED151AE0EE087A892004F1F2
:10E1B0005C074FF00008B0EE670A20F053FB12A88E
:10E1C00023F070FA9B4812A909F054FA14A93846B2
:10E1D0008DED140ACDED150A70F07AF93846CDF8B8
:10E1E0005880CDF85C8070F0B7F98DED160ACDED52
:10E1F000170AB9F1000F00F001810123C4F8D060C3
:10E2000084F8CC308C4E04F1A80116A823F026FA2D
:10E21000B6F9483300EE103A16A8B8EEC00A23F05B
:10E2200041FA16A9A6F54F6009F010FA18A9284678
:10E230008DED180ACDED190A23F010FAB6F948331E
:10E2400095ED007A07EE903AF8EEE77AB0EEC77AED
:10E25000B4EEE77AF1EE10FA00F3CE8095ED017A94
:10E26000B0EEC77AF4EEC77AF1EE10FA4CBF012394
:10E27000002384F8A530B6F9483395ED000A5A42D8
:10E2800007EE903A00EE902AB8EEE71AF8EEE00AB0
:10E29000CA2020F0E7FA85ED000AB6F9483395ED7B
:10E2A000010A5A4200EE902A07EE903AF8EEE00A90
:10E2B000B8EEE71ACB2020F0D5FA85ED010A94F8E4
:10E2C000A4305A1C84F8A4201422B3FBF2F102FB00
:10E2D0001133DBB2002B34D14BF010FA064688F034
:10E2E000FDFE8046D4F8AC000F46F2F715F9CDE9F3
:10E2F0000E01D4F8A800F2F70FF9CDE90C01D4F81B
:10E30000A000F2F709F9CDE90A016868F2F704F90B
:10E31000CDE908012868F2F7FFF8CDE90601139866
:10E32000F2F7FAF8CDE904011298F2F7F5F8CDE921
:10E330000087CDE90201414B414A424930464AF04B
:10E3400009FE1BB0BDEC028BBDE8F08312A823F0E0
:10E350002BFADFED3D7AB4EEE70AF1EE10FA57D46E
:10E3600094F8CC3063B956E0384670F055F994F81B
:10E37000CC3084ED2A0AC4ED2B0A002B3FF442AFC7
:10E38000DFED325ADFED324A9FED324ADFED323AAD
:10E3900012AA2B4605F10801B2EE0E5AB7EE003A6A
:10E3A000B2EC016A94F99D00B0EEC67A67EE256A78
:10E3B00007EE900A76EE842AF8EEE77AB0EE647AF9
